:020000021000EC
:10C0000000F001206DC3010055C3010057C30100BA
:10C0100059C301005BC301005DC3010000000000C3
:10C020000000000000000000000000005FC30100ED
:10C0300061C301000000000063C3010065C301008B
:10C0400067C3010067C30100F145020067C3010037
:10C0500067C3010067C301007DF3020067C30100ED
:10C0600067C3010067C301002DCA020067C3010056
:10C0700067C3010067C3010067C3010067C3010014
:10C0800067C30100315E0300210E020067C3010097
:10C09000955E030067C3010015F7020067C3010046
:10C0A00067C3010067C3010067C3010067C30100E4
:10C0B00067C3010067C3010000000000000000002A
:10C0C00067C3010067C3010067C3010067C30100C4
:10C0D00067C3010067C3010067C3010067C30100B4
:10C0E00067C3010000000000000000000000000025
:10C0F0000000000067C301000000000067C30100EA
:10C10000000000000000000000000000000000002F
:10C11000000000000000000000000000000000001F
:10C12000000000000000000000000000000000000F
:10C1300000000000000000000000000000000000FF
:10C1400000000000000000000000000000000000EF
:10C1500000000000000000000000000000000000DF
:10C1600000000000000000000000000000000000CF
:10C1700000000000000000000000000000000000BF
:10C1800000000000000000000000000000000000AF
:10C19000000000000000000000000000000000009F
:10C1A000000000000000000000000000000000008F
:10C1B000000000000000000000000000000000007F
:10C1C000000000000000000000000000000000006F
:10C1D000000000000000000000000000000000005F
:10C1E000000000000000000000000000000000004F
:10C1F000000000000000000000000000000000003F
:10C20000344935480A1A02D0072291438D463349F2
:10C2100033480A1A06D00722914381F30988022283
:10C2200082F314882F483049304A00F042F83048F1
:10C230003049314A00F03DF830483149314A00F088
:10C2400038F831483149324A00F033F83148324940
:10C25000324A00F02EF832483249334A00F029F8C9
:10C2600032483349334A00F024F833483349002236
:10C2700000F02AF832483349002200F025F832480D
:10C280003249091A082902DB0022026041601F4876
:10C290001F49884205D00268043003B4904703BCAC
:10C2A000F7E700208646EC4600200021284A904708
:10C2B000FEE7884207D0521A05D0037801300B7090
:10C2C0000131013AF9D17047884202D00270013041
:10C2D000FAE7704700F0012000E8012000F001209B
:10C2E00000F00120F4840300601F0020BC1F002028
:10C2F000A0C30100A0C301008E630300F484030007
:10C30000601F0020601F00203467030034670300B3
:10C3100034670300346703003467030034670300A5
:10C320003467030034670300F4840300508503007E
:10C33000BC1F0020BC1F0020BC1F00200056002096
:10C34000005600200056002000560020005A002011
:10C35000E9C50100FEE7FEE7FEE7FEE7FEE7FEE7D0
:10C36000FEE7FEE7FEE7FEE700F002B8FFF7FCBFDE
:10C3700008484FF00701884385460748804707482B
:10C38000016841F470010160BFF34F8FBFF36F8FFD
:10C39000FFF736BF00F0012069F7020088ED00E0EA
:10C3A00041DF704700B58DB02422002103A819F0A9
:10C3B00089FF01238DF80C3007238DF80F300623F9
:10C3C0008DF81430384903A80AF0EEFA50B30B2860
:10C3D00027D1364B1B6813F4804F03D0344B1B68B6
:10C3E000032B13DC314B1B6813F4804F1AD0304BF6
:10C3F0001B68032B16DD2F4BD3F804352E4A009211
:10C4000050222E49042005F043FD0BE0294BD3F8C0
:10C4100004352B4A00924F222849042005F038FDAC
:10C42000E0E7E0B9214B1B6813F4804F03D0204BA9
:10C430001B68032B18DC012014F06CFFF8B91B4BB0
:10C440001B6813F4804F03D0194B1B68032B1BDCB4
:10C4500000200AF047FA10BB0DB05DF804FB194A42
:10C46000552113F04DFADDE7124BD3F80435164A87
:10C47000009258221149042005F00AFDDBE7114A19
:10C48000592113F03DFADAE70A4BD3F804350F4A85
:10C4900000925B220949042005F0FAFCD8E7094A1A
:10C4A0005C2113F02DFAD7E7BC1F0020741F002079
:10C4B000701F002000100140FC670300A367030009
:10C4C000AC67030034670300386803005868030052
:10C4D00000B583B01F4A04214EF2070005F0BCFCF2
:10C4E0001D4B1B6813F4804F03D01C4B1B68032BA0
:10C4F00014DC19F0D3FCE0B900F052F900F022FA94
:10C50000FFF750FF144B1B6813F4804F03D0134BFD
:10C510001B68032B12DC03B05DF804FB104BD3F84F
:10C520000435104A009266220F49042005F0B0FC41
:10C53000DFE70E4A682113F0E3F9DDE7084BD3F893
:10C5400004350B4A00926F220749042005F0A0FC35
:10C55000E1E700BF2D1E0200741F0020701F0020A5
:10C56000001001407C680300A367030034670300E8
:10C57000B868030000B583B00AF0CFF990B900F0B5
:10C580002FFB00F041F90AF0FBF980B9104B1B6852
:10C5900013F4804F03D00F4B1B68032B0CDC03B04C
:10C5A0005DF804FB0C4A742113F0AAF9E7E70A4A84
:10C5B000782113F0A5F9E9E7084BD3F80435084AC8
:10C5C00000927A220749042005F062FCE7E700BFE9
:10C5D000741F0020701F002034670300001001400A
:10C5E000D4680300A367030008B5FFF771FFFFF7E6
:10C5F000C1FF00210F2000F08BF80222C8210F207C
:10C6000000F09CF8FFF7CCFEFCE700001F280CD9D7
:10C6100000F01F00064BD3F8043523FA00F010F0A9
:10C62000010F0CBF0120002070474FF0A043F2E73C
:10C630000003005070B505460024264606E0084B6E
:10C64000185DFFF7E3FFA04006430134032C04D834
:10C650000123A3402B42F8D0F1E7304670BD00BF64
:10C660001069030008B511B112F078FE08BD12F090
:10C6700065FEFBE770B5054600240BE0094B1E5D27
:10C680003046FFF7C3FF80F00101C9B23046FFF723
:10C69000E9FF0134032C04D80123A3402B42F8D036
:10C6A000ECE770BD1069030010B5144B1B684BB16B
:10C6B000134B1868FFF7DEFF104B1C68013C1C6031
:10C6C00024B110BD002013F00DF9F1E70D4819F069
:10C6D00057FC09E00C4B1968E14001F001010B4BDC
:10C6E000185DFFF7BFFF0134032CEAD80123A340F4
:10C6F000034A12681342F6D0ECE700BFC01F0020C7
:10C70000C41F0020C81F0020E81F0020106903007C
:10C7100070B505460E46002405E03146064B185D0F
:10C72000FFF7A0FF0134032C04D80123A3402B42C0
:10C73000F8D0F2E770BD00BF106903003AB338B516
:10C740000C461346132900D838BD114A10605B000F
:10C75000013B104A1360FFF76DFF0F4B1860002577
:10C76000610CE0034FF47A72002310F5FA7069410E
:10C7700019F046FC01462A46084819F0DFFB00285C
:10C78000E2D10121024B1868FFF7C2FFDCE77047D6
:10C79000C41F0020C01F0020E81F0020C81F002069
:10C7A00010B582B012F046FD40B10024ADF804404F
:10C7B0008DF8064001238DF8053009E012F0E8FC01
:10C7C0000028F2D013F08EF8EFE713F08BF8013465
:10C7D000032C07D801A9094B185D12F035FD00287C
:10C7E000F5D0F2E7064A0121064819F091FB08B995
:10C7F00002B010BD13F076F8FAE700BF106903002D
:10C80000A9C601000C690300002800F082802DE910
:10C81000F04FD1B004463F4B1B6813F4804F03D058
:10C820003D4B1B68032B0BDC3A4B1B6813F4804F0A
:10C8300003D0394B1B68032B2ADC51B0BDE8F08FC5
:10C8400000230F2B0FD8E25C34490D681009590002
:10C850002E5C0FA800F8136002F00F020131AA5CF1
:10C8600042540133EDE70FAA00238DF85C3003F149
:10C87000804303F58833D3F804350292284A0192A5
:10C88000284A009242222849042005F001FBCBE708
:10C89000264BD3F804350D932068020202F47F0280
:10C8A00042EA0062010A01F47F4142EA010CA588D4
:10C8B0002A0292B2E688310289B2277A637A94F822
:10C8C0000AE094F80B8094F80C9094F80DA094F87A
:10C8D0000EB0E47B0B94CDF828B0CDF824A0CDF8B1
:10C8E0002090CDF81C80CDF818E00593049741EA1C
:10C8F0001621039142EA152202924CEA106001903F
:10C900000B4A00920D9B43220749042005F0C0FA10
:10C9100093E77047741F0020701F0020781F0020CD
:10C9200094690300A86903008369030000100140B3
:10C93000B069030060DF704769DF704708B503F036
:10C9400083F808BD10B588B012F08CFE00282DD1F8
:10C95000234B0793079A06920023039304930593AE
:10C960008DF80C3003A90120FFF7E6FF08BB002378
:10C9700004930593F8230393069A03A9A120FFF7D4
:10C98000DBFFC8B906A8FFF7D5FF0446069A079B48
:10C990009A4208D0134B1B6813F4804F03D0124BFC
:10C9A0001B68012B0BDCB4B908B010BD12F09AFF64
:10C9B000CEE712F097FFDAE712F094FFE2E70B4BB5
:10C9C000D3F8043501920A4A0092C3220949022091
:10C9D00005F05EFAE7E7204612F084FFE4E700BFC7
:10C9E000601F0020741F0020701F002000100140F5
:10C9F000786A03005F6A03000620704700B587B0BD
:10CA000044F20103984262D01BD8012836D041F28B
:10CA10000103984276D1474B1B6813F4804F36D000
:10CA2000454B1B68002B32DD444BD3F80435029292
:10CA30000191434A009263224249012005F028FAFD
:10CA400025E044F2020398425CD13A4B1B6813F490
:10CA5000804F1CD0384B1B68002B18DD374BD3F8A8
:10CA6000043510680390526802920191364A009290
:10CA700069223449012005F00BFA08E02D4B1B68B0
:10CA800013F4804F03D02C4B1B68002B12DC4FF0AB
:10CA9000A0434FF4F032C3F81825C3F80C25EFF388
:10CAA000108372B64DF6AD6C284B1B78002B3ED030
:10CAB00030BFF9E7214BD3F8043502920191244AA3
:10CAC000009260221F49012005F0E2F9DFE7194BCF
:10CAD0001B6813F4804FDAD0174B1B68002BD6DD90
:10CAE000164BD3F8043510680490506803900291F7
:10CAF00092680192174A009273221249012005F0B0
:10CB0000C7F9C4E70B4B1B6813F4804FBFD00A4B27
:10CB10001B68002BBBDD094BD3F8043501910E4A8D
:10CB200000927B220749012005F0B2F9AFE707B078
:10CB30005DF804FB741F0020701F002000100140EE
:10CB4000506B0300236B0300746B0300601F002015
:10CB5000346B0300946B0300B86B030000B583B023
:10CB6000014600230093054B01936A4644F20200FC
:10CB7000FFF744FF03B05DF804FB00BFB46B030094
:10CB800010B40346044C006859689A68DB680FC407
:10CB90005DF8044B704700BFEC1F00200D4B0E4AA0
:10CBA00092E8030083E8030003F108020B4903C97C
:10CBB00082E8030093F9062002F00F0242F04002DF
:10CBC0009A7193F9082002F03F0242F080021A7233
:10CBD000704700BFEC1F002060000010A400001090
:10CBE00000487047EC1F002000231F2B09D807497D
:10CBF00001EBC30000224280426001F83320013380
:10CC0000F3E7034B00221A60704700BFFC1F0020AF
:10CC1000FC20002030B405460F4B1B6800240AE0BE
:10CC20001F230E4A12F83300A0B102EBC302528850
:10CC3000AA4207D001341F2C0BD85A1E002BEFD06C
:10CC40001346EEE7054A02EBC30252688A42F1D16D
:10CC500000E0002030BC7047FC200020FC1F0020BA
:10CC600030B40A4A13680A4C04EBC3056880696053
:10CC7000012104F833100B441360202B01D030BC89
:10CC80007047134600221A60F9E700BFFC2000201D
:10CC9000FC1F0020F0B414461D46002300E00133C1
:10CCA000072B0ED81A0108498A5A8242F7D101EBA4
:10CCB0000312D2E90267AF4208BFA642EFD10120BA
:10CCC00000E00020F0BC70470021002030B4C169B2
:10CCD0008269C3880D0A0C06C2F30C01994216D270
:10CCE0005B1A1344A3F50053E41845F10005094A03
:10CCF0001368591C116003F00703808A064A190162
:10CD000002EB03135052C3E9024530BC70475B1A73
:10CD10001344E9E78021002000210020C37D002B7F
:10CD200042D0C3780A7802F0800203F07F031343F5
:10CD30000B7002780B7803F07F0343EAC2130B7089
:10CD40000378002B41D030B48378082B14BF002225
:10CD500001224B7803F07F0343EAC2134B70C5886E
:10CD600003F08003C5F3861423434B708A7802F0E6
:10CD7000030242EA8502D2B28A70057A02F0FC020E
:10CD8000C5F3C10422438A70CB7803F01F0343EA42
:10CD90004513DBB2CB70427A03F0E00302F01F02CE
:10CDA0001343CB7030BC7047C3780A7802F0BF02DF
:10CDB0009B0103F0400313430B70027903F0C0039F
:10CDC00002F03F0213430B70B3E770470023032BBD
:10CDD00031D810B402E00133032B28D8C3EBC302CF
:10CDE000164C04EB021292F84820012AF3D1C3EB4F
:10CDF000C30204EB0212948AC2899442EBD1C3EBC2
:10CE0000C3020E4C04EB0212D2888A42E3D1C3EB78
:10CE1000C30204EB0212B2F8582012B1848AA24273
:10CE2000D9D1C3EBC303054800EB031000E0002099
:10CE30005DF8044B70470020704700BFAC21002014
:10CE4000002300E00133032B16D8C3EBC3020B49C8
:10CE500001EB021292F84820022AF3D1C3EBC3027D
:10CE600001EB0212918A828A9142EBD1C3EBC30398
:10CE7000024800EB0310704700207047AC210020EF
:10CE800008B9042070470820704730B403460C46A8
:10CE90000978C17000214162A1680B2903D8217B68
:10CEA000F9B1012100E0012119700020987029B129
:10CEB000A1680731C9080139597218720121D97561
:10CEC00003F10C056169206985E80300E189998215
:10CED000A1691962217F9975216AD9629A6230BC71
:10CEE00070470021E0E700000021164B1B688B42D1
:10CEF00026D90023144A02EBC10252689A421DD976
:10CF000010B4114A52F8312002EBC30412F8332056
:10CF100082420DD001330C4A02EBC10252689A42A0
:10CF2000EFD80131074B1B688B4205D90023F2E78C
:10CF300060685DF8044B70470020FAE70131D4E7E0
:10CF400000207047842100208821002070B58CB01B
:10CF500006460D4614462C22002101A819F0B2F90C
:10CF60000F238DF80430ADF808604FF0000365F32F
:10CF700000038DF80A308DF80B4001A801F0F6F996
:10CF80000CB070BD30B58DB005460C462C2200218A
:10CF900001A819F097F910238DF8043002958DF847
:10CFA0000C4001A801F0E2F90DB030BD00B58DB024
:10CFB00010B913F1020F06D1074B186803F060FE99
:10CFC0000DB05DF804FB01218DF80410029303926B
:10CFD00001A801F0CBF9EFE790210020F8B5069CFD
:10CFE000002960D01E460F4615685168D2F808C067
:10CFF000D368E5602161C4F814C0A3611569516963
:10D00000E5612162002363700278D20922705AB36D
:10D010000423BB4249D8E17D41B3037803F07F0389
:10D02000E3700023A3709AB143789B0103F4FE538D
:10D03000827843EA9203E3808378DB0003F01803ED
:10D04000C27843EA52132372C37803F01F0363725A
:10D05000002363623378032B21D83278144B53F8C2
:10D060002230E3620020F8BD0123D2E70178C1F34A
:10D070008011E170017801F03F01217142B190F916
:10D080000130002B02DB0423A370CCE70823FBE76D
:10D090000421A1700B44BB42C5D90920E3E77846BF
:10D0A000FFF75CFDD9E70920DDE70920DBE700BFDA
:10D0B000946D030070B50C461D4603789BB10426A1
:10D0C0003244A26000F10C032360836A6360C36A88
:10D0D000E36000232374204604F03AF910B9636931
:10D0E0001E442E6070BD0126EAE72DE9F0418EB0A6
:10D0F0000D4616461C46804600282DD0002D2FD008
:10D10000002C31D0636A0233059304F10C00E378FC
:10D11000002B2DD00121A27801AF3B46082A14BF75
:10D120000022012203F0F1FE0697CDF81C80B2B276
:10D13000ADF820200B9515440C95A3788DF834306C
:10D14000237B022B16D00023ADF8283005A803F06E
:10D15000D4FE0EB0BDE8F0817846FFF7FFFCCDE7C6
:10D160007846FFF7FBFCCBE77846FFF7F7FCC9E70B
:10D170000221D0E723692BB1236909931023ADF86D
:10D180002830E3E77846FFF7E9FCF5E72DE9F041C1
:10D1900088B004460D46C37D002B3CD0082605FB15
:10D1A00006F8637AAB4238D0257201AB324602A949
:10D1B0002046FFF77FFF074648BB4DB994F8533030
:10D1C00033B9A369C3F30C03E380012384F853301C
:10D1D000E37D7BB994F8523063B91DBBE06EB4F8BF
:10D1E0004A10A27823468A1A0146FFF77EFF0123E0
:10D1F00084F8523007992046FFF790FDE16E3246E1
:10D200004144019819F035F802A804F0C7F83846EF
:10D2100008B0BDE8F0810C26C1E7B4F84A60A6EB7F
:10D220000806C1E77846FFF799FCD7E770B50546D1
:10D230000E4609B100230B6095F85040002104E030
:10D24000631C85F850300134E4B26B7AA34210D3EA
:10D25000EA6C0123A3401A42F5D121462846FFF784
:10D2600095FF014628B9002EEAD0336801333360B8
:10D27000E6E7084670BDF0B589B004460E4615468F
:10D2800083789A18C37D63B10B239A4221D801ABEE
:10D2900002A92046FFF70EFF074620B1384609B025
:10D2A000F0BD0F23F1E707992046FFF737FDE37D37
:10D2B00043B12A463146019818F0DBFF02A804F07A
:10D2C0006DF8EBE723462A4601993046FFF70DFF3C
:10D2D000F4E70927E2E7000010B5044690F848306B
:10D2E000012B0CD102F08EFE237B012B0BD0094BBE
:10D2F000D968014404F1300002F050FE10BD7846B8
:10D30000FFF72CFCEEE7A17D024BDA681B6903FBFB
:10D310000121EEE79421002030B583B0002403E022
:10D320002846FFF7D9FF0134032C18D8C4EBC403F7
:10D330000C4A02EB031393F84830012BF3D100237E
:10D340000193C4EBC40502EB051501A92846FFF7BC
:10D350006DFF0428E4D0019B002BE4D0E0E703B08C
:10D3600030BD00BFAC21002038B5044690F84830ED
:10D37000022B09D1064B1D6802F044FE411904F14D
:10D38000300002F00BFE38BD7846FFF7E7FBF1E70F
:10D390009421002038B5044690F84830022B10D173
:10D3A0000A4B5D7D5A689B6803FB052502F02AFE47
:10D3B000411904F1500002F0F1FD012384F86830B6
:10D3C00038BD7846FFF7CAFBEAE700BF942100208A
:10D3D00010B50446808A02F07FF901281CD1237B16
:10D3E000E3B194F91620002A1ADBE27D4AB1022B40
:10D3F00018D094F90330002B16DBA378B3B90020C2
:10D400000BE0E2780AB9012B12D1237893B9A37803
:10D41000042B11D1002000E0102010BD1020FCE7EB
:10D420000720FAE71020F8E70720F6E70720F4E7DF
:10D430000720F2E70020F0E70720EEE738B50446C2
:10D4400003784BB1C388C2698169808A05F030F9DD
:10D45000054645B9284638BDC2698169808A05F00C
:10D4600021F90546F5E7E169002201F00101A08AF2
:10D47000FFF76CFDEEE700002DE9F04780460E4611
:10D4800017464B1EDBB2012B0FD8B7F5C07F10D863
:10D490000024032C1AD8C4EBC403314A02EB031353
:10D4A00093F848304BB10134F3E77846FFF756FB69
:10D4B000EBE77846FFF752FBEAE7C4EBC40502EB63
:10D4C0000515384607F011F8E86600E000255DB361
:10D4D000EB6E002B42D043462C4608F1300ED3F8B9
:10D4E00000C058689968DA68C4F800C06060A1603C
:10D4F000E260103310347345F1D10023EB64A5F8DA
:10D500004A70012E13D06FF00103AB62002385F83F
:10D510006830144BAB652D66134BAB632D64012053
:10D5200001F02CFE85F848602846BDE8F0870F4BD7
:10D530001B7D85F85130002385F8523085F8533033
:10D5400085F85030D8F828206A65A5F858306FF073
:10D550000103AB62064BAB632D64E0E71D46E3E7D6
:10D56000AC21002077DF0100C1D801009421002008
:10D570000DD9010000B585B000228DF80F20A0B1B3
:10D580000B46024602320A600DF10F01184603F005
:10D59000B8FC9DF80F3043B10C4B1B6813F0040F1F
:10D5A00003D00B4B1B68032B04DC9DF80F0005B068
:10D5B0005DF804FB074BD3F80435074A009240F2AC
:10D5C00015420649042004F063FCEEE7741F0020B6
:10D5D000701F0020001001404C6C03003D6C0300E4
:10D5E0002DE9F04391B005460E4614461F46D0F88B
:10D5F000188003784BB1C388C8F30C029A4230D22A
:10D600009B1A4344A3F50053AB6105F10C00EB7882
:10D6100053B30121AA780DF130094B46082A14BFF3
:10D620000022012203F071FCC5F81880CDF810909B
:10D630000596AB78E21A92B2ADF8182032440A92FD
:10D6400009978DF82C300023ADF82030EB78002BB3
:10D6500040D02B7B022B09D000236B6201930293F5
:10D6600024E09B1A4344CFE70221D3E71023ADF80F
:10D6700020302B690793EFE70134012C14D810AB4D
:10D6800003EB840353F83C0C70B103A9FFF772FF5E
:10D690000028F1D010AB03EB840454F83C3C6B62DF
:10D6A000002011B0BDE8F083019B3BB102AB01AAA1
:10D6B0002979286A0EF094FB0024DEE72B7B022BED
:10D6C0002CD105F10C01E8890EF044FC0028C0D1F2
:10D6D0000520E6E72B7B012B01D00520E1E7EB8954
:10D6E000ADF80430AB8AADF806300024012C13D815
:10D6F0002946002341F8243F10AB03EB440333F8E1
:10D700003C0C0EF092FB03A9686AFFF733FF08B9DF
:10D710000134EBE70020C4E70520C2E70520C0E79D
:10D7200070B5F0B00E4614461D4610AB0A460146D1
:10D730002046FFF755FF50B1214B1B6813F0040F33
:10D7400003D0204B1B68052B2DDC70B070BD20462C
:10D75000FFF774FE0028F8D103AB01228DF80C20EE
:10D76000A28AADF80E20002204928DF8142010AA8F
:10D770000692A178711AADF81C1008AA93E803006C
:10D7800082E803000AAB2169E06883E80300A37D17
:10D790008DF83830236A0C93636A0D930F9505A8B2
:10D7A00000F0E4FDD1E7084BD3F80435074A0092B6
:10D7B00040F203720649062004F06AFBC5E700BF89
:10D7C000741F0020701F002000100140606C0300D7
:10D7D0003D6C030010B50446C06E06F08AFE04F1ED
:10D7E000300002F0C3FB94F84830022B0AD07022BC
:10D7F0000021204618F066FD002084F8480001F062
:10D80000BDFC10BD04F1500002F0B0FBEFE710B515
:10D810008CB0044690F84830012B0FD101238DF8CD
:10D820000430636D029302F0EDFB039001A800F059
:10D830009DFD2046FFF7CEFF0CB010BD7846FFF7E8
:10D840008DF9EBE730B585B00D460446A8B194F8E4
:10D850004830022B15D02946606DFFF793FB204618
:10D86000FFF7B8FF114B1B6813F0040F03D0104BE8
:10D870001B68032B09DC05B030BD7846FFF76EF955
:10D88000E5E72046FFF722FAE5E70A4BD3F804352F
:10D8900094F8482002950192074A009240F2F31250
:10D8A0000649042004F0F4FAE5E700BF741F0020E5
:10D8B000701F0020001001408C6C03003D6C0300C1
:10D8C00008B508460021FFF7BDFF08BD08B5037B7A
:10D8D000012B02D0FFF79BFF08BD0121FFF7B2FF2C
:10D8E000FAE7000008B590F8513053B1013B80F8D9
:10D8F0005130002380F85030034B186803F0C0F912
:10D9000008BDFFF7E3FFFBE79021002010B50C46B0
:10D9100091F84830012B03D12046FFF7E3FF10BDFB
:10D920007846FFF71BF9F7E7062976D1F0B585B001
:10D9300015460678B20102F4FE5241788478C37825
:10D940001B0443EA0463047943EA042344791C4337
:10D9500076B242EA91012846FFF738FA0746E0B16D
:10D96000002E2FDBC289A98A8A422BD02B4B1B6841
:10D9700013F0040F3ED02A4B1B68012B3ADD294BD4
:10D98000D3F8043502910192274A009240F27D6259
:10D990002649022004F07CFA2CE0204B1B6813F08F
:10D9A000040F27D01E4B1B68012B23DD1D4BD3F822
:10D9B00004351F4A009240F279621C49022004F0AB
:10D9C00067FA17E0002E17DBFD6C2543FD64BCB140
:10D9D0003B78D3B17B7A5A1C01239340013B9D4293
:10D9E00017D0002187F850103846FFF71FFC384643
:10D9F000FFF772FC05B0F0BDAB8AA7F85830E3E73B
:10DA000003213846FFF71EFFF4E77846FFF7A6F834
:10DA1000E0E73846FFF7FBFEECE77047741F002095
:10DA2000701F002000100140E06C03003D6C0300FB
:10DA3000B06C03002DE9F0418AB007460E4614464B
:10DA40001D461046FFF7FAFC50B994F80380B8F170
:10DA5000000F08D12B46224631463846FFF764FFB7
:10DA60000AB0BDE8F0814046FFF73EFA02460028C2
:10DA7000F6D08DF80480236A0793A38AADF812309C
:10DA800005AB2169E06883E80300A37D8DF82030B1
:10DA90000297039623788DF81030E36A099329469C
:10DAA00001A89047DCE710B5547814F0010F03D0BB
:10DAB000D47D14B1FFF7BEFF10BDFFF731FEFBE7C9
:10DAC00008B501390130FFF7EEFF08BDF0B5C7B06A
:10DAD0000F46164682783244C37D2BB14FF48073D3
:10DAE00093427CD3002303E04FF4C073F8E7013383
:10DAF000032B1AD8C3EBC3043B4D05EB041494F875
:10DB000048100129F3D1C3EBC30105EB01118C8A45
:10DB1000818A8C42EBD1C3EBC30105EB0111CC89A7
:10DB2000C1898C42E3D1082552E00121FFF7A4FC12
:10DB30000446002855D032463946C06E18F099FB8D
:10DB40000023459345A92046FFF770FB054608B121
:10DB5000042840D1459B0BBB244B1B6813F0040FDA
:10DB600035D0234B1B68032B31DDB4F84A70802F6E
:10DB700028BF80270023BB4214D2E26ED25C1D492D
:10DB80000D68100959002E5C04A800F8136002F01B
:10DB90000F020131AA5C42540133ECE72046FFF743
:10DBA0009BFBD9E704AA002302F8173003F1804356
:10DBB00003F58833D3F8043502920F4A01920F4AD5
:10DBC00000924FF4AC620E49042004F061F9002584
:10DBD000284647B0F0BD2046FFF7FCFDF8E70925D1
:10DBE000F6E70425F4E700BFAC210020741F0020F5
:10DBF000701F0020781F0020246D0300A869030017
:10DC00003D6C030070B504460D461646FFF7E0FB79
:10DC100030B923782BB1324629462046FFF756FF0C
:10DC200070BD324629462046FFF725FBF8E7000085
:10DC300038B504460D46CB695B780371CB691B7818
:10DC400083F00103C370CB6943628B8A0B2B07D827
:10DC5000CB7A002B35D10B7B012B02D0002300E0C7
:10DC600001232370002B31D0287B02282BD0FFF713
:10DC700007F9A070AB8A03440B33174A82FB0323D6
:10DC80005B10013B6372002323720023E37504F1F0
:10DC90000C0395E8030083E80300AB6923622B893A
:10DCA000A382AB7AA3752B6AA362DF23E3622846C3
:10DCB0000EF07EF920B12B78012B0AD0FF23E3620E
:10DCC00038BD0123CDE7054B987DD0E70423A37031
:10DCD000DBE72023F3E700BFABAAAA2A94210020A8
:10DCE00010B54FF4E0720021134818F0EBFA04F07D
:10DCF000ABFC0024114B1C6080222146104818F018
:10DD0000E1FA104B104A1A60104A5A604CF2503235
:10DD10009A600F49D9601A6104221A759C7508220D
:10DD20005A750C4802F08CFF0B4B18600B4B1C60B3
:10DD30000B4804F083FF10BDAC210020802100209F
:10DD4000002100209421002080969800F0490200D4
:10DD500020A1070069DF010090210020842100201C
:10DD6000ADCF010008B504F08FFC08BD98B110B527
:10DD70008CB00446036983B1C36983B1836983B1FD
:10DD800001466846FFF754FFA28A21696846FFF7FB
:10DD900039FF0CB010BD0E2070470E20F9E70E20A1
:10DDA000F7E70E20F5E7000058B310B590B00A462B
:10DDB000044643683BB383693BB3014604A8FFF7BD
:10DDC00064F8134B1B6813F0040F03D0114B1B684E
:10DDD000062B06DCA268616804A8FFF713FF10B0E9
:10DDE00010BD0D4BD3F804352278A1690291019240
:10DDF0000A4A009240F605020949072004F048F853
:10DE0000E8E70E2070470E20E9E70E20E7E700BFA5
:10DE1000741F0020701F002000100140346D0300AB
:10DE20003D6C0300037B012B01D00020704730B50F
:10DE300091B004460D46334B1B6813F0040F03D01A
:10DE4000314B1B68032B41DC04A900230593CDF85B
:10DE50001730E288C2F3861092008DF811202A0E46
:10DE60008DF812202A0C8DF813202A0A8DF8142020
:10DE70008DF815506278022A0CBF80221A4642EAB9
:10DE800000028DF810204FF0060209924FF00102B7
:10DE90008DF82C20A28AADF82E200C938DF81C3022
:10DEA0000891226A0D928DF82830E36A0F9319D0F9
:10DEB000E389ADF82A30A37DF3B98DF838306FF0DF
:10DEC000010107A8FFF770FF11B030BD0F4BD3F869
:10DED00004350F4A009240F263220E49042003F0F9
:10DEE000D7FFB1E70DF10E0103A80EF04FF8BDF812
:10DEF0000C30ADF82A30DEE7074B5B7D8DF838300B
:10DF0000DDE700BF741F0020701F002000100140DB
:10DF1000606D03003D6C03009421002090F84830B0
:10DF2000022B00D0704710B5044690F86830022BE1
:10DF300000D010BDC16CFFF775FF0028F9D1002398
:10DF400084F86830F5E7000010B5002407E0C4EB62
:10DF5000C402130103481844FFF7E0FF0134032C07
:10DF6000F5D910BDAC21002008B5FFF7D5F9FFF7B2
:10DF7000EBFF012008BD10B50C4691F84830022B8C
:10DF800006D1022384F868302046FFF7C7FF10BD92
:10DF90007846FEF7E3FDF4E7F0B583B00446C569C3
:10DFA0008269C3882F0A2E06C2F30C05AB4232D910
:10DFB0005B1B1344A3F50053F61847F100073246E4
:10DFC0003B46A08AFEF766FE002840F08B80204684
:10DFD000FEF736FF054648B3D0F81CC08269C388F7
:10DFE0004FEA1C214FEA0C60C2F30C0C9C4515D281
:10DFF000A3EB0C031344A3F50053C01841F1000137
:10E00000B94208BFB0420DD38F4208BF864230D319
:10E01000284603B0F0BD5B1B1344CDE7A3EB0C0314
:10E020001344EAE705212846FFF70CFCE388E26980
:10E03000A169A08A04F00EFCE8B9627A531CE17D64
:10E0400099B3082202FB03F289B34FF48073934221
:10E0500030D302212046FFF70FFA05460028D7D11A
:10E0600000212046FFF7DEFE02210020FEF78AFF96
:10E07000CEE70025CCE7E388E269A169A08A04F035
:10E0800061FC60B1237863B1617A4B1C0121994036
:10E0900001392046FFF7C6FE2046FFF7CFF90025DD
:10E0A000B6E77846FEF75AFDEEE70C22CAE74FF4D2
:10E0B000C073CCE70C4B1B6813F0040F03D00B4B61
:10E0C0001B68002B01DC0025A2E7094BD3F80435BF
:10E0D0000192084A009240F27F320749012003F082
:10E0E000D7FEF0E7002593E7741F0020701F002083
:10E0F00000100140706D03003D6C03002DE9F041FC
:10E1000082B007460E46144698461046FFF744FF75
:10E11000002846D00546404B1B6813F0040F03D07F
:10E120003E4B1B68032B3FDC2846FFF71DF92B7B7A
:10E13000012B47D0EB6C217A01228A40134230D167
:10E140001A43EA64043E237AE27D002A42D04FF06B
:10E15000080C0CFB03FC697A8B423ED0002A41D0AC
:10E160000823B34240D1AA69A3699A4209D205F1B2
:10E170000C0E0C340FCCAEE80F0094E803008EE8D0
:10E180000300E86E3246391D604418F072F8EC6CFA
:10E190002B7873B36B7A5A1C01239340013B9C424A
:10E1A0002BD002B0BDE8F0811D4BD3F80435227AA4
:10E1B00001921C4A009240F2A3321B49042003F052
:10E1C00067FEB1E795F86830002BB3D12846FFF71A
:10E1D000E1F8AFE74FF00C0CBBE70CEB0603A5F83A
:10E1E0004A30C0E70C23BCE704212846FFF72AFB8E
:10E1F000D7E77846FEF7B2FCCCE7E96C2846FFF794
:10E2000011FE43462A46B5F84A10E86EFFF74BFC6C
:10E210002846FFF7DFFAC4E7741F0020701F0020B4
:10E2200000100140846D03003D6C03002DE9F041B6
:10E2300090B000284CD00F4614461E468046002A57
:10E2400048D004AB00933346FEF7C8FE054618B12C
:10E25000284610B0BDE8F08104A8FFF7B9F80546DC
:10E260000028F5D100230293039302A960880DF0E2
:10E2700071FE28B19DF8113043F001038DF8113083
:10E280002269E168208904F09DFA38B19DF81130C7
:10E2900003F0FE038DF81130002BD9D09DF811301A
:10E2A000002BD5D013F0010F01D0039B08939DF8EC
:10E2B000103033B1334604AA39464046FFF71EFFFB
:10E2C000C6E7334604AA39464046FFF7F9FBBFE7E5
:10E2D0000E25BDE70E25BBE7F8B508B30E4605468B
:10E2E000164B1F68F7B93C46B4420FD205EBC40386
:10E2F0005B68D3B115F8340015F93430002B16DB08
:10E30000B8B1FEF7F1FDB0B90134EDE70C4B43F8BD
:10E31000375003EBC7035E607B1C084A136002E0C2
:10E320000E2700E004273846F8BD0E27FBE70B2731
:10E33000F9E70F27F7E70F27F5E700BF8421002053
:10E3400088210020084B196861B110B504E0064827
:10E3500003F009FD214624B10C680B79002BF9D09C
:10E36000F5E710BD704700BF7023002038B50546A3
:10E3700030B1104B1C68C4B10F4B01221A7004E07D
:10E380007846FEF7EBFBF4E724683CB12379002BD9
:10E39000FAD154F8043C28469847F5E7064B1B7819
:10E3A000022B03D0044B00221A7038BDFFF7CAFFBE
:10E3B000F8E700BF702300206C23002010B504464E
:10E3C00030B100232372211D034803F0A1FC10BDCE
:10E3D0007846FEF7C3FBF4E77023002010B504462F
:10E3E00058B10A4B1B78013BDBB2012B09D8074B14
:10E3F00002221A700123237210BD7846FEF7AEFB8D
:10E40000EFE7211D024803F0AEFCF5E76C23002086
:10E41000702300200A8883689B5A07339BB223F03D
:10E42000030313449BB20288043A934200D90023A9
:10E430000B80704710B582B004468368C91AADF8E6
:10E4400006100DF10601FFF7E5FFBDF80630A068E4
:10E45000184402B010BD0088043880B27047438869
:10E460008268D018D15201238370704782680023DC
:10E470009370438083807047073189B221F0030194
:10E4800089B2428883889A4204D29B1A99421EDC40
:10E490000020704710B59A420FD90488A41AA142EF
:10E4A00017D98B4217D3032C03D983681344042252
:10E4B0009A7000234380184604E0826813449B78D6
:10E4C0000BB1042010BDFFF7D1FF0020FAE70420B4
:10E4D00070470020F6E70420F4E738B504460D46FF
:10E4E0008368828813448B4202D07846FEF736FB5D
:10E4F0000023AB70211D2046FFF78CFFA288A36884
:10E5000013449B78042B00D038BD0023A380FBE785
:10E5100010B50C468368428813448B4202D078467B
:10E52000FEF71CFB0023A37010BD10B5044630B1EC
:10E530002388042B07D92046FFF78DFF10BD7846AE
:10E54000FEF70CFBF4E77846FEF708FBF3E770B53F
:10E55000054614460E46002944D0002D46D0B6F19B
:10E56000005F08D94FF08053D3F80C3103F5002336
:10E57000B6EB832F0ED3B6F5000F08D94FF08053BA
:10E58000D3F80C3103F50053B6EB832F02D3784652
:10E59000FEF7E4FA631E3344B3F1005F08D94FF08D
:10E5A0008052D2F80C2102F50022B3EB822F0ED359
:10E5B000B3F5000F08D94FF08052D2F80C2102F5C4
:10E5C0000052B3EB822F02D37846FEF7C7FA042C31
:10E5D00010D92C8000236B80AB80AE60043C34806B
:10E5E000B37070BD7846FEF7B9FAB6E77846FEF725
:10E5F000B5FAB4E77846FEF7B1FAEAE738B504466B
:10E60000A0B16288A36813449B78012B12D0EFF36A
:10E61000108572B6A388A16819448B78032B0DD09E
:10E620002046FFF723FF05B962B638BD7846FEF7EE
:10E6300095FAE6E77846FEF791FAE8E72046FFF715
:10E64000F9FEA368C31A638000238370EBE72DE90A
:10E65000F0410E4614460546D0B1EEB16A88AB686B
:10E6600013449B78012B1BD024B32846FFF7F3FEFD
:10E67000A04221D3EFF3108872B621462846FFF757
:10E68000FBFE074680B1B8F1000F16D162B614E068
:10E690007846FEF763FAE0E77846FEF75FFADDE7D3
:10E6A0007846FEF75BFADFE721462846FFF7D7FEFC
:10E6B0003060E8E7092700E009273846BDE8F08127
:10E6C000F8B50C4615460646E0B1FCB1A378012B1F
:10E6D00020D12388AB4221D325B3EFF3108772B644
:10E6E00025800223A370F1183046FFF793FE73884C
:10E6F000B288934203D0B268134400229A7007B9DB
:10E7000062B6F8BD7846FEF729FADEE77846FEF7EE
:10E7100025FADBE77846FEF721FADAE77846FEF7D6
:10E720001DFAD9E77846FEF719FAD6E770B50C4618
:10E73000054690B1ACB1EFF3108672B6AA88AB680B
:10E7400013449A78042A10D09A78022A15D0032A02
:10E7500018D0052006B962B670BD7846FEF7FEF9FE
:10E76000E8E77846FEF7FAF9E5E7291D2846FFF7BE
:10E7700051FEAA88AB681344E6E703229A7023602F
:10E780000020E7E77846FEF7E9F90020E2E738B530
:10E79000044680B1EFF3108572B6A088A1680144E9
:10E7A0008B78042B0BD08878022814BF002001201E
:10E7B00005B962B638BD7846FEF7D0F9EAE72046DB
:10E7C000FFF738FE0146EEE738B5054678B1EFF3BE
:10E7D000108472B6A888A96801448878C31EDBB289
:10E7E000012B08D82846FFF725FE0146F5E77846B5
:10E7F000FEF7B4F9EBE7022814BF0020012004B9AA
:10E8000062B638BD70B50C46064678B194B1EFF3E8
:10E81000108572B6A378012B10D0032B13D121469B
:10E820003046FFF75AFE05B962B670BD7846FEF76E
:10E8300095F9EBE77846FEF791F9E8E7214630468F
:10E84000FFF766FEEFE77846FEF788F9EBE710B5CD
:10E85000EFF3108472B68388816819448B78042B97
:10E8600006D08878B0FA80F0400904B962B610BDCD
:10E87000FFF7E0FD0146F4E7024B1878003818BFB7
:10E880000120704774230020014B1868704700BFB7
:10E890009023002010B5044680B163681BB1236843
:10E8A0000BB1A36813B97846FEF758F9A3685A1E4E
:10E8B000134207D10023E360236110BD7846FEF7C1
:10E8C0004DF9EAE77846FEF749F9F3E7B0B5F0B15C
:10E8D0000446F1B18368F3B1EFF3108572B60369B2
:10E8E0008768DA19C3689A420DD000686268013FF0
:10E8F0003B4003FB020017F0BCFCE3680133E3601C
:10E900005DB962B60AE005B962B6042506E00E25D7
:10E9100004E00E2502E0092500E000252846B0BDF0
:10E92000F8B500B30F4604468368F3B1EFF31085E2
:10E9300072B60369C268934211D001684268866862
:10E94000013E334003FB021117B1384617F091FC2A
:10E9500023690133236155B962B62846F8BD05B96C
:10E9600062B60525F9E70E25F7E70925F5E7002545
:10E97000F3E700000246C0F30B0040BB49B310B4FC
:10E9800001F6FF710C0B144B0221C3F80415124B56
:10E99000D3F80034002BFAD001460AE00E4BC3F83E
:10E9A00008250D4BD3F80034002BFAD002F5805225
:10E9B0000131A142F2D3084B0022C3F80425064BD3
:10E9C000D3F80034002BFAD05DF8044B70471020C8
:10E9D00070470920704700BF00E0014010F0030FAE
:10E9E0002FD110B4044611F0030F2CD16AB312F0EA
:10E9F000030F2CD19008174B0122C3F80425154BA7
:10EA0000D3F80034002BFAD002E00434043110466D
:10EA1000421E50B10B68B3F1FF3FF6D023600D4B9F
:10EA2000D3F80034002BFAD0EFE70A4B0022C3F8EA
:10EA30000425084BD3F80034002BFAD05DF8044BC2
:10EA40007047102070471020F8E70920F6E70920EA
:10EA5000F4E700BF00E00140094B1B7813F0040FFE
:10EA600002D00378122B00D07047064B1A68064B71
:10EA70005A60034B1A786FF382021A70F4E700BFF2
:10EA80003824002028240020C423002010B582B0A0
:10EA900001900C46000C012810D12368094A13602C
:10EAA00009490B7843F001030B705B0883F0010305
:10EAB00003F001031371002002B010BD7846FEF789
:10EAC0004DF8EAE7282400203824002010B582B051
:10EAD00001900C46000C02280FD12268094B1A60E5
:10EAE00022791A71002058719871D871064A1378EA
:10EAF00043F00203137002B010BD7846FEF72EF803
:10EB0000EBE700BF202400203824002010B582B09D
:10EB100001900C46000C032806D1054B18682060B4
:10EB20001B79237102B010BD7846FEF717F8F4E7A1
:10EB30002824002010B582B001900C46000C032858
:10EB40000CD1084B2068186022791A71064A137894
:10EB500043F001031370002002B010BD7846FDF7AA
:10EB6000FDFFEEE7282400203824002010B582B0F5
:10EB700001900C46000C042805D1054B03CB206006
:10EB8000616002B010BD7846FDF7E8FFF5E700BF11
:10EB90002024002010B582B001900C46000C0428FF
:10EBA0000BD1084B2068616803C3074A137843F010
:10EBB00002031370002002B010BD7846FDF7CEFFAF
:10EBC000EFE700BF202400203824002000B583B0E8
:10EBD0000190000C032806D1054B00221A601A711F
:10EBE00003B05DF804FB7846FDF7B8FFF4E700BF1B
:10EBF0002824002000B583B00190000C042806D121
:10EC0000054B00221A605A6003B05DF804FB784699
:10EC1000FDF7A4FFF4E700BF2024002000B585B075
:10EC2000184B1B7813F0400F0FD0164B1B7813F0C6
:10EC3000040F07D1144B5B6803F500530193B3F144
:10EC4000807F06D905B05DF804FB7846FDF786FFA6
:10EC5000EBE70E4B1B788DF808300A4A137843F027
:10EC6000040313700023ADF80C300323ADF80E300D
:10EC700001A9039804F0E6FF0028E3D07846FDF7E9
:10EC80006DFFDFE738240020C42300203924002052
:10EC900000B585B00022ADF809200F4B99680191AD
:10ECA0001B7B8DF808300D490B780133DBB20B70FC
:10ECB0008DF80B30ADF80C200423ADF80E300DEBC1
:10ECC0000301039804F0BEFF10B905B05DF804FB22
:10ECD0007846FDF743FFF8E7C423002039240020DD
:10ECE00000B585B00F4B9A6801921A7B8DF8082009
:10ECF0001B8AADF809300C4B1B788DF80B300023C4
:10ED0000ADF80C300423ADF80E300DEB0301039881
:10ED100004F098FF10B905B05DF804FB7846FDF7E4
:10ED20001DFFF8E7C42300203924002000B58DB072
:10ED30000B4B1B7B012B0ED0094A926804928DF875
:10ED40000830039002238DF8043001A8FFF70EFB72
:10ED50000DB05DF804FB024A9268013A0492EEE7B6
:10ED6000C423002008B51D481D4B036000F064FE5D
:10ED70001C4B1B7813F0200F2AD103F00303032B45
:10ED800014D1194B1968194A916019791173B3F8A4
:10ED900005001082DB79164A1370164A12799342E5
:10EDA00017D0B1B9114B00221A6007E00F4B0022B7
:10EDB0001A609A601A731A82FFF76AFF0B4B1A687F
:10EDC0005A60084A137843F040031370FFF726FF98
:10EDD00008BD084B1A68054B1A60EFE714240020A1
:10EDE00059EA01003824002020240020C4230020F8
:10EDF000392400202824002010B582B00024ADF86A
:10EE000000400123ADF80230009804F04DFFADF84A
:10EE100004400223ADF80630019804F045FF02B02B
:10EE200010BD000008B5002004F068FF084B002268
:10EE30001A605A609A60DA601A61064A137803F021
:10EE4000DF0343F040031370FFF7E8FE08BD00BF87
:10EE5000C42300203824002038B50C4D00242C6039
:10EE60006C60AC60EC602C6101F0CCF8084B586031
:10EE7000084A9A60084ADA601C615C61074B1A789C
:10EE800064F3C3021A706C6038BD00BFC423002055
:10EE9000A0230020F9EF010000879303382400200D
:10EEA00008B50C4B1B7813F0100F00D008BD0A48B2
:10EEB0000A4B036000F0C0FDFFF754FFFFF79CFF13
:10EEC000074801F023F8034A137843F01003137046
:10EED000ECE700BF38240020B823002051F10100E6
:10EEE000A0230020034B1878800880F0010000F078
:10EEF000010070473824002010B501F029FE174B9F
:10EF00001B7B1BBB154B9B7B2BBB144B1A8A41F203
:10EF100082639A4206D8124B1B7813F0080F05D073
:10EF2000012300E001231BB9082410E00023FAE7C5
:10EF30000A4B01221A7300241C829A6801329A60DB
:10EF4000FFF7A6FE2046FFF7F1FE00E0082401F0DF
:10EF500043FE204610BD0824F9E700BFC42300206B
:10EF60003824002010B501F0F3FD214B5B7BABB1E1
:10EF70001F4B9B7B03BB1E4B1A8A41F282639A4252
:10EF800006D81C4B1B7813F0080F05D0012300E0B6
:10EF900001239BB1012302E00023FAE700231C4672
:10EFA0000BB3134B00225A731B7B4BB1012B0ED0BA
:10EFB0007846FDF7D3FD16E00023F0E70023EEE7E7
:10EFC000FFF79AFF78B17846FDF7C8FD0BE0084BD4
:10EFD00000201860586018731882FFF7A7FEFFF72B
:10EFE00057FEFFF71BFE01F0F7FD204610BD00BFE6
:10EFF000C42300203824002008B52C4B1B7BDBB138
:10F00000012B2ED07846FDF7A9FD284A138A01333B
:10F010009BB21382264AA2FB03121209C2EB021210
:10F02000A3EB42039BB2002B3DD0204B5B8A13B174
:10F03000013B1E4A538208BD1C4B1A8A41F282636F
:10F040009A4206D81B4B1B7813F0080F07D00123F8
:10F0500000E00123002BD8D0FFF784FFE5E7002371
:10F06000F8E7124B1B8A41F28262934206D8114A9A
:10F07000127812F0080F14D0012200E00122002AB9
:10F08000C3D042F2B012934202D9084B01225A7304
:10F09000FFF768FF0028C8D1044B5B7B012BB4D17C
:10F0A000C3E70022EBE7FFF71BFEBEE7C423002007
:10F0B000898888883824002010B5244B1B7B002BBE
:10F0C00035D10446214B5B8A2BBB1AB91F4B9B6879
:10F0D0008B4205D3FAB11D4B9B6801338B421AD288
:10F0E0001A4B9B682A338B4223D3184B9B7B03BB61
:10F0F000164B996000221A605A601A8242F6065135
:10F1000059825A731A73FFF7C3FDFFF787FD204634
:10F11000FFF70CFE0DE062B10C4B9B6801338B4294
:10F1200007D10A4B01225A73FFF71CFF01E0012BA4
:10F1300000D010BD002AFCD1044B9B688B42F8D153
:10F14000024B01225A73FFF70DFFF2E7C4230020A0
:10F150000378042B00D0704743681B78002BFAD04B
:10F1600010B58468027E437E012A14BF002201226A
:10F17000416904F11000FFF79FFF10BD08B538B1D9
:10F180000D4B01229A730D4A13680133136008BDB9
:10F190000A4B1B685BB1094A1368013B1360002BE3
:10F1A000F5D1054B00229A73FFF7DCFEEFE77846B6
:10F1B000FDF7D4FCEFE700BFC42300209423002018
:10F1C00000B58DB0ADF808008DF810200391032331
:10F1D0008DF8043001A8FFF7C9F80DB05DF804FB05
:10F1E000014B9868704700BFC4230020054B1B7B70
:10F1F000012B02D0034B98687047024B9868013886
:10F20000704700BFC42300201D4B1B7813F0400F34
:10F2100034D070B504460D461A4B1A685B689A42A2
:10F2200028D2184B1B7B012B17D0174B9A4216D2B2
:10F23000144B1A685B68403B9A4218D2EFF3108671
:10F2400072B6104A1368591C11602B60FFF7CEFF8D
:10F25000206006B962B6002070BD0C4BE6E7094B92
:10F2600001225A73FFF77EFE0028E7D1E0E7FFF79F
:10F27000D5FCE3E7FFF7D2FC0F20EDE70F20704746
:10F2800038240020C4230020FFFF7F0000E0FF009F
:10F29000044B9B68584010F0010F00D0013B18460A
:10F2A000704700BFC4230020014B187B704700BF8C
:10F2B000C4230020F8B5104B1B7813F0200F01D0A9
:10F2C0000820F8BD17460C4E43F0200333700B4D59
:10F2D000A860297300242C82FFF7DAFC2046FFF790
:10F2E00025FD2F606F60337843F040033370FFF7E4
:10F2F00095FC2046E5E700BF38240020C423002009
:10F300002DE9F041002624E02449BC2303FB04F34B
:10F31000CA5A0132CA520221284602F0F9FB0137CB
:10F320000221284602F0C4FB014679B11B4ABC23E6
:10F3300003FB0423D3F80880B8F1000FE4D0BC230A
:10F3400003FB04F3D25A3046C047DDE797B90136D4
:10F35000F6B2022E1FD83446BC2303FB06F3083353
:10F360000E4D1D4404350221284602F0A1FB014642
:10F370000027DAE7284602F033FC0828E7D1074BDC
:10F38000BC2202FB0434A368002BE0D00022044915
:10F3900030469847DBE70120BDE8F0814424002097
:10F3A000B46D030008B5082383731023437300F181
:10F3B0001C0343610323037300F1180303610C3042
:10F3C00002F0E0FB08BD000008B50378012B06D071
:10F3D000022B06D07846FDF7C1FB002002E02B206F
:10F3E00000E0014808BD00BFCC55010008B5037816
:10F3F000012B07D0022B12D07846FDF7AFFB4FF45C
:10F40000FA7307E08368591A89082B2303FB01F379
:10F4100003F5FA730648984228BF184608BD83686A
:10F42000591A090B034B03FB01F303F5FA73F1E7D8
:10F4300060850100CC55010038B5044601210C302F
:10F4400002F036FB054678B1084BC4F89C30002327
:10F45000C4F8A0306168FFF7C9FFC4F8A800C4F879
:10F46000AC40012384F8B830284638BD8DF5010042
:10F4700010B50446FFF7E0FF20B104F19C000DF049
:10F4800081FB00B910BD7846FDF768FBFAE7000084
:10F49000F8B505460C46164617680378012B19D1B6
:10F4A0001249A1FB0431C9088B00AC68E41BB4EB22
:10F4B000810F00D31C468CB1686827F00307E96808
:10F4C000224639443844FFF789FA58B933681C4456
:10F4D0003460F8BD7846FDF741FBE1E77846FDF77B
:10F4E0003DFBE9E77846FDF739FBEFE783BEA02F48
:10F4F000F8B506460C46154617680378022B17D157
:10F50000114BA3FB04231B0C1A03B468E41BB4EBDC
:10F51000033F00D314467CB1706827F003072146EF
:10F520003844FFF727FA58B92B681C442C60F8BD03
:10F530007846FDF713FBE3E77846FDF70FFBEBE7B3
:10F540007846FDF70BFBEFE72D57BDBF38B50546F5
:10F550000C4611462378012B06D0022B0FD078469B
:10F56000FDF7FCFA002304E0021D2046FFF790FFA0
:10F57000A3686868984214BF0020012038BD021DAE
:10F580002046FFF7B5FFA368F3E700002DE9F84335
:10F590000F46D1F8A850254B1B786BB90446A5F54A
:10F5A000FA7501F10C080121404602F081FA064685
:10F5B00048B14FF0000924E00DF020FB002387F84C
:10F5C000B830BDE8F8837846FDF7C8FAF1E70DF0EA
:10F5D00015FB0121404602F09BFA00237B6087F86F
:10F5E000B830134B186801F04BFB3846FFF740FF6B
:10F5F000E7E7A4EB00093046FFF7E6FE4844A842DF
:10F600000DD8A5EB090231463846FFF79FFF0028C9
:10F61000DDD101F04BF9B0EB0409ECD5E9E70DF0D1
:10F62000EDFA3846FFF724FFCBE700BF4024002067
:10F630003C24002010B5084801F002FB074B18607D
:10F64000002406E0064BBC2000FB0430FFF7AAFEB6
:10F650000134022CF6D910BD01F301003C24002036
:10F660004424002038B50446EFF3108572B610B973
:10F67000164B1B6873B18CB1144A136801331360C5
:10F68000124B1B68003B18BF0123114A137005B9C8
:10F6900062B638BD7846FDF761FAECE70B4B1C68A3
:10F6A000013C1C6034B1EBE7BC2000FB0420FFF7F9
:10F6B000DFFE0134022CE3D8064ABC2303FB0423FB
:10F6C00093F8B830002BF4D1EEE700BF7826002085
:10F6D000402400204424002018B1830B024AD05C4F
:10F6E00070470020704700BFC46D030012DF7047F1
:10F6F00000B583B001F0FCFE40B10C4B1B6813F069
:10F70000400F03D00A4B1B68012B02DC03B05DF8ED
:10F7100004FB084BD3F804350190074A0092752288
:10F720000649022002F0B4FBF0E700BF741F00207E
:10F73000701F0020001001403C6E0300316E03007A
:10F7400000B58DB0114B1B78022B06D07846FDF723
:10F7500005FA01200DB05DF804FBFFF7C3FB18B9F3
:10F760000B48FEF72BFEF4E70DF080FF074B03225A
:10F770001A702C22002101A816F0A4FD1D238DF87B
:10F78000043001A8FEF7F2FDE3E700BF8026002069
:10F79000641F00200B4B1B78042B00D0704700B572
:10F7A0008DB0084B05221A702C22002101A816F0FA
:10F7B00089FD1C238DF8043001A8FEF7D7FD0DB09C
:10F7C0005DF804FB8026002008B50378122B00D0DA
:10F7D00008BD0448FEF702FE034B186801F050FA1A
:10F7E000F6E700BF641F00207C26002070B58AB0B9
:10F7F0000DF07EFF48B3064600238DF8103005ACAF
:10F8000005460FCD0FC42B682360727D052A04D9ED
:10F81000337D03F00F03072B1ED1174B1A688AB1F3
:10F8200004AB0393337DC3F303038DF80430737D7E
:10F83000062B1BD9063B8DF8053006F11D030293FC
:10F8400001A8904730460DF033FF0DF06DFF80F0BA
:10F850000100C0B20AB070BD307D04AB063A06F1BB
:10F860001D0100F00F000CF015FCD6E700238DF809
:10F8700005300293E4E700BF8426002070B582B013
:10F88000314B1B78002B54D10446002855D0067A02
:10F890000F2E01D0062E52D104F026FEE06870B182
:10F8A000FDF76EF90DF10700FFF720FF0546002870
:10F8B00040D19DF80730012B04D002253AE0FDF736
:10F8C0006DF9EFE7FDF790F900F008FB304601F025
:10F8D000D3F8E07800F02CF900F0B4FE0DF0D4F885
:10F8E0001A480DF0BDFF0CF07DFD0CF0B5FBFFF7E5
:10F8F000A1FE04F08DF900F001FD04F0B5FD04F067
:10F9000071FB204601F00EFDFEF7EAF903F0ECFC76
:10F91000FDF772F808B1062813D10D4801F090F9EF
:10F920000C4B18600C4B00221A60074B01221A7016
:10F9300000E00825284602B070BD0E25FAE707252D
:10F94000F8E70546F6E700BF80260020EDF7010046
:10F9500041F701007C2600208426002010B582B0EB
:10F96000204B1B78012B0DD05AB2002A35D0043B16
:10F97000DBB2012B33D80DF0F5F8044628B320464E
:10F9800002B010BD01F0DEFCFEF7ECF9FDF734F833
:10F990000446B8B1062815D0134B1B6813F4804FEA
:10F9A000EDD0124B1B68012BE9DD114BD3F8043568
:10F9B0000190104A00924FF4C2720F49022002F0E7
:10F9C00067FADCE701F084F8D5E7064B02221A70EB
:10F9D0000A4B186801F054F9D1E70824CFE708244E
:10F9E000CDE700BF80260020741F0020701F00207C
:10F9F00000100140686E0300316E03007C26002079
:10FA000008B5094B1B78032B01D0082008BD064B15
:10FA100004221A7005480DF059F80028F6D07846EF
:10FA2000FDF79CF80020F1E78026002095F7010003
:10FA300008B5FEF79BF908BD08B5FEF7BFFC08BD89
:10FA400008B5FEF7CBFC08BD08B500F0C1FD0020ED
:10FA500008BD7047064A136801331360B3F1704F55
:10FA600002D0034B18687047134601221A60F8E76A
:10FA70008826002010B5044618B100232360636077
:10FA800010BD7846FDF76AF8F7E738B50C4605462D
:10FA900068B184B100236360EFF3108372B62A6803
:10FAA0006AB16A6854606C6003B962B638BD784662
:10FAB000FDF754F8EDE77846FDF750F8EAE72C60DB
:10FAC000F1E710B5044658B1EFF3108372B6206821
:10FAD00008B142682260226832B103B962B610BD33
:10FAE0007846FDF73BF8EFE76260F6E710B50446AD
:10FAF00008B1206810BD7846FDF730F8F9E735DF2A
:10FB00007047000008B54FF0FF30FFF7F8FFBFF374
:10FB10004F8F0549CA6802F4E062044B1343CB607F
:10FB2000BFF34F8F00BFFDE700ED00E00400FA05D2
:10FB3000072814D8DFE800F0080C1504110F0A0696
:10FB40006420704714207047FA2070471E207047C9
:10FB50004FF4FA707047322070474B207047FA20FC
:10FB60007047962070470000024B5868103840B22A
:10FB7000704700BF00ED00E0034600280FDB5B117B
:10FB8000084A52F82330424200F01F0002F01F02E0
:10FB900058BF504223FA00F000F00100704700F116
:10FBA0001F03ECE700E100E046DF7047F8B50446CC
:10FBB0000D464B1EDBB2012B09D800232361636184
:10FBC000A361E3612046FFF7EFFF012016E07846CE
:10FBD000FCF7C4FFF1E7CA5CCE185200D2B27678C7
:10FBE00042EAD612CA5401339BB20E2BF3D9CB7B17
:10FBF0005B00CB73002F08DB0130C0B2A8420BD8EA
:10FC0000214611F9207F0023EFE794F82F3083F08D
:10FC1000870384F82F30EFE7F8BD2DE9F04190B06D
:10FC200084460C4696461F4602F10F084FEA2816F6
:10FC300004AD0068DCF80410DCF80820DCF80C30B7
:10FC40000FC50EF00F055FEA181302D07DB1002337
:10FC500000E00023984663B1012104A8FFF7A6FF46
:10FC6000B8F1000F1AD0701E000110230EE001231E
:10FC7000F0E70221F1E7013B9BB22218D25C10A908
:10FC8000194411F8101C4A400DF80320002BF2D142
:10FC900000250C950D950E950F9533E0711EADB2B4
:10FCA0002A4604EB0111684616F0E3FA80230DF8AA
:10FCB00005306B1C03E000220DF8032001330F2BED
:10FCC000F9DD10230AE0013B9BB21DF8032010A9C7
:10FCD000194411F8101C4A400DF80320002BF2D1F2
:10FCE000D6E7013A92B210AB134413F8100C631824
:10FCF0009B5C584008AB9854002AF2D104A8FFF747
:10FD000053FF0135731EAB4202DD29011022F3E7D8
:10FD100010230AE0013B9BB210AAD11811F8402C25
:10FD200011F8101C4A4008A9CA54002BF2D104A8AB
:10FD3000FFF73AFF0CAC0FCC38607960BA60FB601B
:10FD400010B0BDE8F081000010B50446134B1B68ED
:10FD500093B14168114B1B685B68CB1A002B0BDB1E
:10FD60000E4B1B6818465B691BB15A68521A002A71
:10FD7000F8DB6361446103E0084B1A6862611C6050
:10FD8000064A93889BB201339BB2938013B101233F
:10FD9000237010BD7846FCF7E1FEF8E794260020BA
:10FDA00038B505461CE07846FCF7D8FE6369204A62
:10FDB00013600023636193889BB2591E89B29180BE
:10FDC000F3B1A36803B302232370A3682169284613
:10FDD000984700F017F905462378DBB2022B17D0BD
:10FDE000134B1B681BB3124B1B685B685B1B642BBC
:10FDF0001DD50F4B1C682378DBB2012BD6D0D2E780
:10FE00007846FCF7ABFEDCE77846FCF7A7FEDAE7BE
:10FE1000E26812B900232370E2E763681344636069
:10FE20005B1B642BF9D42046FFF78EFFD8E738BD63
:10FE30009426002010B50446144B1B68834207D05B
:10FE4000124B1B68D3B15A69A2420ED01346F9E790
:10FE500043690E4A136093889BB2591E89B2918000
:10FE600063B97846FCF77AFE08E062695A6107498F
:10FE70008B889BB25A1E92B28A8013B100232370E2
:10FE800010BD7846FCF76AFEF8E700BF9426002014
:10FE900008B5064B1B6833B1044B1B68044958680E
:10FEA00000F05CF908BD00F0B7F9FBE794260020EC
:10FEB000CDFE010008B500F0A5F8FFF771FF00F0D6
:10FEC000A1F8FFF7E5FF012008BD000008B5024BCF
:10FED000186800F0D5FE08BD8C26002008B5002368
:10FEE000064A1370064A13605360064800F0A8FEE5
:10FEF000054B186000F078F808BD00BF9026002080
:10FF000094260020B5FE01008C26002010B5044682
:10FF1000154B1B789BB900F087FFA0B1BCB1A3685B
:10FF2000CBB12378DBB2012B19D0002363612046CB
:10FF3000FFF70AFF00F066F8FFF7AAFF10BD78464A
:10FF4000FCF70CFEE7E77846FCF708FEE6E77846A4
:10FF5000FCF704FEE3E77846FCF700FEE1E77846AD
:10FF6000FCF7FCFDE1E700BF9026002010B5044639
:10FF700000F05AFF50B16CB12046FFF75BFF002341
:10FF8000636100F03FF8FFF783FF10BD7846FCF790
:10FF9000E5FDF0E77846FCF7E1FDEDE738B504460E
:10FFA0000D46104B1B788BB900F03EFF90B1ACB101
:10FFB0002046FFF73FFF0023636165602046FFF79F
:10FFC000C3FE00F01FF8FFF763FF38BD7846FCF76B
:10FFD000C5FDE9E77846FCF7C1FDE8E77846FCF7A0
:10FFE000BDFDE5E79026002008B515F0DFFF00B164
:10FFF00008BD15F053FF0028FAD07846FCF7AEFD97
:020000022000DC
:10000000F6E7000070B4EFF3108172B6184B1A686F
:10001000184BD3F80455D3F80431012B22D001B981
:1000200062B645EA026500266B01EA0E5B1B62EBD5
:100030000602510241EAD3515802431941EB06002E
:10004000810141EA93619A01D31A61EB00005B19C7
:1000500046EB000013F580437041DB0B43EA404060
:1000600070BC7047034BD3F804550132D7E700BF8B
:100070009C2600200010014010B50A4B4FF40032BE
:10008000C3F84823C3F80823074B1B682BB1064B62
:100090001C68FFF7B7FFA04710BD7846FCF75EFD70
:1000A000F5E700BF00100140A8260020EFF3108103
:1000B00072B6254B0022C3F80421244A1368013389
:1000C000136001B962B6224B1B68002B3AD0204B5B
:1000D0001A68013A1A601B68002B33D103F1804380
:1000E00003F58833D3F804251A4B1B689A421BD2B8
:1000F000EFF3108272B6144BD3F80435981C1549EF
:10010000096888420DD303330F49C1F8443502B959
:1001100062B60D4B4FF40032C3F84423C3F80423F6
:1001200070470C4B1B68EFE710B50B4B1B682BB1EE
:10013000094B1C68FFF766FFA04710BD7846FCF727
:100140000DFDF5E7704700BF001001409C26002020
:10015000A0260020A4260020A826002030B583B0C9
:100160000446002301930D46002936D0244B1D6020
:10017000FFF748FF031B002B33DB0023590CD80388
:10018000204C214A002300194FF0000444EB0101E8
:1001900015F036FFEFF31083019372B61B4BD3F8C3
:1001A0000435032838BF0320C3F1FF1202F57F4254
:1001B000824218D30344154AC2F844354FF4003341
:1001C000C2F84433C2F80433114A1460114A14606F
:1001D000019B03B962B603B030BD7846FCF7BEFCA4
:1001E000C4E7231ACAE7034403F17F4301331A0E1D
:1001F000013207490A6023F07F43064A1360E7E7AC
:10020000A826002020A1070040420F000010014056
:10021000A0260020A4260020074B4FF40032C3F88C
:100220004823C3F808230023044A1360044A1360D8
:10023000044A1360704700BF00100140A026002050
:10024000A4260020A826002030DF704731DF704749
:1002500010B4034602684068A2EB70129C6880EA02
:10026000F4301860D9680C445C6011449960104403
:10027000D8605DF8044B704770B582B00D460646F5
:1002800008B100240BE07846FCF768FCF9E79DF81C
:1002900007103019FFF7DAFF9DF807301C44A5421C
:1002A0000DD90DF10700FFF7CFFF9DF80730002BA8
:1002B000F7D02A1B9342EAD98DF80720E7E702B06E
:1002C00070BD000030B583B00546002401940421C0
:1002D0000DEB0100FFF7D0FF074B2B60019B6B601C
:1002E000AB60EB6003E02846FFF7B2FF0134132C4C
:1002F000F9D903B030BD00BFED5EEAF1704708B533
:10030000032003F0FBFC08BD48DF704749DF70475E
:100310004ADF7047044B01225A7143F2B0629A607F
:1003200043F69822DA60704708270020094B032221
:100330001A74094A5A611A6840F6D8639A4204D975
:10034000054B43F2B0629A607047034B40F6D862A7
:100350009A607047E82600200827002008B50F4B58
:100360001B78022B12D0032B08D0012B03D0784628
:10037000FCF7F4FB0EE0022303740BE0084B0022B1
:100380005A71084999600849D9608271032303743E
:10039000034B4361014B00221A7008BD192700204E
:1003A00008270020A0860100FF1FA10738B50446DA
:1003B00000250574012343710E4A1368013313604D
:1003C00000F0D2FA0CF094FC23680B4A1168283133
:1003D00001FB03F1094AA2FB0121A3EB9141084A69
:1003E0007839284600F03CFA00B938BD7846FCF769
:1003F000B5FBFAE71C2700200427002083DE1B43FF
:100400002D03020010B5044600238360C360036817
:100410000D4A92680260817991B10121017403B99A
:100420000A4B991A6161B1F57A7F01D39A4202D9D8
:100430004FF47A736361FFF76DFF0123A37110BD61
:10044000FFF7B4FFF7E700BF082700208096980069
:1004500010B50C4631B1C3680133C360426903680B
:10046000134403608368013383600122027442698C
:1004700052084261012B0DD0022B19D0426903684A
:10048000134417498B4222D840F6D7639A4221D8A9
:1004900000231DE0B2F5FA7F05D040F6D8639A42FA
:1004A000ECD84361EAE7002CF7D100234361E5E78C
:1004B000C368022B06D0012BE0D1002CDED1002333
:1004C0004361DBE70268064B9B1A4361D6E70023D2
:1004D00013B110BD0123FBE7FFF768FFF9E700BF89
:1004E0008096980043791BB90D4B00221A70704713
:1004F00010B504460CF018FC23680A4A106828302E
:1005000003FB00F0084AA2FB0020A3EB90407838E0
:1005100000F05AFA00236371014B00221A7010BDDB
:10052000182700200427002083DE1B4308B5254B35
:1005300001221A71244B1B7813B1244B1B781BB377
:10054000204B00221A7404281AD8DFE800F00314A4
:10055000110C07001B48FFF755FF1CE0012119484B
:10056000FFF776FF17E000211648FFF771FF12E052
:100570000CF06AFB0FE000F0B9F90CF09FFB0AE009
:100580007846FCF7EBFA06E000F090F90D4B1860A6
:100590001846FFF7E3FE0B4B1B7C023BDBB2012B43
:1005A00008D9084B1B7C022B08D006480023037196
:1005B000103008BD0348FFF795FFF2E7014B012219
:1005C0001A76F2E7E82600201927002018270020D5
:1005D00008B50438042814D8DFE800F018261403FE
:1005E0000E00164B1B7E012B0BD1FFF78FFE40B187
:1005F0007846FCF7B3FA04E0104B00221A760CF0B0
:10060000BBFB08BD7846FCF7A9FAFAE7FFF782FEC4
:100610000B4840F6D8638360FFF77AFE0028F0D0DD
:100620007846FCF79BFAECE70548FFF771FE0028D7
:10063000E7D07846FCF792FAE3E700BFE82600200F
:100640000827002010B40E4A0023137013710121F3
:10065000517143F2B064946043F69824D460094A1F
:100660001060094A1370094A1370094A1360094A55
:10067000137153711360137691715DF8044B7047D9
:100680000827002004270020182700201927002011
:100690001C270020E826002008B5104B1B7E012BEC
:1006A00008D0022B17D00BB1002008BD0C48FFF773
:1006B0002BFE40B90B48FFF72BFE40B9074B022237
:1006C0001A760020F1E77846FCF748FAF2E7784618
:1006D000FCF744FAF2E71120E7E700BFE826002024
:1006E0002D050200082700200B4B1B7C023BDBB2D0
:1006F000012B0BD9094B1B78012B09D0022B09D0F8
:10070000032B01D000207047012070470120704763
:100710000120704701207047E8260020192700209B
:10072000014B1868704700BFE82600200D4B5B792D
:100730000BB90020704710B50A4B1C680A4B1B68A8
:10074000283303FB04F3094AA2FB0323A4EB9344DD
:10075000783C00F0ABF80346201A00D410BD181BFB
:10076000FCE700BFE82600200427002083DE1B43AF
:10077000014B5879704700BFE8260020014B1879DB
:10078000704700BFE8260020024B187E003818BFD3
:1007900001207047E8260020EFF3108372B6054A67
:1007A000527922B1044A4FF48071C2F8001103B9A2
:1007B00062B67047E826002000E100E008B5054B6E
:1007C0001B7E022B00D008BD034B01221A70FFF7DD
:1007D000E3FFF8E7E82600201927002008B5074BBB
:1007E0001B7E022B00D008BD012804D0044A1370E0
:1007F000FFF7D2FFF7E70323F8E700BFE826002062
:100800001927002008B5094B1B782BB148B9084BB4
:100810001B7813B1012300E00023044A107013B9C0
:1008200008BD0023F9E7FFF7B7FFF9E71827002015
:100830001927002010B4094B00F15002002443F89E
:10084000224000F110040122A240C3F8042300F565
:10085000A87043F820105DF8044B704700800040FA
:10086000022817D810B5EFF310840C4B1C6072B639
:100870000B4B43F820200B4B002243F820200A4B5F
:100880001B7823B9054B186830B962B605E0FFF74D
:10089000D1FFF7E707207047002010BD3027002068
:1008A000202700203C2700202C270020EFF3108277
:1008B0000A4B1A6072B60A4B1B7863B1094B0022CF
:1008C000C3F84C210122DA64D3F84C05034B1B68B2
:1008D00003B962B67047044B1868F7E73027002069
:1008E0002C27002000800040342700202DE9F04113
:1008F000002411E00027174B43F82470012303FA6A
:1009000005F5154EC6F80853FFF7D0FFC04704F1B0
:10091000500346F823700134022C18D804F1500318
:100920000D4A52F82330002BF5D0D2F8043304F1ED
:100930001005EB4013F0010FEDD0064B53F8248067
:10094000B8F1000FD6D17846FCF708F9D2E7BDE838
:10095000F08100BF2027002000800040014B1B6871
:10096000184470473827002010B500230CE0114AC6
:1009700003F5A871002042F8210003F1500142F86C
:10098000210052F821200133022BF0D90A4B1B68B9
:100990001BB90A4B4FF480721A60094B01221A707E
:1009A000FFF730FB0446FFF781FF241A054B1C605C
:1009B00010BD00BF008000403027002000E100E0B3
:1009C0002C27002038270020002307E000220C49B4
:1009D00041F823200B4941F823200133022BF5D99C
:1009E000094B1860094B00221A70094B4FF0FF3277
:1009F000C3F80823074B4FF48072C3F88021704777
:100A0000202700203C270020342700202C2700200E
:100A10000080004000E100E008B503783BB1012B05
:100A200004D1436813B1C1688068984708BD436822
:100A3000002BFBD080689847F8E70000044B1B7838
:100A40000F2B04D0034B4FF48022C3F800217047D2
:100A5000AC28002000E100E010B501460548FDF794
:100A600035FF10B10424204610BD0446FFF7E6FF11
:100A7000F9E700BF4827002010B5104C207010483F
:100A8000104B0360102343608360FDF703FF0E48A3
:100A9000FEF7F0FF23780F2B0FD0072B0AD8EC229C
:100AA0001A4112F0010F05D05B01DBB2074A82F850
:100AB000123302E07846FCF751F810BDAC28002054
:100AC000482700205C270020B028002000E100E03B
:100AD00008B5124B1B780F2B00D108BD104B93F8B3
:100AE00012335A09EC23134113F0010F0ED00D4BB2
:100AF0009B6833B10B4A136843F4802313600023CF
:100B000006E0074A4FF48021116001E042F202033F
:100B1000002BE2D07846FCF721F8DEE7AC28002075
:100B200000E100E06C54002030B585B00C4605466D
:100B300048B100238DF80030019502946846FFF714
:100B40008BFF05B030BD7846FCF708F8F1E70000F0
:100B500038B5EFF3108472B6194A1368591C116046
:100B600003BB184B1B780F2B1CD0EFF3108272B60F
:100B7000154B9B68E3B9144901238B60134BD3F8E1
:100B80008000134D28400860C3F88050D3F88400DB
:100B900048604FF0FF31C3F884100E4B00211970EC
:100BA00002B962B6064B1B6833B104B962B638BDF0
:100BB000084B01211970F3E77846FBF7CFFFF4E704
:100BC0005C280020AC2800206C54002000E100E0EC
:100BD000FC06FFBDAD28002010B5EFF3108472B6FF
:100BE000124B1B68F3B1114A1368013B1360B3B990
:100BF0000F4B1B780F2B12D00E4B1A780E4B9B68A5
:100C00006BB162B9EFF3108172B60B4B18680B4AE7
:100C100010605868506000229A6001B962B604B949
:100C200062B610BD7846FBF799FFDCE75C28002030
:100C3000AC280020AD2800206C54002000E100E02A
:100C400010B5044680B10C4B1B68102B10D8EFF385
:100C5000108272B6084B1868411C1960074B43F8A4
:100C6000204002B962B610BD7846FBF777FFEAE78D
:100C70007846FBF773FFEAE760280020642800202D
:100C800038B504460D4B1B68834213D9EFF310852A
:100C900072B661090A4A04F01F04012303FA04F43E
:100CA00052F82130234342F82130FFF7C7FE05B93F
:100CB00062B638BD7846FBF751FFE7E760280020B1
:100CC000A828002070B50D461646044658B175B1E7
:100CD000EFF3108372B6A560E660002222742460F0
:100CE00003B962B670BD7846FBF738FFEFE7784688
:100CF000FBF734FFECE7000038B5044650B1A368B9
:100D000063B1EFF3108572B6237C5BB1112005B996
:100D100062B638BD7846FBF721FFF0E77846FBF76F
:100D20001DFFEEE70123237421460348FEF7ADFEC5
:100D3000FFF784FE0020EAE7B028002010B5044643
:100D400008B1207C10BD7846FBF708FFF9E70000EA
:100D500070B584B02C4B1B7823B901252A4B1D702C
:100D600000240AE07846FBF7F9FEF6E7274B53F834
:100D7000243098470646F0B10134254B1B68A34246
:100D80001ED96109234A52F8213004F01F00C340E4
:100D900013F0010FF0D0EFF3108672B6012303FABF
:100DA00000F052F8213023EA000342F82130002EEF
:100DB000DCD162B6DAE72046FFF762FF3546DBE7B3
:100DC0001548FEF77EFE0AE07846FBF7C7FEA368EB
:100DD000E0689847002323740F48FEF772FE20B1A5
:100DE0000468237C002BF2D1EEE769460B48FDF73F
:100DF00097FD18B96846FFF70FFEF6E7024B002291
:100E00001A70284604B070BDB8280020642800205D
:100E100060280020A8280020B028002048270020B3
:100E200008B5FFF795FF08BD00B583B0FEF79CFE3F
:100E30008DF807009DF807305BB213F1100F18D042
:100E40009DF807305BB2002B21DB03F1604303F513
:100E5000614393F800335B090093154B1B78009AAC
:100E6000934220D0009A934217D3002003B05DF83C
:100E700004FB0F4B1B780F2B01D10120F6E712204A
:100E8000FEF77AFE08B10020F0E70120EEE703F05C
:100E90000F03084AD35C5B09DEE71220FEF76CFE05
:100EA00018B10020E2E70120E0E70120DEE700BF03
:100EB000AC28002014ED00E046DF704770B58CB020
:100EC00003460E4614466D46006859689A68DB680A
:100ED0000FC530687168B268F3680FC56846FFF7E0
:100EE000EBFF08AD0FCD20606160A260E3600CB045
:100EF00070BD08B5FEF791FE08BD08B501F06DF9AB
:100F000008BD08B501F0A2F908BD38B5022931D8ED
:100F10004CB2002C54D100297ED11970817A5A78B4
:100F200061F306025A70C17AD2B261F3C7125A70E5
:100F3000C168C1F3074201F47F44224300249A7040
:100F4000120ADA70197101890A0A42EA0122A3F829
:100F50000520DC711C7201690A0202F47F0242EA78
:100F60000162080A00F47F40024342EA1162C3F8BA
:100F7000092038BD03294FD1197000215970C46868
:100F8000C4F3074204F47F452A439A70120ADA70C8
:100F90001C710489220A42EA0422A3F80520D971AF
:100FA000197201690A0202F47F0242EA0162080A28
:100FB00000F47F40024342EA1162C3F80920D8E7F7
:100FC0001970597801F0800162F3C7115970C16836
:100FD000C1F3074201F47F4422439A70120ADA7087
:100FE000197101890A0A42EA0122A3F80520418801
:100FF0000A0A42EA0122A3F8072001690A0202F460
:101000007F0242EA0162080A00F47F40024342EA9A
:101010001162C3F80920ACE77846FBF79FFDA8E70B
:1010200070B584B00D461446064668B162B100231F
:10103000009301930293039323462A463146684660
:10104000FFF757FF04B070BD7846FBF787FDEEE76A
:101050002DE9F04184B00E4614461D460B9F804694
:1010600010B10AB103B117B97846FBF777FD6B46AB
:10107000324641462046FFF73CFF3B469DF828207C
:1010800029466846FFF735FF04B0BDE8F08100004F
:101090002DE9F0418EB00E4614461F46054608B1B4
:1010A00001B113B97846FBF759FD002C4DD0102C37
:1010B0004FD82A4B049305AA042104A8FFF7B0FFD8
:1010C0006B461022294605A8FFF713FF224631463A
:1010D00005A815F0CEF80EAB2344012203F8242C0A
:1010E000A21805AB92B219466846FFF702FF9DF8B9
:1010F000233003F07F033D4605F8013B224631468D
:1011000009A815F0B6F804F110080EAB98440223B4
:1011100008F8243C1134A4B22B46224605A968469F
:10112000FFF7E7FE05AE28686968AA68EB680FC696
:10113000032308F8243C07F11103224605A9684659
:10114000FFF7D7FE0EB0BDE8F0817846FBF706FD4D
:10115000ADE77846FBF702FDABE700BF736D6B327E
:1011600030B589B00C460546F8B1F1B1114B039387
:1011700004AA042103A8FFF753FF04AB1022294659
:101180001846FFF7B6FE0C4B93E8030001908DF86C
:10119000081004AB052201A91846FFF7AAFE06AB0A
:1011A00003CB2060616009B030BD7846FBF7D6FC08
:1011B000DCE700BF736D6B33906E030030B587B012
:1011C0000C460546E8B1E1B1104B019302AA042197
:1011D0000DEB0100FFF724FF02AB10222946184651
:1011E000FFF787FE0A4B009302AB042269461846BC
:1011F000FFF77FFE9DF8173003F03F03237007B021
:1012000030BD7846FBF7AAFCDEE700BF736D6B3498
:101210006964360110B5044678B123789BB1E26861
:10122000B2F1807F11D2E27A0AB1022B0FD094F989
:101230000A30002B05DB012006E07846FBF78EFC28
:10124000EBE7002000E0002010BD0020FCE70020BC
:10125000FAE730B587B00446037C8DF800300268A9
:101260008368D27A32B30822134409330193236886
:10127000029363680393E368049305A9684601F049
:10128000E3FC50EA01031AD0237C012B07D020682D
:1012900000F10C011030FDF7B7FF054660B9216879
:1012A000059800F006FA059B09336361002528467E
:1012B00007B030BD0422D7E701F06EFDF7E7042543
:1012C000F5E7000070B582B00446694600890AF06F
:1012D00041FE18B10025284602B070BD0646012027
:1012E00003F0F0F805460028F5D0A37A012B14D9B5
:1012F0002378012B09D00A4B1B68002BEBD0A27A74
:101300006188208998470546E5E7694660880AF0C4
:1013100021FE0028EFD03546DDE73546DBE700BF8C
:10132000BC28002008B538B14268054B1A60FDF7AB
:1013300093FD02F011FA08BD014B00221A60F6E796
:10134000BC28002008B5FDF7ABFD02F045FA08BD4A
:1013500010B5044668B123687BB123685B6983B12B
:10136000237C012B11D8E3689BB12046FFF771FF66
:1013700010BD7846FBF7F2FBEDE77846FBF7EEFB96
:10138000EBE77846FBF7EAFBEAE77846FBF7E6FB94
:10139000E9E77846FBF7E2FBE7E70000F0B5C7B006
:1013A000064630B3736943B3336853B333685B693C
:1013B0005BB3706900F0E3F90546254B1B6813F039
:1013C000020F3BD0234B1B68042B37DD00231C2B63
:1013D0001FD8EA5C2049086814095900075D05AC6C
:1013E00004F8137002F00F020131825C6254013381
:1013F000EDE77846FBF7B2FBD4E77846FBF7AEFBA8
:10140000D2E77846FBF7AAFBD0E77846FBF7A6FBC6
:10141000CFE705AA00238DF84E3003F1804303F592
:101420008833D3F8043502920C4A01920C4A009298
:101430004FF497720B49052000F02AFD00232A463D
:10144000B168306800F0EAFA01F06CFC47B0F0BD1A
:10145000741F0020701F0020781F00200C6F0300F5
:10146000A8690300016F0300F0B589B004460E4679
:101470001546837A013B8372029004924FF0FF334A
:101480000393DF23059301238DF8183002A8FFF79B
:10149000E0FE074698B1114B1B6813F0020F16D0FF
:1014A0000F4B1B68012B12DD0E4BD3F804350E4A8F
:1014B0000092AD220D49022000F0EAFC07E02A4626
:1014C0003146079814F0D5FE02A8FFF767FFA37A0C
:1014D0000133A372384609B0F0BD00BF741F00206D
:1014E000701F002000100140146F0300016F030003
:1014F000F0B5D5B0002800F0B6800E461746054678
:1015000000F041F9421B29464CA814F0B2FE574B9B
:101510001B6813F0020F31D0554B1B68042B2DDDD7
:10152000B646802E28BF4FF0800E00230FE0E85C07
:10153000504A116802095C0011F802C005AA02F8BD
:1015400013C000F00F000134095C115501337345DD
:10155000EDD305AA002302F81E3003F1804303F502
:101560008833D3F804350292434A0192434A0092E9
:1015700040F253124249052000F08AFC00230093F8
:101580004CAB2A46314646A800F0FCF9044610B19F
:10159000204655B0F0BD46A8FFF73CFE0028F7D026
:1015A000324B1B6813F0020F30D0314B1B68042BF9
:1015B0002CDDB446802E28BF4FF0800C0FE04CABE2
:1015C0001B5D2C4A106819096200455C05A901F8E9
:1015D000145003F00F030132C35C8B540134644593
:1015E000EDD305AA002302F81C3003F1804303F574
:1015F0008833D3F804350292224A01921F4A00929E
:101600004FF4AE721E49052000F042FC4B9B03B321
:10161000314646A800F0ABF8C5B23B4646AA29467B
:101620000DF23910FCF702FE0446394646A8FFF7D2
:1016300049FE90B13B462A460DF2391146A8FFF704
:1016400013FF0028A4D14999BDF82001FBF708FB3E
:101650009EE77846FBF782FADAE74999BDF8200160
:10166000FBF7FEFA94E70E2492E700BF741F0020F8
:10167000701F0020781F0020446F0300A86903003A
:10168000016F0300546F03004B78DB09C3724B7882
:1016900003F07F0383728A78CB781B0243EA02430C
:1016A0000A791343C3604A798B7943EA02230381A1
:1016B000704738B50C460546002840D0002C42D073
:1016C0002089FEF709F8012841D194F90A30002B4E
:1016D00041DBE368B3F1807F41D26369002B42D0E4
:1016E000236903F001022B7803F07F0343EAC2135E
:1016F0002B706269127803F0800302F07F021343BB
:101700002B70E27A6B7803F07F0343EAC213DBB2FB
:101710006B70A27A03F0800302F07F0213436B70B8
:10172000E3681A0CAA701A0AEA702B7123891A0A44
:101730006A71AB7163881A0AEA712B7238BD7846F8
:10174000FBF70CFABAE77846FBF708FAB8E77846F1
:10175000FBF704FAB9E77846FBF700FAB9E77846F1
:10176000FBF7FCF9B9E77846FBF7F8F9B8E7C37A75
:101770001BB10820081A093870470420FAE7093815
:101780007047073070470130704770B588B0044625
:101790000D461646002300938DF8043002691302AB
:1017A00003F47F0343EA0263110A01F47F410B4310
:1017B00043EA1263CDF805302846FFF7E2FF0368DD
:1017C000CDF8093082888379ADF80D208DF80F307F
:1017D000606904AA69461130FFF770FB3046FFF7D5
:1017E000D2FF04462846FFF7CEFF06234BB1013B4C
:1017F0009BB2C25C08A9194411F8101C4A40E2547B
:10180000F4E708B070BD00002DE9F041D2B0044605
:101810000D4617461E469DF8648100238DF847311A
:10182000ADF8283149934EAB46931046FFF7A9FF18
:1018300047903046FFF7A5FF4B90589B63613246B7
:1018400039462046FFF7A1FF31462046FFF71CFF2F
:101850002089FDF741FF012811D1A5F10902E37AA2
:1018600023B108239A4203D2002309E00423F9E7B5
:10187000E1682089FBF7CEF9E8B9012300E00023F5
:1018800083B3E37ACBB10821C9B28DF834116D1A54
:10189000073DADB2ADF82051479B1D444C95B8F1C2
:1018A000000F0ED0B8F1010F09D07846FBF756F9BA
:1018B0004FF0000805E00023E2E70421E4E74FF0E1
:1018C00003084EAB002241462046FFF71EFB63692A
:1018D000013345930DF2471145A8FFF712FB9DF820
:1018E000473123B99DF8470152B0BDE8F081F37943
:1018F000307A40EA03206080FDF7EEFE20701B4B3B
:101900001B6813F0020FEDD0194B1B68032BE9DDA8
:10191000BDF82061802E28BF802600230FE04B9A5F
:10192000D25C14490C6810095900255C04A800F821
:10193000135002F00F020131A25C42540133B34252
:10194000EDD304AA002302F8163003F1804303F517
:101950008833D3F804350292074A0192074A00926D
:10196000E4220749042000F093FABBE7741F00202B
:10197000701F0020781F0020DC6F0300A86903009F
:10198000CD6F03002DE9F04784B00E4615461F4683
:101990009DF83090804618B112B10BB19A4202D135
:1019A0007846FBF7DBF8082E30D91D2E30D8287882
:1019B000C009FDF76DFCC8F810000023C8F814300A
:1019C00095F800A00AF07F0A0293039301E0029BBE
:1019D000D3B103AA02A950460AF0C4F90024012C8D
:1019E000F5D804AB03EB840353F8080C0028EED0C1
:1019F000CDF8049000903B462A4631464046FFF71A
:101A000003FF48B90134EAE7052002E0092000E0BD
:101A1000092004B0BDE8F0870020FAE7F0B58FB0E8
:101A20000D4616461C46074650B16EB1012C0FD824
:101A30009CB1012C10D07846FBF790F800240CE004
:101A40007846FBF78BF8F0E77846FBF787F8EDE789
:101A50007846FBF783F8EBE703240AAB0022214624
:101A60003846FFF752FAFB7A03B308238DF8243087
:101A70007B69013301930AAB02933046FFF781FE85
:101A800003900790A91C89B2ADF810100023ADF89F
:101A9000183005930844089001A8FFF72EFA324643
:101AA00031463846FFF771FE0FB0F0BD0423DDE785
:101AB00038B50D460446C8B12378AB421AD9EDB902
:101AC00062682378134413F8013CA1780B44DBB21D
:101AD00012789B1ADBB2CBB16368585DA378013BE7
:101AE0001840A368627802FB003038BD7846FBF7E7
:101AF00035F8E1E77846FBF731F8E0E7626853191B
:101B000013F8013C525D9B1ADBB2E4E70020ECE7DE
:101B100038B50C460546A0B12B78A34215D9C4B9F7
:101B20006A682B78134413F8013CA9780B44DBB2A4
:101B300012789B1ADBB21BB16A68135D013313552F
:101B400038BD7846FBF70AF8E6E77846FBF706F873
:101B5000E5E76A68131913F8013C125D9B1ADBB2C2
:101B6000E9E710B5044640B1002322789A4208D92B
:101B700062680021D1540133F7E77846FAF7EEFFA7
:101B8000F2E710BD10B5044643786BB12378012B02
:101B90000ED9A36883B1636893B1A378A3B15A1E29
:101BA000134217D0002310E07846FAF7D7FFEDE78D
:101BB0007846FAF7D3FFECE77846FAF7CFFFEAE783
:101BC0007846FAF7CBFFE8E700232BB12046FFF772
:101BD000C8FF10BD0123F8E77846FAF7BFFFF5E725
:101BE00038B50C46054678B12B78A34210D99CB97C
:101BF0006A682B78134413F8010CAB781844C0B210
:101C00001378C01AC0B238BD7846FAF7A7FFEBE7E1
:101C10007846FAF7A3FFEAE76B681A1912F8010C85
:101C20001B5DC01AC0B2EEE728B108B529B1FFF7B5
:101C3000C5FA002008BD0E2070470E20FAE770B1EB
:101C400030B583B00B4661B100248DF80740012206
:101C50000DF10701FFF71CFA204603B030BD0E203E
:101C600070470E20F9E7000000B330B58BB00C468A
:101C70000546E9B11031FFF773FA0E4B09930E4B8D
:101C800093E803000790ADF8201003AA042109A8E7
:101C9000FFF7C6F901940623009307AB03AA1021AE
:101CA0002846FFF7D5F900200BB030BD0E20704755
:101CB0000E20F9E76E6B626BF06F030010B330B566
:101CC00087B00C460546F9B1104B019302AA0421D6
:101CD0000DEB0100FFF7A4F902AB102229461846CC
:101CE000FFF707F99DF816301B0203F47C536FEAE7
:101CF00043436FEA53439DF817201343238000208A
:101D000007B030BD0E2070470E20F9E7767461648D
:101D100070B50E46044648B141B12368B34209D0BC
:101D2000256865B926600023336017E07846FAF726
:101D300015FFF2E77846FAF711FFF1E725462C6820
:101D40002CB1B442FAD17846FAF708FFF6E735B17C
:101D50002EB1B54202D02B6833602E6070BD78463C
:101D6000FAF7FCFEF5E738B505460C4689B180B1B7
:101D70002B68BBB1A34210D01A461B680BB1A3421B
:101D8000FAD18AB1A34211D12368136000202060E8
:101D900038BD7846FAF7E2FEEAE723682B600020B8
:101DA0002060F5E70520F3E70520F1E70520EFE7E0
:101DB0002DE9F0410E461746054608B101B112B9AA
:101DC0007846FAF7CBFE2B68B34204D02C6834B1C6
:101DD0004FF0000809E07846FAF7C0FEF6E72E60FB
:101DE000002030600FE0A0462C4654B1314620461A
:101DF000B84730B92568AE42F5D17846FAF7AEFE5D
:101E0000F1E714B10F20BDE8F081B8F1000F09D05F
:101E100046B1B04504D0D8F800303360C8F800604F
:101E20000020F0E77846FAF799FEF2E730B583B084
:101E300010461A4606AC54F8045B00900B46054960
:101E400000200CF009F92246294600200CF010F879
:101E500003B030BDF86F0300034B1860034B1960EB
:101E6000034B1A60704700BF741F0020701F0020D2
:101E70007C1F002030B583B0044C246824B1079D3A
:101E80000195069D0095A04703B030BD7C1F002042
:101E900030B585B008AC54F8045B03940194009508
:101EA000FFF7E8FF05B030BD2DE9F04F85B00F46D4
:101EB00091460093834650B10120FDF7D3FBFCF718
:101EC000E3FC01904FF0000AD04601259CE07846E3
:101ED000FAF744FEF0E7019901F5805102910AF109
:101EE0000101914213D0327816447288013A92B2BD
:101EF00047F6FE618A420ED84EB1019A131D107941
:101F000072880299184400F04FFE00B10290019BC4
:101F10000433029E89E003F50053344603951D46C1
:101F200016E07846FAF71AFE15E024F47F6424F0F0
:101F30000F0404F5805423781C44A5421DD9A64201
:101F40001ED26388013B9BB247F6FE62934211D9D1
:101F50002388002BE5D0238804EB830323F47F62DE
:101F600022F00F029342E0D06288B2F5FE4FDCD03F
:101F70001C46E2E7039D2646BEE7039D0026BBE71D
:101F8000039D0026B8E7002343B108F10108B9F129
:101F9000000F03D000992046C8470546238823B385
:101FA000238804EB830323F47F6222F00F02934221
:101FB0001FD06288B2F5FE4F1BD01C46B44221DA16
:101FC000012D1FD16288531E9BB247F6FE618B42E2
:101FD000D9D837B179883B884A40134203D00023CF
:101FE000D2E70123D0E70123CEE77846FAF7B6FD22
:101FF000D6E724F47F6424F00F0404F5805423789A
:102000002344DAE70AF1010ADBF8102052450FD920
:10201000012D0DD1DBF80C4004EB0A3303F580569B
:102020000199096899423FF456AF1C781C44C5E7F2
:102030000020FDF717FB404605B0BDE8F08F00001B
:1020400008B50648FCF703FC08B9002008BDFCF7FA
:1020500013FC08B90120F9E70020F7E7C0280020A9
:1020600046DF70472DE9F04707460E468589012473
:1020700011E0013B9BB2C1181EF801201CF803A01F
:1020800082EA0A0208F80120002BF2D1A5EB09052B
:10209000ADB20134A4B2BDB1230A43EA0423F383F1
:1020A0003046FFF7DDFFA946102D28BF4FF010097D
:1020B000D7F81880601E0001D7F808E006F1200C60
:1020C0005FFA89F94B46DFE7BDE8F0872DE9F04775
:1020D0008146884617461C4600F1100500F120068F
:1020E00016E052464146281914F0C3F82744BFB2FF
:1020F000103FBFB2D0441DE0013B9BB2F45CEA5CF0
:102100005440EC54002BF7D14846FFF7A9FF0024B8
:1021100097B1C4F1100A5745E3DA3A464146281907
:1021200014F0A7F83819C0F110020021284414F067
:10213000C9F800271023E5E7BDE8F08770B505462C
:102140000C461646838A002B3BD0402295F820305F
:10215000023B03EBD3735B10DB0003F03803134344
:1021600043F0010323746B68186859689A68C4F8CF
:102170001100C4F81510C4F819201B7B6377AA89D5
:10218000130A43EA0223E3832046FFF769FFAB8A81
:102190006BB1B3F57F4F16D2AA8A130A43EA022322
:1021A00023820223AA8A29692046FFF78FFFAA8982
:1021B0006AB995F8202004F12001304614F059F84E
:1021C00070BD0022C2E77846FAF7C8FCE4E70023B6
:1021D000A9682046FFF77AFFEBE730B58DB00446DB
:1021E00003686D46186859689A68DB680FC5E2692C
:1021F00069462046FFF7A2FFE569636801228DF872
:102200001020186859689A68CDF81100CDF815109B
:10221000CDF819201B7B8DF81D300023ADF81E3042
:102220006846FFF71DFF94F820304BB1013B9BB28D
:10223000EA5C0CA9194411F8101C4A40EA54F4E76E
:1022400069462046FFF70EFF0DB030BD70B590B067
:1022500004460E4690F82030102B35D8236804AD84
:10226000186859689A68DB680FC5A38983BBA5689D
:10227000A369A3606A4604A92046FFF75FFF63686D
:1022800001228DF82020186859689A68CDF821003D
:10229000CDF82510CDF829201B7B8DF82D3000239B
:1022A000ADF82E3004A8FFF7DBFE94F820303BB3E6
:1022B000013B9BB210AAD11811F8402C11F8101C48
:1022C0004A400DF80320F2E77846FAF747FCC5E7E5
:1022D000636801228DF82020186859689A68CDF843
:1022E0002100CDF82510CDF829201B7B8DF82D304D
:1022F0000023ADF82E3004A92046FFF7B3FEB6E761
:10230000A56094F82020E169684613F07FFFB0FAD9
:1023100080F04009307010B070BD000030B583B05F
:1023200001900D46040C293CA4B2272C05D8054B7E
:1023300033F814302B8003B030BD7846FAF70EFC2A
:10234000F5E700BF7C2A002030B583B001900D4630
:10235000040C293CA4B2272C06D82A88044B23F865
:102360001420002003B030BD7846FAF7F7FBF4E7FD
:102370007C2A002030B583B001900D46040C013C4E
:10238000A4B2272C09D8074B03EBC40153F834201F
:102390004B682A606B6003B030BD7846FAF7DEFB0D
:1023A000F1E700BFD828002030B583B001900D467A
:1023B000040C013CA4B2272C11D80B4B03EBC40234
:1023C0002868696843F834005160084B1B781BB9D2
:1023D000074A136801331360002003B030BD78460C
:1023E000FAF7BCFBE9E700BFD8280020D42800207A
:1023F000D0280020F0B583B0FCF7F2FE054600249B
:1024000013E07846FAF7AAFB1FE0364B1B6822E080
:102410007846FAF7A3FB39E07846FAF79FFB3FE0EE
:102420007846FAF79BFB4BE001342F4B1B68A34225
:1024300054D92E4E06EBC4062A4B1F88F3889F42C0
:1024400003D001339BB29F42DBD1F2889742DCD2AA
:10245000244B1B68013B1B0C1B0413449D42E3D01F
:102460006A1E9A42E0D0204A1368013B1360204A5A
:1024700012680192A6B2721CADF806201B4901EB4E
:10248000C301019801F0DEFB0028C1D1164B1B6887
:102490000133ADF80630019801F006FC0028BBD1ED
:1024A000134B5B6801932936ADF806600E4B196833
:1024B000104B03EB4101019801F0C4FB0028AFD1A0
:1024C000094B1B682933ADF80630019801F0ECFB8D
:1024D0000028AAD07846FAF741FBA6E7014B1D6019
:1024E00003B0F0BDCC280020D0280020D828002040
:1024F000247003007C2A002008B50378022B00D04A
:1025000008BDFFF777FFFBE72DE9F04383B088466E
:1025100016461F460024474D2D68A5424FD9464D0B
:1025200005EBC405AB88834201D00134F3E7424D8B
:1025300005EBC405414BB3F80090EB88994503D0F7
:1025400001339BB2994514D1EA88914515D23B4B92
:102550001B68013B1B0C1B0413449E4210D09E427F
:1025600015D90123ABB907B13C60002003B0BDE829
:10257000F0837846FAF7F2FAE6E7304B1B68E9E7B2
:102580002D4A52F834209045E9D90123EAE7002387
:10259000E8E7294B03EBC402D68043F83480284B8C
:1025A0001B680193631CADF806302946019801F0C1
:1025B00049FB0028D7D07846FAF7D0FAD3E7272D81
:1025C00001D90420D2E71C4B03EBC5018880CE80E3
:1025D00043F835801A4B1B6801930135ADF806505E
:1025E000019801F02FFBE8B9124B1B6815494FF613
:1025F000FF7221F81320124A5268019203F1290256
:10260000ADF8062001EB4301019801F01BFB68B90E
:1026100017B1084B1B683B60064A1368013313600F
:102620000020A3E77846FAF799FADDE77846FAF74B
:1026300095FAEDE7D0280020D8280020CC280020EB
:10264000247003007C2A002010B50A48FDF7F4F935
:102650000024094B1C70094B1C604FF4A0722146EA
:10266000074813F02FFE50222146064813F02AFE99
:1026700010BD00BF801F0020D4280020D0280020DB
:10268000D82800207C2A002008B5044B01221A70AB
:10269000FCF7A6FD024B186008BD00BFD42800203F
:1026A000CC28002008B50023FFF72EFF08BD00004E
:1026B0002DE9F04784B006460C461546ADF80630C5
:1026C0008B4260D803AB2A4621463046FFF71CFFF9
:1026D0000646002853D1039F364B33F817204FF698
:1026E000FF739A423ED0BDF80680334B03EBC70917
:1026F000324BB3F800A0B9F806309A4503D0013345
:102700009BB29A4543D1B9F80620924543D22B4B50
:102710001B68013B1B0C1B041344274A52F837C0AB
:10272000244A32F81720190A1806CCF30C039342F6
:1027300034D2D21A6244A2F50052801841F100014D
:102740002B0A2A06C4F30C0545452AD2A8EB050836
:102750004444A4F50054121943F10003994208BF00
:1027600090420CD2164B5B680293039B2933ADF861
:102770000A300DF10601029801F064FAA8B930465A
:1027800004B0BDE8F0877846FAF7E8F99AE77846AA
:10279000FAF7E4F9B7E7094B1B68BBE7D21A6244C2
:1027A000CBE7A8EB05084444D5E77846FAF7D6F915
:1027B000E5E700BF7C2A0020D8280020CC28002094
:1027C000247003002DE9F0410E46154600241E4BEF
:1027D0001B68A34235D91D4B03EBC4039B8883427E
:1027E00001D00134F3E7194F07EBC407184BB3F8D6
:1027F0000080FB88984503D001339BB2984510D1E7
:10280000FA88904511D2124B1B68013B1B0C1B042C
:1028100013449D420CD09D4211D9012080F001004B
:1028200010E07846FAF79AF9EAE7094B1B68EDE7FA
:10283000064A52F834209642EDD90120EEE70020F6
:10284000ECE70020BDE8F081D0280020D828002047
:10285000CC2800208B426AD82DE9F8430F469046D9
:102860001E460024334D2D68A5425DD9324D05EB3F
:10287000C405AB88834201D00134F3E72F4B33F812
:1028800014204FF6FF739A4201D100204DE02A4DEB
:1028900005EBC4052A4BB3F80090EB88994503D0AB
:1028A00001339BB2994530D1EA88914531D2244B0E
:1028B0001B68013B1B0C1B0413441F4A52F8345085
:1028C0001E4A32F81420190A1806C5F30C03934265
:1028D00022D2D31A2B44A3F50053C01841F10001B2
:1028E0004FEA18234FEA0862C7F30C04B44216D229
:1028F000361B3744A7F50057D21943F1000399421C
:1029000008BF90420ED301200FE07846FAF726F96F
:10291000CAE70B4B1B68CDE7D31A2B44DDE7361B08
:102920003744E9E7002000E00020BDE8F8830120FB
:10293000704700BFD0280020D82800207C2A002023
:10294000CC2800208B4267D82DE9F8430F469046EB
:102950001E460024314D2D68A5425AD9304D05EB55
:10296000C405AB88834201D00134F3E72C4D05EB5D
:10297000C4052C4BB3F80090EB88994503D0013384
:102980009BB2994534D1EA88914535D2254B1B68D5
:10299000013B1B0C1B041344214A52F834202249EA
:1029A00031F81440190A1806C2F30C03A34226D2C8
:1029B000E51A1544A5F50055421941F100034FEA07
:1029C00018214FEA0860C7F30C05AE421AD9761BEE
:1029D0003744A7F50057C01941F100014FF6FF75C4
:1029E000AC4212D0994208BF904210D0002011E0B2
:1029F0007846FAF7B3F8C6E70A4B1B68C9E7E31A4B
:102A00009D18D9E7761B3744E5E7002002E0012056
:102A100000E00020BDE8F88300207047D0280020A7
:102A2000D8280020CC2800207C2A002010B50024C3
:102A3000084B1C604FF4A0722146074813F042FC7B
:102A400050222146054813F03DFC052001F056F9BF
:102A500010BD00BFD0280020D82800207C2A0020EC
:102A6000F0B5C7B00C4616460546F0B12CB3E1B23E
:102A70000139C9B22878E0B1012820D02C4B1B685D
:102A800013F4807F03D02B4B1B68012B1CDC284BDD
:102A90001B6813F4807F10D0264B1B68032B0CDDC2
:102AA000802C28BF802400232BE07846FAF756F8C4
:102AB000DCE73246681C0EF06BF947B0F0BD3246D9
:102AC000681C00F0C7FEF8E71B4BD3F804350190F3
:102AD0001A4A00924C221A490220FFF7D9F9D6E788
:102AE0006A1CD25C174807681609580017F806C018
:102AF00005AE06F813C002F00F020130BA5C325482
:102B00000133A342ECD305AA002302F8143003F1E9
:102B1000804303F58833D3F8043502920A4A0192C0
:102B20000A4A00924D2206490420FFF7B1F9C4E792
:102B3000741F0020701F002000100140A8700300C7
:102B40009D700300781F0020D0700300A869030067
:102B50002DE9F0410546E0B10F4616461C46DAB1B4
:102B6000E3B1FF291CD01C2B1CD803F102085FFA2B
:102B700088F808F1010109F076FC054648B180F8B3
:102B800011802B238374C77422463146143013F00E
:102B900070FB2846BDE8F0811546FAE70025F8E706
:102BA0000025F6E70025F4E7F8B506460D4617467A
:102BB000884201D8344613E07846F9F7CFFFF9E7A9
:102BC0007846F9F7CBFF21E024F47F6424F00F046A
:102BD00004F5805423781C44A5422AD9A6422BD25E
:102BE0006288BA4226D024F47F6323F00F0303F5F2
:102BF0008053AB4207D3B2F5FE4F16D0238804EBC7
:102C00008303AB4213D22388002BD9D0238804EB53
:102C1000830323F47F6222F00F029342D4D06288B0
:102C2000B2F5FE4FD0D01C46D6E7002402E00024C7
:102C300000E000242046F8BD0024FBE7014B1860AB
:102C4000704700BF202B0020F8B50E46054688B11E
:102C5000A6B12B78012B15D8304BD3E908231343A9
:102C600014D16B681D2B15D82B78012B16D02C4B4B
:102C70001C6820E07846F9F771FFE9E77846F9F734
:102C80006DFFE6E77846F9F769FFE5E77846F9F77B
:102C900065FFE6E77846F9F761FFE5E7EB68B3F132
:102CA000FF3FE4D003F50073012BE0D97846F9F734
:102CB00055FFDCE7246814B3A4F108002A6914F86E
:102CC000033C1A42F6D054F8083C1B682946984742
:102CD0000028EFD114F8041C0122A1F12003C1F156
:102CE000200002FA03F322FA00F003438A400B4962
:102CF0000F6A486A3A4303430A624B62DAE7074BBA
:102D0000D3E90823134304D06A68044B03F8012B6A
:102D10003360024BD3E90801F8BD00BFF82A002058
:102D2000242B0020F8B51A4BD3E90823134302D013
:102D3000184B1C6804E07846F9F710FFF8E72468A0
:102D400004B3A4F1080C124A136A506A14F8045C24
:102D5000C5F12001A5F12002EB4000FA01F10B437F
:102D600020FA02F2134303F00106002756EA070394
:102D7000E5D054F8083C5B68054911F8012B604622
:102D80009847DCE7024B00200021C3E90801F8BDA9
:102D9000F82A0020242B0020F8B5194BD3E908238A
:102DA000134302D0174B1C6804E07846F9F7D6FEAF
:102DB000F8E72468ECB1A4F1080C114A136A506AD0
:102DC00014F8045CC5F12001A5F12002EB4000FAE3
:102DD00001F10B4320FA02F2134303F0010600272E
:102DE00056EA0703E5D054F8083C9B6860469847CC
:102DF000DFE7034B00200021C3E90801F8BD00BF55
:102E0000F82A0020242B00202DE9F0410F46164619
:102E10001C46804650B1074B1D682DB123463246F3
:102E200098F804103846A847BDE8F0817846F9F7CD
:102E300095FEF0E7202B002070B50C46154606469F
:102E4000D8B1F4B10DB3FF2D23D023682BB3636841
:102E50003BB3A368002B28D0184B1B783F2B28D8F6
:102E60003460164A1378591C11703371757106F16C
:102E700008011348FEF74CFF70BD7846F9F76EFE67
:102E8000DFE77846F9F76AFEDCE77846F9F766FE91
:102E9000D9E77846F9F762FED7E77846F9F75EFE9C
:102EA000D5E77846F9F75AFED3E77846F9F756FEA4
:102EB000D2E77846F9F752FED2E700BFF42A0020A5
:102EC000242B0020054B5B6833B14FF6FF72934211
:102ED00002D0013B014A5360704700BF342B0020F1
:102EE00000B583B0019040F20713B3EB104F09D146
:102EF000064B00221A605A609A60DA601A6103B0C9
:102F00005DF804FB7846F9F729FEF1E7342B002041
:102F10002DE9F04104460F4616461D465B68C3B1D5
:102F20000A232370002323732B88E381DFF82C808E
:102F3000B8F800006082FCF7CFFB20746B68A361D7
:102F40006760A66098F80C302377FF232362BDE802
:102F5000F0817846F9F702FEE2E700BF342B00204B
:102F600000B58DB003460D4A127B02F07F028DF84A
:102F700000200B4A127800218DF801108DF80220F4
:102F80000322694603A8FFF7C3FF6FF0020103A8FD
:102F9000FAF70AFF0DB05DF804FB00BF342B0020E8
:102FA0005C2B00200E4B1B88CBB100B583B00D4BC2
:102FB0001B683BB10B4B1B686846984730B103B0A8
:102FC0005DF804FB7846F9F7C9FDF3E76846FFF7BB
:102FD000C7FF003818BF0120034B1870EFE7704798
:102FE000342B0020982B00207D2B002008B5094BA6
:102FF0001B7818420CBF012200228A4200D008BD73
:103000004340044A1370044BDB890342F7D0FFF7B7
:10301000C9FFF4E75C2B0020342B002000B583B0FF
:103020000191C1F30741012902D003B05DF804FB0F
:103030000028FAD111780120FFF7D8FFF5E700004A
:1030400008B50378012B00D008BD034B1B78002B7B
:10305000FAD0FFF7A7FFF7E77D2B002008B5144B48
:103060001B8823B1124B5B6813B1012300E00023DE
:103070008BB1104B1B6893B10E4A13681846B3F519
:10308000E16F28BF4FF4E1600B4901FB00F11161D2
:103090001B1A136008BD074B00221A61FAE7FFF7FD
:1030A00011FFFFF77FFF024B9A68024B1A60E3E7BC
:1030B000342B0020602B002040420F0030B583B03D
:1030C00001900C4640F20713B3EB104F09D1074DA6
:1030D0000FCD20606160A260E3602868206103B0CA
:1030E00030BD7846F9F73AFDF1E700BF342B0020F8
:1030F00010B50D4B1B789BB10C4B9B681C46B3F570
:10310000E16F28BF4FF4E1641B1B094A1360FCF711
:1031100079FF084901FB04010748FCF73FFF10BD98
:103120000024034B1C60F2E77C2B0020342B002092
:10313000602B002040420F00642B002008B5044B98
:1031400000225A609A600348FCF710FF08BD00BFD8
:10315000342B0020642B002070B582B001900C4607
:1031600040F20713B3EB104F36D12088FCF7B4FAC6
:1031700002283FD06368B3F5004F03D94FF6FF72C2
:10318000934239D1A368B3F5803F37D894F90C3016
:10319000002B35DB1B4D26460FCE0FC533682B6049
:1031A00023882BB9A5F1100300225A609A601A7384
:1031B000154B1B78A3B1134B5B684FF6FF7293421C
:1031C00014BF0023012313B10E4B9B6873B9FFF7A3
:1031D000B5FF002002B070BD7846F9F7BFFCC4E728
:1031E000084B5B68003B18BF0123ECE7FFF780FF4B
:1031F0000020EFE70720EDE70720EBE70720E9E7EE
:103200000720E7E7342B00207C2B00200D4B9B6828
:103210001BB1013B0B4A9360704710B58CB00A4854
:10322000FCF7A4FE074C0021A1602C2201A813F09A
:1032300049F806238DF80430029401A8FBF796F8AC
:103240000CB010BD4C2B0020802B002003780A2BE3
:1032500047D1C389234A1288934242D1418A214AE5
:10326000528891423DD18268032A3AD11D4A926820
:10327000002A36D000B58DB01A4A5268B2F5004F18
:1032800002D2013217494A6005228DF804204168B4
:103290000A7802F07F028DF808200A7802F07F0297
:1032A000007F121AD2B20132D2B28DF80920897889
:1032B00001F00F01ADF80A10ADF80C3093B2094AD5
:1032C0009289934201D2074A9381064AD289934256
:1032D00001D9044AD38101A8FBF748F80DB05DF885
:1032E00004FB70474C2B002008B501210C48FAF76D
:1032F000F3FF80B90B4B0C4ADA600C4B0C4A9A6016
:103300000C4ADA600C480D4B0360FBF757F80C4B86
:1033100001221A7008BD7846F9F720FCEAE700BFE1
:10332000F0700300602B00205D300200802B002035
:103330000D32020040420F00282B002041300200D5
:103340007C2B002070B590B0044600283ED00FA919
:103350000DF13E0008F01AFEA368B3F5803F43D894
:103360002088FCF7B9F9012804D02088FCF7B4F9CB
:10337000002839D16088FCF7AFF958BB254B0BAD5D
:103380000FCB85E80F00A3681BB122880AB16188C2
:1033900061BB204B00221A805A809A601E48FCF7BD
:1033A000E5FD2C220021684612F08CFF06238DF8E3
:1033B0000030BDF82E305BB30BAB0193154B02937D
:1033C0006846FAF7D3FF002010B070BD7846F9F7D1
:1033D000C5FBBCE76088FCF77FF90328CED0628884
:1033E000BDF83E309A42C9D00720EDE7094C228053
:1033F0006180A360084DEE68FCF704FE3118284692
:10340000FCF7CCFD7F23A3810023E3816360C8E741
:103410000023D2E74C2B0020802B0020004870476F
:103420004C2B002000487047342B002008B5014683
:10343000034B00221A70034B186800F003FC08BD10
:103440007C2B0020E470030008B5044B186000B129
:1034500008BD7846F9F782FBFAE700BF982B0020F9
:10346000114B196848680288013202EB820293000E
:103470005B089BB2B3F5167F28BF4FF416730A2B77
:1034800038BF0A2383804A6893780133DBB2937094
:10349000022B00D07047044A1368596800238B70D0
:1034A000126852681380F5E79C2C002000B583B0A9
:1034B0000190084B01221A70074808F09BFFFCF7A7
:1034C000A1FD064BD96801441846FCF767FD03B01F
:1034D0005DF804FB7C2C00209C2B0020842C002019
:1034E00010B582B001900C46000CB0F5837F04D17A
:1034F000044B1B78237002B010BD7846F9F72EFB01
:10350000F6E700BF7C2C002010B582B001900C467D
:10351000000CB0F5837F0BD12478114B1B7803B9D5
:1035200054B903B1A4B10E4B1C70002002B010BD01
:103530007846F9F713FBEFE70A4808F05BFFFCF762
:1035400061FD094BD96801441846FCF727FDEAE7FD
:10355000044808F081FF0448FCF708FDE3E700BFDA
:103560007C2C00209C2B0020842C002030B585B0C2
:103570000546084614466B460D222946FDF7B9FC60
:103580006B4603CB2060616005B030BD2DE9F0478C
:1035900092B004460DF147025449002008F052FC55
:1035A0000CE0191B9288524B03FB02F38B4213D998
:1035B0000DF147024D49002008F044FC4B4B1B68BD
:1035C000002B5BD05868FFF74BFF484B1B685A68CD
:1035D0009368E11AE6D5E4E7FBF702FE0546FBF740
:1035E00063FE9DF84730022B4BD0404A11680831EA
:1035F000022B14BF002201229DF8303062F3000339
:10360000012814BF0022012262F341036FF38703F4
:103610008DF830300B4653F8102F5B68CDF8312011
:10362000CDF835302B0203F47F0343EA05632A0A01
:1036300002F47F42134343EA1563CDF839300DF1AC
:103640003D020CA8FFF792FF15230CAA012129487F
:10365000FFF77EFA014688B101230371254808F07F
:103660003FFF254B1B6813F0020F03D0234B1B6851
:10367000042B0ADC1D4B1B685B689C6012B0BDE824
:10368000F0871A4A11682031B2E71D4BD3F8043590
:103690009DF831109DF832009DF833609DF834702C
:1036A0009DF835C09DF836E09DF837809DF838903C
:1036B0009DF83020C2F3400A02F001020B950A92F5
:1036C000CDF824A0CDF82090CDF81C80CDF818E0DE
:1036D000CDF814C00497039602900191094A009214
:1036E000F72209490520FEF7D3FBC3E79C2C0020F5
:1036F00040420F009C2B0020741F0020701F0020F0
:1037000000100140707103006171030008B5FCF7FF
:1037100079FCFFF73BFF08BD08B5FFF737FF08BD91
:1037200030B583B005460C4608220131103012F046
:103730006DFD10B1002003B030BD6A462946204619
:10374000FFF714FF082204F10D01684612F05EFD38
:10375000B0FA80F04009EEE710B582B00023154AB8
:103760001360154C154AE260154AA26023610421DA
:103770000DEB0100FCF780FDFCF744FCE2680199C9
:10378000B1FBF2F302FB1313184460600D4C3423B9
:103790000D4A0E49204608F0D7FF4FF47A712046B3
:1037A00008F04CFF0A4A04210A48FDF739FC02B030
:1037B00010BD00BF9C2C0020842C00208096980017
:1037C000193702009C2B0020382C00200D370200F6
:1037D0006C2C0020B471030008B5074B1B7803B1B3
:1037E00008BD064808F006FE0548FCF78FFB024BB3
:1037F00001221A70F4E700BF7C2C00209C2B0020D3
:10380000842C002000B585B08DF807000DF107016C
:10381000054B186800F016FA10B905B05DF804FB06
:103820007846F9F79BF9F8E70072030000B583B01A
:103830000DF10701064B186800F016FA20B99DF843
:10384000070003B05DF804FB7846F9F787F9F6E75F
:10385000007203002DE9F04F9BB017460446F8B103
:1038600000231893D4F809301D0205F47F0545EABA
:1038700003651A0A02F47F42154345EA1365464B75
:103880001B6813F0020F03D0444B1B68042B0BDCA6
:10389000661C0DF1670218A9304608F0D3FA61E002
:1038A0007846F9F75BF9DBE73D4BD3F804356178EF
:1038B000A078E67894F804C094F805E094F80680BF
:1038C00094F8079094F808A02278C2F3400B02F015
:1038D00001020B950A92CDF824B0CDF820A0CDF8C6
:1038E0001C90CDF81880CDF814E0CDF810C00396E8
:1038F000029001912B4A00924FF4D2722A4905207E
:10390000FEF7C6FAC4E77846F9F728F92FE09DF8E4
:1039100067300BB3214618982030FFF701FFD8B16C
:10392000189A20322CE001330B8004238DF83430B8
:10393000214611F80D3BC3F340008DF84C00C3F352
:1039400000038DF84D301295189B0E930F9210972F
:1039500011910DA8FAF70AFD0DF1670218A930467A
:1039600008F070FA189B9BB15B68002BCBD0214606
:1039700018980830FFF7D4FE0028C8D0189A0832EB
:10398000189B59680B884FF6FF708342CBD1CCE768
:103990001BB0BDE8F08F00BF741F0020701F002017
:1039A00000100140BC7103006171030082B00191FD
:1039B00089B203681A88914202D0002002B0704791
:1039C0005B88BDF80620934205D8C1880B4493421A
:1039D00003DC0020F2E70020F0E70120EEE7000022
:1039E00010B582B00190074C074B9C4206D001995C
:1039F0002046FFF7DBFF10B91C34F5E70024204612
:103A000002B010BDC0630300EC6603000246054827
:103A1000054B984204D00388934202D00830F7E760
:103A20000020704704670300346703002DE9F0416C
:103A300082B00546884601921F460B4C00E00834D0
:103A40000A4A94420CD0226811682846FFF7AEFF5C
:103A50000028F4D066683A4601994046B047EEE740
:103A600002B0BDE8F08100BFEC660300046703000C
:103A700000B58DB02C22002101A812F023FC1223E6
:103A80008DF8043001A8FAF771FC01200DB05DF843
:103A900004FB000070B5164D1DE07846F9F75EF89E
:103AA00023E01C34B44215D0A54213D02A681088F4
:103AB000236819888842F4D152885988E3880B44D6
:103AC0009A42EEDAEB881A449142EADA7846F9F73C
:103AD00045F8E6E71C35074EB54208D02B685B88F1
:103AE000EA881344B3F5803FD7D2014CDAE770BDC2
:103AF000C0630300EC66030030B583B00446019157
:103B000003685D88C5EB1145C388AB4203D9A06942
:103B1000284403B030BD7846F9F720F8F7E70000F5
:103B2000F0B58FB001900D46144680B24FF6FE738B
:103B3000984216D155F8040B0190141F01231D4A19
:103B400013701E460198FFF74BFF0746C8B18388E4
:103B5000A34218D8C36829460198984738B101266E
:103B600012E0114601A806F0BBFF0026EAE736B1D5
:103B7000032401993846FFF7BFFF047016E00224C2
:103B8000F7E7022600E000262C22002103A812F00D
:103B900099FB14238DF80C308DF810600198CDF846
:103BA00012000695079403A8FAF7E0FB01200FB076
:103BB000F0BD00BFAC2C002070B582B004460846B2
:103BC00001911546E36811469847064610B1304604
:103BD00002B070BD01992046FFF78EFF037843F0D5
:103BE0000303037023681888FFF710FF50B1074BD9
:103BF0001868FDF745F82B46019A00212046FFF78B
:103C000015FFE4E77846F8F7A9FFF0E7A02C0020BD
:103C100008B50023064A1360064A1360064A13706B
:103C2000FFF738FF0548FDF70BF8054B186008BD96
:103C3000A42C0020A82C0020AC2C0020713A0200FB
:103C4000A02C002010B582B0019049B10C46FFF7BE
:103C5000C7FE38B122460199FFF7AEFF02B010BD92
:103C60000E20FBE70520F9E730B583B00190B1B134
:103C70000D46FFF7B5FE044698B1037A33B12369C8
:103C8000294601989847002003B030BD0199FFF7FD
:103C900033FF037813F0020FF1D10820F4E70E2070
:103CA000F2E70520F0E7000010B582B00190FFF7C1
:103CB00097FEE8B104460199FFF71EFF037813F061
:103CC000020F17D003F0FD0343F001030370636993
:103CD0000BB101989847084B1868FCF7D1FF0023F7
:103CE000019A01212046FFF7A1FE002002B010BD7D
:103CF0000520FBE70820F9E7A02C002070B582B072
:103D00000646FFF783FE60B3174C21E00023019ABB
:103D100001212046FFF78AFEA269535D23F00303C9
:103D200053550135E388AB4211D9A3695B5D13F0AC
:103D3000020FF6D023681868019005EB1040ADF82B
:103D400006006369002BE1D001989847DEE71C3438
:103D5000064B9C4205D023681B88B342F7D100254F
:103D6000E0E702B070BD00BFC0630300EC66030073
:103D700010B5134800F02CF8124B1B780BB9124CFD
:103D800008E0104B00221A704FF6FE70FFF7B6FFE6
:103D9000F5E708340D4B9C4210D0A378022BF8D1E4
:103DA00022884FF6FE739A42F3D0606800F06AF8FA
:103DB0000028EED12088FFF7A1FFEAE710BD00BF81
:103DC000213B0200AC2C0020046703003467030091
:103DD00038B5054608B1002408E07846F8F7BEFE7D
:103DE000F9E72946586800F031F80134064B1B68A2
:103DF000A34207D9054B1B6803EBC4039A78002A3A
:103E0000F3D0EEE738BD00BFB02C0020B42C00206A
:103E100000B583B00B4649684288CA805968098852
:103E2000ADF80410ADF80620014631F8042B02F17C
:103E30008042013A1B68920001989847024B185C37
:103E400003B05DF804FB00BF0872030030B583B017
:103E50000C46054658B174B1009401956B46084A6A
:103E6000002105F10800FEF71FF803B030BD7846C9
:103E7000F8F774FEEFE77846F8F770FEECE700BF5E
:103E8000113E020043691A795979521A03EB023341
:103E900002699B1AC06998428CBF002001207047BC
:103EA00010B50A4B834202D07846F8F757FE084B0C
:103EB0001B6833B1064C206800F01BFB0023236015
:103EC00010BD7846F8F74AFEF4E700BFB82C002092
:103ED000D02C0020F8B50D461446114B834202D079
:103EE0007846F8F73BFE0F4B1B681B69A34212D3C1
:103EF0000C4E37682246294607F1140012F0B9F932
:103F000039460948FBF7C1FD00233360074B1868A9
:103F1000FCF7B6FEF8BD7846F8F720FEE8E700BFEC
:103F2000B82C0020D02C0020C42C0020CC2C002049
:103F300010B50C46104B834202D07846F8F70EFEBF
:103F4000236913F0200F13D00C4B1B680BB1012019
:103F500010BD6068143000F0C8FA084B186048B112
:103F600023780372E368C360636803610020EFE7AE
:103F70000120EDE70220EBE7B82C0020D02C002038
:103F800030B587B000230093019302930393049309
:103F9000059303238DF800301048FBF792FD04468B
:103FA000CCB1E3680193257AFCF72CF80246E3686C
:103FB00029460B48FEF728FF6A46216904F11400E0
:103FC000FDF796FA0548FBF77CFD0546204600F014
:103FD00090FA2C46E4E7012007B030BDC42C002045
:103FE000B82C002008B50748FCF72AFE064B1860DD
:103FF000202206490648FEF71FFF0648FBF73AFD58
:1040000008BD00BF813F0200CC2C00200C720300D1
:10401000B82C0020C42C002082B0002002B07047D1
:1040200082B002B07047000030B583B001900D46F9
:10403000C0F30744012C17D80D4804EB84035A0140
:1040400000EB43131B792B7083586B7004EB8404D3
:1040500000EB4414636F03F5FA73064AA2FB0323D3
:104060009B096B8003B030BD7846F8F777FDE3E736
:10407000542D0020D34D621030B583B001900D4611
:10408000C0F30744023CE4B2012C09D804EB8404D9
:10409000054B03EB441494F82C302B7003B030BD67
:1040A0007846F8F75BFDF1E7542D002010B582B09B
:1040B0000190C0F30744012C19D804EB8403154A7E
:1040C00002EB43131B79B3B1012C1CD004EB840326
:1040D0005B01104A0121D15004EB84040D4800EB30
:1040E00044101421043008F0A9FA02B010BD78463B
:1040F000F8F734FDE1E704EB840002EB40100430F4
:1041000008F078F9E0E704EB84035B01014A012140
:10411000D150E1E7542D002030B583B001900D4619
:10412000C0F30744012C0CD86B78013BDBB2072BA2
:1041300038D86B88143B9BB2B3F5967F05D907201E
:1041400031E07846F8F70AFDEEE704EB8403174AFE
:1041500002EB43131A792B7803B18AB103B9C2B9C0
:104160006A78124804EB84035B01C25004EB8404B8
:1041700000EB44106988043008F060FA002012E077
:1041800004EB8400094B03EB4010043008F032F9D3
:10419000E6E704EB8400054B03EB4010043008F025
:1041A0005BF9DDE7072003B030BD00BF542D0020D0
:1041B00010B582B00190C0F30744023CE4B2012C78
:1041C0000AD804EB8404064800EB441008210430AC
:1041D00008F076FA02B010BD7846F8F7BFFCF0E7B9
:1041E000542D002030B583B001900D46C0F3074434
:1041F000023CE4B2012C0BD804EB8404064800EB2B
:1042000044102978043008F05BFA002003B030BD78
:104210007846F8F7A3FCEFE7542D002010B584B0E2
:104220000190C0F30744043CE4B2012C0DD802A86D
:1042300008F060FA04EB8404064800EB441002A97D
:10424000043008F0D6F904B010BD7846F8F786FCC3
:10425000EDE700BF542D002030B583B001900D462E
:10426000C0F30744043CE4B2012C08D82B7813F0C7
:10427000FE0308D0022B06D0072003B030BD7846DD
:10428000F8F76CFCF2E704EB8404044800EB4410FC
:104290002946043008F0ADF90020EEE7542D002047
:1042A00030B583B001900D46C0F30744043CE4B23E
:1042B000012C0ED804EB840464016834074B1C44C1
:1042C00054F8043F2B60A288A379AA80AB7103B095
:1042D00030BD7846F8F742FCECE700BF542D0020D3
:1042E00010B50D4B834202D07846F8F737FC0B4BE4
:1042F0005B686BB1094C207800EB8000084B03EB46
:1043000040106168043008F033F90023636010BD89
:104310007846F8F723FCEDE7482D0020942E002086
:10432000542D0020F8B50F461546134B834202D09A
:104330007846F8F713FC114B5B68C3B10F4E7468F5
:104340002A23A3746B1C63742A46394604F11300B4
:1043500011F08FFF307800EB8000094B03EB401029
:104360002146043008F0BCF800237360F8BD78469D
:10437000F8F7F4FBE2E700BF482D0020942E002060
:10438000542D002010B50C46144B834202D07846C1
:10439000F8F7E4FB124B5B6813B17846F8F7DEFBE5
:1043A0002078616800EB80000E4B03EB4010023177
:1043B000043008F058F80A4B586068B1E3680360AD
:1043C000237803EB83035B01064AD35803712278F9
:1043D000034B1A70002010BD0220FCE7482D00207E
:1043E000942E0020542D002010B50B4604380549AA
:1043F000401A4011044C04FB00F0C1B20348FEF720
:1044000003FD10BD542D0020CDCCCCCC482D002078
:1044100001280ED800B583B0074B1B68019300F547
:104420008070ADF806000198FFF70CFC03B05DF852
:1044300004FB0720704700BF1C72030001280ED840
:1044400000B583B0074B1B68019300F58070ADF891
:1044500006000198FFF708FC03B05DF804FB072095
:10446000704700BF1C72030070B5104C0126254632
:1044700045F8046B4FF480730D4A0E49284608F046
:1044800063F9284607F0B6FFC4F8A060A43480237F
:10449000094A0021204608F057F9204607F0AAFFF4
:1044A000324606490648FEF7C7FC70BD542D002071
:1044B000A82E0020E9430200A82F00203472030038
:1044C000482D002010B50446012806D804EB8404CA
:1044D000044800EB4414207910BD7846F8F73EFB01
:1044E000F4E700BF542D0020704708B511F0F0FD2F
:1044F00008BD08B511F034FE08BD0000002839D011
:10450000002939D01D4A10601D4B19604FF0A0439F
:104510000C22C3F82027C3F81C270322C3F818274E
:104520004021C3F80815C3F81427164B0622C3F818
:104530000C250822C3F814250722C3F810250522EC
:10454000C3F808250121C3F86C150F4AC3F82425C8
:104550000422C3F800258420C3F804030020C3F814
:104560000801C3F81C011960084BC02183F802132D
:104570001A6070470E2070470E2070472C300020C4
:10458000303000200020004000E0D70100E100E0D2
:1045900008B5134B1B789BB1124BD3F808317BB194
:1045A000104B0022C3F80821D3F808310E4B1B68CA
:1045B000002BEED00B4AD2F81805C0B29847E8E7B6
:1045C000084BD3F81C314BB1064B0022C3F81C2119
:1045D000D3F81C31054B1B6803B1984708BD00BFD9
:1045E00028300020002000402C30002030300020F7
:1045F00008B5FFF7CDFF08BD014B1870704700BF2D
:104600002830002008B5024B1868FCF739FB08BDBC
:104610003830002008B51B4B1B78ABB11A4B1B6818
:10462000B3B1194B1968194B1B880A79501C834286
:1046300017D0934214DC19440A79013313490B80D3
:10464000134BC3F81C250BE07846F8F787FAE5E72B
:104650000F4B0122DA600B4B00221A70FFF7D2FFDA
:1046600008BD0133094A13800A48FAF7CBF8002342
:10467000054A1360064A0121D160024A1370FFF710
:10468000C1FFEDE7543200207034002034300020A8
:10469000002000406034002008B50D4B1B780BB1A2
:1046A000012008BD0B490C48FAF740F80028F7D163
:1046B0000122074B1A70074B1B681979074BC3F887
:1046C0001C1507490A800021C3F81C119A60E7E70E
:1046D000543200207034002060340020002000405C
:1046E0003430002008B54FF4027211491148F9F72F
:1046F0002EFF4FF4027210491048F9F728FF1049B5
:104700001048FFF7FBFE78B90120FFF775FF002383
:104710000D4A13700D4A13800D4A13800D48FCF7A3
:104720008FFA0D4B186008BD7846F8F717FAEBE7DB
:1047300058320020603400204030002048320020F1
:1047400015460200E548020054320020563200208F
:1047500034300020994602003830002030B583B054
:1047600004460D46421C92B201A90548F9F76FFFB5
:1047700018B9019B1A1D2A601C7103B030BD00BF1F
:104780006034002038B50446B0B1251F14F8023C4F
:10479000012B15D1227834F8043C9A4214D8FCF746
:1047A000D7F9FFF72FFF34F8042C29460848F9F70A
:1047B00087FFFCF711FA38BD7846F8F7CFF9E4E740
:1047C0007846F8F7CBF9E5E77846F8F7C7F9E6E772
:1047D0006034002030B583B004460D4601A90320A3
:1047E000FFF7BCFF08B103B030BD019B84225A70B3
:1047F000019B9D70019BDC700198FFF7C3FFF2E7FE
:1048000010B50446012807D90F48F9F78EFEA042DB
:1048100002D3B4F5807F08D9013C0C4B1C800021E9
:104820008420FFF7D7FF002010BD22460849064824
:10483000F9F70DFF08B90120F6E7064B1C800020B0
:10484000FFF7DAFE0020EFE7483200203C3000207E
:104850006C3400205632002038B505460C4B1C88BD
:104860000CB901310C462046FFF7CAFF70B1084B66
:104870001B885BB1064B00221A80064B1B682A88F6
:10488000013C13441C712B8801332B8038BD00BFC1
:10489000563200206C34002038B503889BB10446A2
:1048A0000E4A11680A79013293420DD0497884206A
:1048B000FFF790FF094D29680948F9F7A3FF002386
:1048C0002B600023238038BD0A880548F9F7F8FEDD
:1048D000024B00221A6000F099FBF2E76C340020D2
:1048E00048320020134B1B881BB1013B114A138037
:1048F000704710B50446104B1B8883B10F490B68F5
:104900000D4A108803441C71138801339BB2138035
:104910000A681AB112790132934207D010BD0146DC
:104920000548FFF799FF0028E8D1F7E70248FFF7AD
:10493000B3FFF3E73C300020743400206C340020D7
:1049400010B582B0044601A90A48F9F7EFFE10B18C
:10495000002002B010BD019931F8042B204611F05F
:1049600088FC01990348F9F74DFF0120FFF744FE49
:104970000120EEE74832002070B50446084651B9E0
:1049800015461E4600F05EFB014633462A46204689
:1049900000F096FB70BD00F055FB014600231A465F
:1049A000204600F08DFBF5E770B5054600239342E5
:1049B0001BD2687801EBC30611F83340A04201D046
:1049C0000133F4E773782A78934204D20133B17843
:1049D0000B449A4205DD00231A46842100F070FB47
:1049E00009E073682846984705E000231A468221AB
:1049F000687800F065FB70BD30B5ADF53F7D0446CD
:104A00007D23ADF806300DF1060202A9408804F0BE
:104A1000F1FA054608B1092816D1BDF80620ADF80F
:104A2000FC21520002A90DF5FF7011F022FC647800
:104A3000284600F007FB0146FC237FAA204600F031
:104A40003FFB0DF53F7D30BD647800F0FBFA014679
:104A500000231A46204600F033FBF2E710B582B07F
:104A600004460DF102024168408804F08DFA0146C7
:104A7000BDF80230ADF80430022301AA6078FFF7D8
:104A80007BFF02B010BD10B582B004466946408875
:104A900004F052FA0146009B019304230DEB03023C
:104AA0006078FFF769FF02B010BD10B582B0044610
:104AB00001A9408804F02EFA0146012301AA60787A
:104AC000FFF75AFF02B010BD10B582B0044601A92D
:104AD000408804F00DFA0146012301AA6078FFF72F
:104AE0004BFF02B010BD10B582B004460DF10201BB
:104AF000408804F0EDF90146BDF80230ADF804300D
:104B0000022301AA6078FFF737FF02B010BD10B58D
:104B100004468188408804F0BBF9647800F092FA7A
:104B2000014600231A46204600F0CAFA10BD10B50F
:104B300082B0044601A9408804F086F901460123A9
:104B400001AA6078FFF718FF02B010BD10B5044647
:104B50000179408804F046F9647800F073FA014660
:104B600000231A46204600F0ABFA10BD10B582B003
:104B700004460DF10201408804F0CEF80146BDF86C
:104B80000230ADF80430022301AA6078FFF7F4FE8A
:104B900002B010BD10B504468188408804F08CF83E
:104BA000647800F04FFA014600231A46204600F0D0
:104BB00087FA10BD30B5ADF53F7D04467D23ADF8D5
:104BC00006300DF1060202A9408804F033F80546CC
:104BD00008B1092816D1BDF80620ADF8FC21520015
:104BE00002A90DF5FF7011F044FB6478284600F02F
:104BF00029FA0146FC237FAA204600F061FA0DF550
:104C00003F7D30BD647800F01DFA014600231A464E
:104C1000204600F055FAF2E710B504468188408836
:104C200003F0CEFF647800F00DFA014600231A4627
:104C3000204600F045FA10BD10B504468188408832
:104C400003F086FF647800F0FDF9014600231A4660
:104C5000204600F035FA10BD30B5ADF53F7D044675
:104C60007D23ADF806300DF1060202A9408803F05D
:104C70001FFF054608B1092816D1BDF80620ADF87A
:104C8000FC21520002A90DF5FF7011F0F2FA6478D0
:104C9000284600F0D7F90146FC237FAA204600F001
:104CA0000FFA0DF53F7D30BD647800F0CBF9014679
:104CB00000231A46204600F003FAF2E710B5044636
:104CC0008188408803F0AAFE647800F0BBF90146B1
:104CD00000231A46204600F0F3F910BD10B5044633
:104CE0008188408803F050FE647800F0ABF90146FB
:104CF00000231A46204600F0E3F910BD10B582B03B
:104D000004460DF1050201A9408803F007FD0146A4
:104D1000022301AA6078FFF72FFE02B010BD10B584
:104D2000044642790179408803F090FD647800F0F0
:104D300089F9014600231A46204600F0C1F910BD4A
:104D400010B582B004460DF10201408803F06CFCFE
:104D50000146BDF80230ADF80430022301AA6078A4
:104D6000FFF70AFE02B010BD10B5044681884088E6
:104D700003F02AFC647800F065F9014600231A4626
:104D8000204600F09DF910BD10B504464378F42B81
:104D900005D8152204492046FFF706FE10BD7846C7
:104DA000F7F7DCFEF5E700BF4072030030B587B0CF
:104DB00004464078A0F14003142B5FD8DFE803F0ED
:104DC0000B110B0B0B0B5E5E5E5E5E5E5E5E5E5EEF
:104DD0005E5E5E32450000231A46822100F070F9C3
:104DE00056E02378012B05D000231A46842100F0D9
:104DF00067F94DE0684607F07DFC9DF80030C3F38D
:104E000046038DF80830DDF80130CDF80930BDF8E3
:104E10000530ADF80D30072302AA0021607800F0BC
:104E20004FF935E02378112B05D000231A46842151
:104E300000F046F92CE0A01CF7F7A2FE00231A466A
:104E40001946607800F03CF922E02378012B05D068
:104E500000231A46842100F033F919E0F7F7C0FE69
:104E6000034602AD006859689A68DB680FC51023D5
:104E700002AA0021607800F023F909E04038C0B2AE
:104E80001F2807D800231A468221607800F018F9FD
:104E900007B030BD7846F7F761FEF3E710B504467A
:104EA0004078782805D000231A46822100F008F9BE
:104EB00010BD204610F8021B00220139F7F79CFDB7
:104EC000647800F0BFF8014600231A46204600F03F
:104ED000F7F8EDE708B5064B1B780BB1082008BDC5
:104EE000FFF700FC024B01221A700020F7E700BF19
:104EF0007734002010B50B4B1B78022B02D008240E
:104F0000204610BDFFF72AFC0446042807D00928D4
:104F100005D00028F4D07846F7F720FEF0E701F03E
:104F2000D5FCEDE77734002010B50446054B1B781F
:104F3000022B03D12046FFF725FC10BD7846F7F77A
:104F40000DFEF7E77734002010B584B0284B1B78AE
:104F5000012B17D0274B1B6813F4004F03D0264BAF
:104F60001B68012B03DC0824204604B010BD234B32
:104F7000D3F80435224A0092992222490220FCF7F4
:104F800087FFF0E71A4B02221A7003A90420FFF7EB
:104F9000B1FF0446C0B1174B1B6813F4004F03D098
:104FA000154B1B68002B03DC114B01221A70DBE749
:104FB000124BD3F804350190134A0092A3221149F1
:104FC0000120FCF765FFEFE7039B81225A70039BEA
:104FD00002229A704FF08043D3F8003403F00803A4
:104FE000039AD3700398FE230371FFF79DFFBBE77D
:104FF00077340020741F0020701F00200010014033
:105000005C730300537303007073030008B50A4B0D
:105010001B781BB9094B1B78022B00D008BD064B2F
:1050200001221A7000210648FBF77EFD0028F5D00A
:10503000014B00221A70F1E776340020773400200B
:105040002151020011280ED811282CD8DFE800F0D9
:10505000092D2D11131517192D1B2D1D1F2123256A
:1050600027290020704743F2010398421FD18E2068
:105070007047812070478E2070478E2070478E20A9
:1050800070478520704784207047872070478420B0
:10509000704793207047812070478E20704787208B
:1050A000704786207047802070478320704780209B
:1050B00070470000014B1878704700BF773400201C
:1050C000F0B583B006460D461C46174602B11BB923
:1050D00047B17846F7F742FD104B1B78022B04D0FE
:1050E00003B0F0BD002CF7D0F3E7E01C01A980B2BB
:1050F000FFF700FF0028F3D1019B84225A70019B27
:105100009E70019BDD702FB1224639460198043014
:1051100011F0AFF80198FFF707FFE1E777340020BF
:1051200000B5C3B0204B00221A7026E00133082BD3
:1051300013D81E4A12F833109DF809209142F5D871
:105140001A4901EBC30149788A42EFD8174A02EBAA
:10515000C3035B6802A898470FE0154B1B6813F464
:10516000004F03D0134B1B68012B0CDC00231A46A5
:1051700082219DF80900FFF7A3FF02A8FFF7E0FBDB
:1051800078B10023D3E70C4BD3F804359DF8092000
:1051900001920A4A0092812209490220FCF778FE16
:1051A000E4E743B05DF804FB76340020C0730300ED
:1051B000741F0020701F002000100140A87303001E
:1051C000537303000023012B0ADC06494FF49A7243
:1051D00002FB0312824201D00133F4E7D8B27047D8
:1051E000FF20704728380020F0B583B004460378CC
:1051F0000C2B11D8DFE813F00D004100530089009B
:105200009D0049016301F40010006700B0000D012A
:105210007E01B74B1B780BB903B0F0BD01A91A2072
:10522000FFF768FE0028F7D1019BC0225A70019B4E
:10523000224652F8045F50689168D268C3F8025061
:10524000C3F80600C3F80A10C3F80E20E26992F909
:105250000D209A74227DDA74E269927BC2F34602D1
:105260001A75E26952F80F1FC3F815109288A3F857
:1052700019200198FFF758FECEE701A90220FFF799
:1052800039FE0028C8D1019BC1225A706068FFF71F
:1052900099FF019B98700198FFF746FEBCE701A9B2
:1052A0000320FFF727FE0028B6D1019BC2225A70C7
:1052B000019D6068FFF786FFA870237AEB70019864
:1052C000FFF732FEA8E701A90B20FFF713FE002825
:1052D000A2D1019BC3225A70019D6068FFF772FF43
:1052E000A870237AEB70E37A2B71237B6B71637B5D
:1052F000AB71E389A5F80730237C6B72B4F81130E9
:105300006B810198FFF710FE86E701A90320FFF7E4
:10531000F1FD002880D1019BC4225A70019D606874
:10532000FFF750FFA870237AEB700198FFF7FCFDA0
:1053300072E701A90220FFF7DDFD00287FF46CAFC2
:10534000019BCA225A706068FFF73CFF019B98706E
:105350000198FFF7E9FD5FE701A92C20FFF7CAFDDF
:1053600000287FF459AF019BC5225A70019D6068E7
:10537000FFF728FFA870E368D3F81230C5F80330B0
:10538000E368DB8AA5F80930E3681B8AA5F80730D3
:10539000E3681B7EC3F30003EB72E3681B7EC3F379
:1053A00040032B73A368186859689A68DB68C5F8CE
:1053B0000D00C5F81110C5F81520C5F81930E368BF
:1053C000186859689A68DB68C5F81D00C5F821108F
:1053D000C5F82520C5F829300198FFF7A5FD1BE782
:1053E00001A90520FFF786FD00287FF415AF019B7A
:1053F000C6225A70019D6068FFF7E4FEA870012381
:10540000EB7000232B7110236B710198FFF78CFD5B
:1054100002E701A96220FFF76DFD00287FF4FCAED2
:10542000019BC7225A70019D6068FFF7CBFEA870F0
:10543000A368EA1C03F1400C1F685E689868D9688D
:10544000176056609060D160103310326345F3D11D
:10545000E3681C6858689968DA68C5F84340C5F87D
:105460004700C5F84B10C5F84F201C695869996969
:10547000DA69C5F85340C5F85700C5F85B10C5F8A0
:105480005F200198FFF750FDC6E601A91320FFF742
:1054900031FD00287FF4C0AE019BC8225A70019DE7
:1054A0006068FFF78FFEA870237AEB70627AE1687C
:1054B000281D10F0DEFE0198FFF736FDACE601A9CD
:1054C0000520FFF717FD00287FF4A6AE019BC6223A
:1054D0005A70019D6068FFF775FEA8700323EB709A
:1054E000237A2B71637A6B710198FFF71DFD93E6A8
:1054F000DC3A002001A90320FFF7FCFC00287FF420
:105500008BAE019BC9225A70019D6068FFF75AFE5D
:10551000A870237AEB700198FFF706FD7CE600BFC8
:1055200010B582B01D4B1B6813F4004F03D01C4B09
:105530001B68032B06DC1B491B480BF0CBF968B931
:10554000002413E0194BD3F80435194A009240F2B5
:105550000B1218490420FCF79BFCECE77846F7F7A0
:10556000FDFAEDE77846F7F7F9FA0134012C11D886
:10557000114B4FF4E47000FB04300CF05BFF01466C
:105580000E4B4FF49A7000FB04300BF08DF900289D
:10559000EBD0E7E7002002B010BD00BF741F002071
:1055A000701F0020083800209C3A002000100140A5
:1055B0008C740300737403007834002028380020B2
:1055C000F0B58BB004464078A0F16103092B00F2DE
:1055D0000A81DFE813F00A00250039008100080184
:1055E0009B00B400CF00E6000A018D4B1B782BB165
:1055F00000231A468321FFF763FDF4E0884B012264
:105600001A7088480BF0C4FA30B900231A461946BC
:105610006078FFF755FDE6E07846F7F79FFAF4E784
:105620007F4B1B7823B91A468321FFF749FDDAE047
:1056300000257B4B1D700BF0B3FA2B462A462946FA
:105640006078FFF73DFDCEE0A378012B09D90B214F
:10565000A3788DF80C30012303AA6320FFF78CF99F
:10566000C1E003AD234653F8130F59689A68DB680D
:105670000FC5B4F82330ADF81C30D4F82530CDF880
:105680001E30B4F82930ADF8223094F82B3094F85D
:105690002C2003F0010362F341038DF82430A0783D
:1056A000604B0093604B614A6149624D4FF49A76BA
:1056B00006FB00500BF0CDF801460028C8D1A078B9
:1056C0000123009303AB94F82D20E11C06FB00504E
:1056D0000BF0A6F90146BBE7524B0093524B534ADD
:1056E000534954480BF0B5F848B16478FFF7AAFC69
:1056F000014600231A462046FFF7E2FC73E001232F
:10570000002211464B480BF001F9EEE7A578012D78
:1057100009D90B21A3788DF80C30012303AA662048
:10572000FFF72AF95FE063792279E17841484FF485
:105730009A7606FB05000BF0A2F90146EAE7A3788A
:10574000012B09D90B21A3788DF80C30012303AA72
:105750006720FFF711F946E0214611F8032B023AC2
:10576000D2B234484FF49A7505FB03000BF090F960
:105770000146E8E7A378012B09D90B21A3788DF81E
:105780000C30012303AA6820FFF7F6F82BE0E11C98
:10579000284A4FF49A7000FB03200BF0EFF9014602
:1057A000ECE7224D264656F8020F7168B268F3689E
:1057B0000FC530697169B269F3690FC504F122053B
:1057C0001B4F04F1620C3E4628686968AA68EB68C2
:1057D0000FC6103537466545F5D100231A461946E0
:1057E0006078FFF76DFC0BB0F0BDA3780E48037036
:1057F0000021012343708170E378C3702379037122
:10580000237A0372B4F80930A0F809306379437140
:10581000E388C3800B460A466078FFF751FCE2E755
:10582000DC3A0020E9510200903A002008380020BC
:105830009C3A00202838002010B582B00446037836
:10584000073B062B0AD8DFE803F0516F7F99B704B6
:105850002B0001A91620FFF74DFB08B102B010BDC7
:10586000019BA5225A702279019B9A70019A2346C6
:1058700053F8050F5968C2F80300C2F807101B89D6
:10588000A2F80B30019854F80F2F6368C0F80D2070
:10589000C0F811302389A0F81530FFF745FBDDE78C
:1058A00001A91620FFF726FB0028D7D1019BA622CD
:1058B0005A702279019B9A70019A234653F8050F7A
:1058C0005968C2F80300C2F807101B89A2F80B3010
:1058D000019854F80F2F6368C0F80D20C0F81130FC
:1058E0002389A0F81530FFF71FFBB7E701A90D20AA
:1058F000FFF700FB0028B1D1019BA0225A7022794A
:10590000019B9A70019A234653F8050F5968C2F813
:105910000300C2F807101B89A2F80B300198E37B43
:105920004373FFF701FB99E701A90220FFF7E2FAB1
:10593000002893D1019BA1225A702279019B9A7071
:105940000198FFF7F1FA89E701A90D20FFF7D2FAD4
:10595000002883D1019BA2225A702279019B9A7060
:105960006279019BDA70019854F8062F63684260EF
:10597000836023898381FFF7D7FA6FE701A90E209F
:10598000FFF7B8FA00287FF469AF019BA3225A7091
:105990002279019B9A706279019BDA700198234603
:1059A00053F8061F5A68416082601B898381237CFB
:1059B0008373FFF7B9FA51E701A91520FFF79AFAA7
:1059C00000287FF44BAF019BA4225A702279019BDF
:1059D0009A70019A234653F8050F5968C2F80300DC
:1059E000C2F807101B89A2F80B3023690198C0F890
:1059F0000D306369C0F81130237E4375FFF794FAC8
:105A00002CE7000008B50348034B0360FAF714F8CD
:105A100008BD00BFE03A00203958020010B58AB036
:105A200004464078A0F1D003062B04D822787049B0
:105A3000CB5C9A420AD1A0F1D003062B00F2C980B8
:105A4000DFE803F00B1727354170860000231A4664
:105A50008421FFF735FB0AB010BDF6F7CDFF64785F
:105A6000FFF7F0FA014600231A462046FFF728FB0D
:105A7000F1E7D4F80D20E11CA078F6F7BDFF6478BB
:105A8000FFF7E0FA014600231A462046FFF718FB0D
:105A9000E1E7E11CA078F6F7AFFF6478FFF7D2FAF0
:105AA000014600231A462046FFF70AFBD3E7F6F724
:105AB000A3FF6478FFF7C6FA014600231A46204682
:105AC000FFF7FEFAC7E76946A078F6F795FFF8B941
:105AD0009DF800308DF81430DDF80120DDF8053038
:105AE000CDF81520CDF81930BDF80930ADF81D30CE
:105AF0009DF80B308DF81F30039B0893049B09938E
:105B000014230DEB030200216078FFF7D9FAA2E716
:105B10006478FFF797FA014600231A462046FFF7FC
:105B2000CFFA98E72378022B05D000231A46842168
:105B3000FFF7C6FA8FE7A078F6F75EFF6478FFF705
:105B400081FA014600231A462046FFF7B9FA82E798
:105B50002378012B05D000231A468421FFF7B0FAE1
:105B600079E70023CDF80230CDF80630ADF80A30E1
:105B70006846F6F741FF10BB9DF800308DF81430F1
:105B80009DF801308DF81530DDF80220DDF8063083
:105B9000CDF81620CDF81A30BDF80A30ADF81E3019
:105BA0009DF80C308DF820309DF80D308DF82130A7
:105BB0000E2305AA00216078FFF782FA4BE764788C
:105BC000FFF740FA014600231A462046FFF778FA0D
:105BD00041E700F13003DBB20F2B02D97846F6F72C
:105BE000BDFF00231A4682216078FFF769FA32E789
:105BF000B074030010B582B0019148B91446BDF8E5
:105C000004302BB9BDF80630032B03D0042B13D07E
:105C100002B010BD14490520FFF76CF90028F7D138
:105C2000114B1A68DA2151701A682168C2F8021003
:105C30001868FFF779F9EBE70B490820FFF75AF9E5
:105C40000028E5D1084B1A68D92151701A682168DB
:105C5000C2F80210186823798371B4F80530A0F8EF
:105C60000730FFF761F9D3E7F83A002070B582B04A
:105C700004460378052B5BD8DFE803F003935568EF
:105C80005A7B0689EB2E00D9EB2606F114004E490B
:105C900080B2FFF72FF900284AD14B4B1D682389AA
:105CA000A5F81330237D012B25D1D0236B70E38A17
:105CB000AB80E3896B80206A05F059FAE880E069DF
:105CC00005F03EFA288194F82430AB72A36A9B7BDE
:105CD000C3F34603EB72A36A53F80F2FEA609B8865
:105CE0002B82A36A93F90D30AB74AEB9364B1868AA
:105CF000FFF71AF91CE0D1236B700DF1060104F1D6
:105D0000140005F0B1F918B9BDF80630AB80D0E742
:105D10007846F6F723FFF7E73246616805F115008C
:105D200010F0A7FAE2E728490520FFF7E3F808B1E9
:105D300002B070BD244B1A68D32151701A68E16813
:105D4000C2F802101868FFF7EFF8F1E71E490420C7
:105D5000FFF7D0F80028EBD11B4B1A68D421517003
:105D60001A68A18851801868237B0371FFF7DCF85B
:105D7000DEE715490720FFF7BDF80028D8D1124B00
:105D80001A68D82151701A68217991701A6861795E
:105D9000D1701868E38883802389C380FFF7C4F833
:105DA000C6E709490520FFF7A5F80028C0D1064B32
:105DB0001A68D22151701A686168C2F80210186816
:105DC000FFF7B2F8B4E700BFFC3A002010B58AB084
:105DD00004460023ADF820300423ADF8223006A994
:105DE0000898FDF741FFF0B90023ADF824300323F4
:105DF000ADF8263004A90998FDF736FF0146069B49
:105E000001939DF81C308DF80830BDF81D30ADF8B9
:105E10000930049BCDF80B300B2301AA6078FEF704
:105E2000ABFD0AB010BD014600231A466078FEF7AC
:105E3000A3FDF6E700B583B00823ADF804300223D4
:105E400001AA00214078FEF797FD03B05DF804FB3E
:105E500000B583B02023ADF80430022301AA00214D
:105E60004078FEF789FD03B05DF804FB00B583B010
:105E70000A23ADF80430022301AA00214078FEF77E
:105E80007BFD03B05DF804FB00B583B00823ADF8DB
:105E90000430022301AA00214078FEF76DFD03B013
:105EA0005DF804FB00B583B00823ADF8043002238D
:105EB00001AA00214078FEF75FFD03B05DF804FB06
:105EC00010B504468179D0F80920003918BF0121A6
:105ED000D0F80200F9F7EEF9014600231A4660787F
:105EE000FEF74AFD10BD10B5044640880FF058F982
:105EF000014600231A466078FEF73EFD10BD10B53E
:105F0000044600F041FD00231A4619466078FFF769
:105F1000D7F810BD10B582B0044601A804F0BCFE4D
:105F2000BDF80430ADF80030BDF80630ADF80230F1
:105F300004236A4600216078FEF71EFD02B010BD02
:105F400010B58CB004462422002103A810F0BAF941
:105F5000F9F780FD029003A9E08804F091FF014663
:105F600030B1042302AA6078FEF706FD0CB010BD24
:105F700001A804F091FEA288BDF804309A4235D3FE
:105F8000BDF806100B449A4201DB1021E9E709AA8B
:105F900061884FF6FF7005F08FFE01460028E0D1C2
:105FA000A388ADF81430237A8DF81630637A003B5D
:105FB00018BF01238DF81730A37A8DF81830237895
:105FC0000B2B0ED904F10C03079323780B3BADF890
:105FD0002030029B0B93002103A8F9F729FD01460D
:105FE000BFE700230793ADF82030F2E71021B8E7B0
:105FF00070B5ADF53E7D05467E230093694601A848
:1060000004F0EEFF0646009C74B1620001A97FA86F
:1060100010F02FF963009BB27FAA31466878FEF733
:10602000ABFC0DF53E7D70BD00231A460146687835
:10603000FEF7A2FCF5E730B589B0044606A9408812
:1060400004F01EFF00230093019302930393049333
:10605000ADF81430054638B100236A462946607809
:10606000FEF78AFC09B030BD6388ADF800309DF8BA
:1060700018308DF8023006A805F09AFF8DF803005D
:10608000BDF81A30ADF80430079B6BB11868596839
:106090009A68DB68CDF80600CDF80A10CDF80E201E
:1060A000CDF812301623D8E70623D6E710B582B014
:1060B0000446408804F050FE01466388ADF8043081
:1060C000022301AA6078FEF757FC02B010BD10B59C
:1060D00082B004460DF10601023004F037FE01469D
:1060E000BDF80630ADF80430022301AA6078FEF74F
:1060F00043FC02B010BD10B582B004460DF106019C
:10610000408804F0D7FD0146BDF80630ADF80430F4
:10611000022301AA6078FEF72FFC02B010BD10B573
:1061200082B00446408804F0F5FE01466388ADF86D
:106130000430022301AA6078FEF71EFC02B010BDF5
:1061400010B582B004460DF10601023004F04DFE98
:106150000146BDF80630ADF80430022301AA60788C
:10616000FEF70AFC02B010BD10B582B004460DF176
:106170000601408804F034FE0146BDF80630ADF853
:106180000430022301AA6078FEF7F6FB02B010BDCE
:1061900010B582B004464388ADF804308388ADF86A
:1061A000063001A804F044FD014600231A46607839
:1061B000FEF7E2FB02B010BD10B582B00446408885
:1061C00005F090FB01466388ADF80430022301AA74
:1061D0006078FEF7D1FB02B010BD10B582B0044666
:1061E0000DF10203821D8188408805F0EFFA014617
:1061F000BDF80230ADF80430022301AA6078FEF742
:10620000BBFB02B010BD70B5ADF53E7D05467D23EC
:10621000019301AA02A9408805F02CFD0646019CC5
:1062200044B900231A4601466878FEF7A5FB0DF530
:106230003E7D70BD6B88ADF8FC31620002A90DF5A2
:10624000FF7010F016F8631C5B009BB27FAA31460A
:106250006878FEF791FBEAE710B582B00446408803
:1062600005F062FC01466388ADF80430022301AA00
:106270006078FEF781FB02B010BD10B582B0044615
:10628000011D408805F0E4FB01466388ADF8043049
:10629000022301AA6078FEF76FFB02B010BD10B5B3
:1062A00082B004460DF10203821D8188408805F00A
:1062B0003FFB0146BDF80230ADF80430022301AACD
:1062C0006078FEF759FB02B010BD70B5ADF53E7DAC
:1062D00005467E230093694601A805F069FA064643
:1062E000009C44B900231A4601466878FEF744FB37
:1062F0000DF53E7D70BD620001A97FA80FF0B9FFCA
:1063000063009BB27FAA31466878FEF735FBEFE762
:1063100010B582B00446408805F022FC014663882F
:10632000ADF80430022301AA6078FEF725FB02B025
:1063300010BD10B582B00446011D408805F08AF8F2
:1063400001466388ADF80430022301AA6078FEF7A5
:1063500013FB02B010BD10B582B004460DF102026D
:10636000011D408804F0ACFF0146BDF80230ADF8D5
:106370000430022301AA6078FEF7FEFA02B010BDD5
:1063800010B54478F9F73CFB014600231A46204635
:10639000FEF7F2FA10BD10B54478F9F7DFFA0146BE
:1063A00000231A462046FEF7E7FA10BD08B5034859
:1063B000034B0360F9F740FB08BD00BFEC3A002037
:1063C0006D5C020038B5044643787033DBB22F2B86
:1063D0001FD86078AF2820D8A0F19005174B13F88C
:1063E000353098421FD1154B03EBC5035B782178FC
:1063F0008B4207D20133114A02EBC5029278134453
:10640000994214DD00231A4684216078FEF758FE75
:1064100038BD7846F6F7A2FBDBE700231A46822157
:10642000FEF74EFEF4E77846F6F798FBDBE7034B02
:1064300003EBC5056B6820469847E9E7C074030085
:1064400038B50546002400E00134012C17D804EBD0
:1064500044030D4A02EB83035B6893B104EB4401F0
:106460000422094B03EB810128460FF0CFFE0028E0
:10647000EAD104EB4404044800EB840000E000206F
:1064800038BD0020FCE700BF003B002030B5C1B0A4
:106490000446851C3FA9408802F04EFD68B93FA81C
:1064A000FFF7CEFF00B300228DF800208368694615
:1064B000284698479DF8003053B96478FEF7C2FD2E
:1064C000014600231A462046FEF7FAFD41B030BDD2
:1064D0006478FEF7B7FD01469DF8003001336A4647
:1064E0002046FEF7EDFDF1E70520E6E730B583B085
:1064F0000446851C2846FFF7A3FF0023ADF80430AF
:1065000080B143680DF10201284698470146BDF865
:106510000230ADF80430022301AA6078FEF72CFAAD
:1065200003B030BD0521F6E730B5C1B00446FA220C
:10653000002101A80FF0C6FE00230DE001A901EB28
:10654000820103EB4305134850F82500C1F802000F
:106550000132ADF804200133012B0CD803EB4302C8
:106560000C4901EB8202526892B1BDF804203D2A29
:10657000E4D90C2100E00021BDF804309B009BB25F
:1065800002339BB201AA6078FEF7F6F941B030BD44
:106590000021F1E7003B002010B504464378FF2BB3
:1065A00005D0032204492046FEF7FEF910BD7846C7
:1065B000F6F7D4FAF5E700BFC075030008B500216F
:1065C000034B19600B460A464078FEF779FD08BD7B
:1065D000543C002000B583B0064B1B680193042394
:1065E0000DEB030200214078FEF76AFD03B05DF871
:1065F00004FB00BF543C0020F0B583B0074686780A
:1066000036B935468DF8006000248DF802401BE055
:1066100000231A4685214078FEF752FD42E0784675
:10662000F6F79CFA204A4FF49E7303FB052323449C
:1066300093F87820253A012303FA02F29DF80230FC
:1066400013438DF802300134174A4FF49E7303FB55
:10665000052393F87B30A3420CD9134A4FF49E7361
:1066600003FB0523234493F87830253BDBB2022B50
:10667000D8D9D4E713464FF49E7202FB0636736FE7
:1066800003F5FA73094AA2FB03239B09CDF80330F3
:1066900096F82C308DF8013007236A46002178786F
:1066A000FEF70EFD03B0F0BD183B0020D34D621085
:1066B00008B500231A4682214078FEF701FD08BD87
:1066C00000B583B00223ADF8043001AA0021407860
:1066D000FEF7F6FC03B05DF804FB08B500231A468C
:1066E00082214078FEF7ECFC08BD000030B583B095
:1066F000044683785BB107206478FEF7A3FC01466B
:1067000000231A462046FEF7DBFC03B030BD154DD2
:106710004FF49E7202FB03531D1DD0F8051028464E
:1067200005F08CFF002300938DF8043000E0013366
:10673000022B10D822791A4112F0010FF7D09DF8E0
:106740000320511C8DF8031003F1250102A8024417
:1067500002F8081CEBE76946284605F018FF002000
:10676000CAE700BF183B002070B504468078B8B96E
:106770004FF49E7303FB00F30F4AD35C012B01D04F
:1067800008200EE016464FF49E7505FB00200430ED
:1067900005F0A1FFA37805FB03F50020705500E08C
:1067A00007206478FEF74EFC014600231A46204677
:1067B000FEF786FC70BD00BF183B0020F8B504460C
:1067C000807850B107206478FEF73CFC0146002336
:1067D0001A462046FEF774FCF8BD2578023D124BA0
:1067E0004FF49E7202FB00302946043005F03BFE58
:1067F0000646B8B1FF2303712A46E11C11300FF0A1
:1068000038FDA078084F4FF49E7505FB00703146A7
:10681000043005F065FEA37805FB03F501237B55E5
:106820000020D0E70420CEE7183B002010B5044636
:106830000120F9F767F900231A468E216078FEF7E8
:106840003FFC10BD10B582B0044601A90078FEF7E8
:1068500051FB08B102B010BD019B82225A70019811
:1068600010F8022B013AA11C0FF003FD0198FEF76E
:106870005BFBEFE738B5002404B138BD09494FF49C
:106880009E7303FB04F3CD18043503F1A0029C238F
:106890000A440021284605F057FF284605F0AAFDC6
:1068A0000134E9E7183B002010B5044643781F2B5C
:1068B00005D80B2204492046FEF776F810BD78462D
:1068C000F6F74CF9F5E700BFD8750300044B1B68D9
:1068D000B3F1FF3F02D00133014A1360704700BF9C
:1068E000543C002038B50446FEF7E4FB90B9FEF7AF
:1068F00017FE054678B9FEF7EDFA054658B9FFF7D9
:10690000B9FFFFF753FDFFF77DF824B1204600F0F3
:1069100009F800E00825284638BD08B5FEF714FB45
:1069200008BD0000014B1860704700BF583C0020B4
:1069300010B504460A4B1B6853B110F8021B01390D
:10694000984700231A4619466078FEF7B9FB10BD38
:1069500000231A468E214078FEF7B2FBF7E700BF0E
:10696000583C00200378142B00D07047C3880F2BAD
:10697000FBD8024B01221A70F7E700BFB43C00209D
:1069800008B5F8F7EBFF08BD08B5F9F7B8FC01F05A
:10699000EEFC04F0F7F8F8F745FAFCF747F808BD05
:1069A00008B505F02BFB08BD70B582B0002841D0BA
:1069B0000E460446F8F762FF054610B1284602B0BD
:1069C00070BD04F021F901F0DDFC20690EF0B8FB88
:1069D00005460028F2D1237F0193A36900936369E0
:1069E0004FF6FF72002114480EF022FF05460028E2
:1069F000E4D1236A03B19847104C2046F9F71CF8FC
:106A0000FDF7B6F92046F9F71BF804F0A5F804469F
:106A100001F0CEFA0B2C04D00B2802D0084B1B78C7
:106A200013B1FFF7B1FF0B25FFF7BAFF002EC5D05A
:106A30003070C3E70E25C1E75C3C00208C1F0020AE
:106A4000B43C002038B50546837803F00303032BDC
:106A500021D8DFE803F0020C131981788B081A4A59
:106A600011681944A960194B1B6800241AE0837847
:106A700003F0FC0101EB93014B00F0E783789B08E6
:106A8000642101FB03F3EAE783789B0841F270710C
:106A900001FB03F3E3E77846F6F760F80023DEE74F
:106AA0001C46DB681BB19A688A1A002AF8DA1CB106
:106AB00033B1E560EB6038BDEB60044B1D60FAE775
:106AC000E5600023EB60F6E7D03C0020D83C0020D6
:106AD00010B5714B19688B7803F003036F4A127875
:106AE000934240F3B5808C686D4B1B68E31A6D4C84
:106AF00004FB03F4032A26D8DFE802F0022A21234C
:106B0000684BB4FBF3F4644B1B689B7803F00303FE
:106B1000022B36D0032B57D0012B1BD00023184655
:106B2000002B40F0AC80F9F76DFA04465B4B1B7804
:106B3000032B00F28680DFE803F07D8980825A4BC8
:106B4000DFE75A4BDDE77846F6F708F80023D8E789
:106B5000574BD6E703F1CC33A3FB0423DB0803EB4D
:106B60008303B4EB430F02D000231846D8E7F9F7AC
:106B700049FA00F5742000F510700123474A13709C
:106B8000CEE7464B1A783AB94A4BA3FB04135B098C
:106B9000642101FB13436BB1012A02D00023184684
:106BA000BEE7454BA3FB0423DB0803EB8303B4EBF5
:106BB000430F3CD1F9F726FA03463B481844374BBC
:106BC00002221A700123ABE7344B1A7842B93B4BCF
:106BD000A3FB0413DB0941F2707101FB134383B182
:106BE000012A04D0022A16D00023184698E7344B15
:106BF000A3FB04139B094FF4167101FB1343002BF5
:106C0000F0D1F9F7FFF9034628481844234B032233
:106C10001A70012384E72B4BA3FB04235B09C3EB0E
:106C20000313B4EB830FECD00023184678E700235E
:106C3000184675E71B48204421E01B48FBE71B482A
:106C4000F9E77846F5F78AFF0020F4E71848F2E7FD
:106C5000F9F7D8F90446104B1B689B7803F003033F
:106C6000032B11D8DFE803F002150C0E0D48204469
:106C7000094B1B689B78C3F30103084A137010BDCE
:106C80000948F4E70948F2E77846F5F767FF00207E
:106C9000EDE70748EBE700BFD83C0020D53C0020DB
:106CA000D03C0020A0860100809698000046C323B7
:106CB00040420F001F85EB51CDCCCCCCF1197605AD
:106CC000B5814E1B8988888838B5294B1B7873B9E4
:106CD000284B1B68002B43D0FFF7FAFE0146244BDC
:106CE0001B78002B34D02448F9F758F93BE0224BAD
:106CF0005D68F9F787F90446204B1B78032B16D8FB
:106D0000DFE803F0021A11131D4B601B18441B4BE4
:106D10001B789BB94CF2503398420FD9194A13682B
:106D200001331360D4E7184BEFE7184BEDE77846D3
:106D3000F5F714FF0023E8E7154BE6E74009154B8C
:106D4000A3FB00300F4A136803EBD0101060BFE7BD
:106D5000074B01221A7008484160F9F7D7F802E0A2
:106D6000034B1B7803B938BD0348F9F7FFF8FAE77E
:106D7000D43C0020D83C0020B83C0020D53C00206A
:106D8000A0860100D03C0020809698000046C323D6
:106D900040420F00C55A7C0A30B583B009E07846FE
:106DA000F5F7DCFE63680199284698472046FFF70F
:106DB00049FE0F4B1C68B4B1A3680E4A1268934297
:106DC00004D00C4A12689B1A002B0CDA2588E26862
:106DD000074B1A600023019301A9284602F03EF9EF
:106DE0000028DFD0DBE7FFF76FFF03B030BD00BF47
:106DF000D83C0020D03C002008B5134B1B78032B57
:106E00001ED8DFE803F0020C1116104A1368013394
:106E100013600F4B00221A70FFF7BEFF08BD0B4A2C
:106E200013680A331360F4E7084A13686433136085
:106E3000EFE7064A136803F5BB5310331360E8E726
:106E40007846F5F78BFEE4E7D53C0020D03C0020E7
:106E5000D43C002010B50446FFF7F4FD034B1B683B
:106E6000A34200D010BDFFF72FFFFBE7D83C002066
:106E7000074A002313605360D360136153610549CF
:106E80009160054A1360054A1360054A1370704704
:106E9000B83C0020F96D0200D03C0020D83C002016
:106EA000D43C002008B5054B1B7813B9FFF7E0FF71
:106EB00008BD0348F9F75AF8F8E700BFD43C0020B2
:106EC000B83C002070B50E461546044650B1F9F79F
:106ED0003FFE144B1B68002043B1A34206D0184666
:106EE000DB68F9E77846F5F739FEF0E7A17866F355
:106EF000010165F38701A17013B138B1DA68C2608E
:106F000045B903B150B1F9F767FE70BDD968054ABC
:106F10001160F5E72046FFF79DFFF4E7FFF7D4FE89
:106F2000F1E700BFD83C002000234FF6FF70012B93
:106F300022D830B404E0184601339BB2012B19D893
:106F400003EBC30291000D4A0A4492F83920002A4B
:106F5000F2D04FF6FF729042EDD0084A1144096B0F
:106F600000EBC005AC002244126B8A1A002AE3DA57
:106F70001846E1E730BC7047704700BFDC3C00209A
:106F800070B5044600EBC0021A4B03EB820393F882
:106F9000393033B3174BB3F8603033B3154A04EBD1
:106FA000C40302EB8303002183F83910B2F8603088
:106FB000013B9BB2A2F8603023B913464FF6FF7233
:106FC000A3F862200B4DE60004EBC40305EB83033A
:106FD000986AFDF78EFA344405EB84050023AB6212
:106FE00070BD7846F5F7BAFDD4E77846F5F7B6FDFB
:106FF000D4E700BFDC3C0020F8B505464E4BB3F8A3
:1070000060301BB105F57A77002421E07846F5F76A
:10701000A5FDF7E72046FFF7B3FF17E0002861D191
:1070200006EBC602444B03EB820292F83830013B78
:10703000DBB282F83830002B58D03F4A06EBC6034B
:1070400002EB8303596B1A6B114419630134A4B228
:10705000012C4FD8264604EBC403374A02EB8303C6
:1070600093F83930002BF1D004EBC40302EB830317
:107070001B6BDB1B002BE9DA104604EBC401890013
:10708000183104EBC40200EB8202938D926A014432
:10709000204601F04DF91028C0D801A353F820F084
:1070A000217002001D7002001D7002001D700200A0
:1070B00021700200157002001D70020015700200A0
:1070C00021700200157002001D7002001D70020088
:1070D0001D7002001D7002001D7002002170020070
:1070E000157002007846F5F739FD99E72046FFF75D
:1070F00047FFABE7FFF718FF0F4BA3F86200B3F8A9
:107100006030A3B101280CD80B4BB3F8622002EB1E
:10711000C20203EB82031B6B5A1B06D4064BDA60D8
:10712000F8BD7846F5F71AFDEEE7EA1AF6E7024BE6
:107130000022DA60F4E700BFDC3C00202DE9F843D0
:107140000446884616469946F8F75CFF8646154F72
:1071500004EBC40507EB850505F1180C96E80F0054
:107160008CE80F00C5F82890BDF82030AB8598F862
:107170000030C3F3020385F8383098F80000C308E4
:107180004CF2503003FB0000686370442863012315
:1071900085F83930B7F860300133A7F86030BDE8C2
:1071A000F88300BFDC3C002010B50446FFF7BCFEAE
:1071B0000E4BB3F86230834211D00C4BA3F862003F
:1071C0004FF6FF7398420DD00848B0F8623003EBD9
:1071D000C30300EB8303196BF8F7E0FE10BDA34275
:1071E000FCD1EAE77846F5F7B9FCEDE7DC3C002096
:1071F00010B5064C6222002120460FF063F8044BC4
:10720000A3604FF6FF73A4F8623010BDDC3C002091
:10721000F96F02002DE9F04182B004460D46164692
:107220001F46BDF8208001281FD815B32EB32B7838
:1072300013F0070F25D047B3B8F1000F29D004EBA6
:10724000C403184A02EB830393F839302BBBCDF803
:1072500000803B46324629462046FFF76FFF204616
:10726000FFF7A2FF02B0BDE8F0817846F5F776FCA3
:10727000DBE77846F5F772FCD8E77846F5F76EFC61
:10728000D5E77846F5F76AFCD5E77846F5F766FC6A
:10729000D2E77846F5F762FCD1E72046FFF770FEAB
:1072A000D5E700BFDC3C00204FF6FF7399420CD0BD
:1072B0000C4B00EB400203EB4202D27800EB4000A3
:1072C00003EB4000531CC3707047064B00EB4002B9
:1072D00003EB4202927800EB400003EB4000531CAA
:1072E00083707047843D002030B482B001911B4B05
:1072F00000EB400103EB4101897800EB400403EB14
:107300004403DB78D94201D0002303E0002021E0D0
:1073100001339BB2012B1CD8C3EBC301104C04EB0F
:10732000C10189898142F3D1C3EBC30104EBC101DF
:107330004C88BDF806108C42EAD1C3EBC30508495E
:1073400031F83540BDF804108C42E1D113800120A2
:1073500000E0002002B030BC704700BF843D002038
:107360009C3D002082B000230093027802F0C0030D
:10737000802B1ED012D80BB1402B05D1ADF80020C8
:107380004FF6FF73ADF80230009B00209AB262F313
:107390000F001B0C63F31F4002B07047C02BF3D1EA
:1073A000ADF800204378827843EA0223ADF802303A
:1073B000EAE7437843EA0222ADF800204FF6FF7374
:1073C000ADF80230E0E782B001904FF6FF72B2EB09
:1073D000104F08D0030CBDF804200A704B701B0A34
:1073E0008B7002B07047BDF8043013F47F4F03D0A8
:1073F0001A0A0A704B70F4E70B70F2E782B0019042
:107400004FF6FF73B3EB104F18D1BDF8040010F422
:107410007F4F07D000F44040B0F5004F14BF00206C
:10742000012014E020F07F039BB22BB97F2801D00C
:1074300001200CE000200AE0002008E0BDF8040074
:1074400020F03F0080B2C02814BF0020012002B00D
:10745000704770B506460D460024AC4207D256F878
:107460003400FFF7CBFF034610B10134F5E70123E9
:10747000184670BD30B482B00191002300E00133A2
:10748000818D994210D9816A01EBC30531F83340EF
:10749000BDF804108C42F2D16C88BDF806108C4205
:1074A000EDD11360012000E0002002B030BC704735
:1074B000C389012B01D90020704703EB4303094A1C
:1074C00002EB830304334A0953F8223001F01F0111
:1074D00023FA01F111F0010F01D0012070470020C3
:1074E000704700BF143E0020000CA0F5405080B251
:1074F000012826D8144B1B7813F0040F1DD0002050
:10750000704751F82320D44300EB4002D5180F4AAE
:1075100002EB850254600133012BF2D90B4A00EBD8
:10752000400312F8233000EB400003F0F90302F8A7
:107530002030002002B030BC704730B482B000234D
:10754000EAE70520704700BF103E0020143E0020EF
:1075500082B0000CB0F5805F1AD1114B1B7813F08C
:10756000040F18D1A0F5805080B20A8800EB4001CA
:107570000C4B33F811309A420FD10A4B03EB410206
:10758000527903EB410002F0F9034371002000E05F
:10759000052002B070470020FBE70B20F9E700BF91
:1075A000103E0020843D002082B0000CB0F5804FDA
:1075B00005D10A78034B1A70002002B070470520ED
:1075C000FBE700BF981F002010B582B001900C4669
:1075D000000C012806D1012363800223A3802380AD
:1075E00002B010BD7846F5F7B9FAF4E710B582B0ED
:1075F00001900C46000C01280FD16388012B10D19B
:10760000A388022B10D12388022B0FD1084A1378AC
:1076100043F001031370002004E07846F5F79EFA6A
:10762000EBE70B2002B010BD0B20FBE70B20F9E7C6
:10763000103E002030B583B001900D46040CA4F537
:107640004054A4B2012C01D800230EE07846F5F78F
:1076500085FAF9E704EB4402D018064A02EB8002EF
:107660005268D24345F823200133012BF2D903B0ED
:1076700030BD00BF143E002030B583B001900D46F0
:10768000040CB4F5805F0AD1A4F58054A4B204EBD5
:107690004404054B33F814302B8003B030BD7846DA
:1076A000F5F75CFAF0E700BF843D002010B582B02A
:1076B00001900C46000CB0F5804F04D1044B1B78B0
:1076C000237002B010BD7846F5F748FAF6E700BF20
:1076D000981F0020F8B504460D4616461F4653B1C4
:1076E0002B89B3F5BE7F0AD309233B603868B0FA13
:1076F00080F04009F8BD7846F5F730FAF0E7012C44
:107700000BD9002333B1C4EBC4031B4A02EBC30300
:107710009B8983B105233B60E8E7C4EBC403164AA9
:1077200002EBC30393F8343013F0010F01D10023AF
:10773000E8E70123E6E736B12868FFF75FFEB8B94E
:1077400007233B60D2E7C4EBC4030B4A02EBC3033D
:107750009A884FF6FF739A42F2D0C4EBC404064BEA
:1077600003EBC404E2884FF6FF739A42E4D1E7E7E3
:1077700000233B60BAE700BF9C3D0020F8B50E46F1
:1077800017461D460C4603281AD8DFE800F005020C
:10779000101401EB81004400BDF81800B4FBF0F0B8
:1077A0003F2816D800233B7076B92B70F8BD6420B3
:1077B00000FB01F4F0E741F2707000FB01F4EBE72D
:1077C0007846F5F7CBF9E7E7012838BF01202870A4
:1077D000ECE740F27623984208D801233B7003F18E
:1077E000CC33A3FB0030C0082870DFE741F69C03D0
:1077F000984207D802233B70064BA3FB0030400998
:107800002870D3E703233B70034BA3FB0030C00970
:107810002870CBE71F85EB51F119760530B583B0A1
:1078200001900D46040CA4F50054A4B2012C11D80B
:107830000A4AC4EBC40402EBC40352F834205C6867
:107840009868D9682A606C60A860E9601A692A6142
:1078500003B030BD7846F5F781F9E9E79C3D00209B
:10786000000CA0F5005080B2012846D8294B1B78A7
:1078700013F0040F43D1F0B482B08C89C0EBC00385
:10788000254A02EBC3039B899C423AD10A88C0EB8C
:10789000C003214C34F833309A4236D14C88C0EBC7
:1078A000C0031D4A02EBC3035B889C422FD1CC89E5
:1078B000C0EBC00302EBC303DB899C4201D00B2069
:1078C00020E01346C0EBC00502EBC5020C68D1F8FE
:1078D00004C08F68CE6843F83540C2F804C0976092
:1078E000D6600C69146192F8342003EBC50002F0F5
:1078F000F90380F83430002004E0052070470020B0
:1079000070470B2002B0F0BC70470B20FAE70B2049
:10791000F8E700BF103E00209C3D002038B504462B
:10792000C0884FF6FF73984211D1E389022B4DD0E6
:1079300003EB4303274A02EB83031D1D5A68002310
:107940005AB90133012B13D855F82320F8E703F077
:10795000B7F903460028E8D039E051420A401E49F1
:1079600001FB02F2D20E1D498C5C04EB43140DE0C6
:1079700028240BE062421440174A02FB04F4E40E90
:10798000164A145D04EB431400E02824282C1BD075
:10799000A0B203F02FFA0346C8B90134272CF4D85B
:1079A000630955F8232004F01F04012101FA04F4AF
:1079B00064421440002CDDD10133012B02D855F86C
:1079C0002340F7E72824E1E7002300E000231846DE
:1079D00038BD00BF143E002031B57C07647703003A
:1079E00008B5837C13F0FC0F00D108BD9A0803F0A2
:1079F00003011430FFF766FAF7E700000E4B1B781F
:107A000013F0040F09D10D4A00EB400112F82130A8
:107A100043F0040302F82130704700B583B0084BEF
:107A20001B68019300F54050ADF806000198FCF783
:107A30003BF903B05DF804FB103E0020143E00202B
:107A4000347703001A4B1B7813F0040F0AD000B5EB
:107A500085B0184B1B68019300F54053ADF8063014
:107A6000002317E0144A00EB400112F8213043F0E4
:107A7000020302F82130704700EB4002D1180E4A91
:107A800002EB81025268D24304A901EB830141F861
:107A9000082C0133012BEFD902A90198FCF7D2F889
:107AA00010B905B05DF804FB7846F5F757F8F8E72C
:107AB000103E002034770300143E0020134B1B7847
:107AC00013F0040F09D1124B00EB400203EB42020A
:107AD000537943F002035371704700B583B00D4BE7
:107AE0005B68019300F58053ADF8063000EB400071
:107AF000074901EB40010198FCF7A4F810B903B065
:107B00005DF804FB7846F5F729F8F8E7103E002009
:107B1000843D002034770300144B1B7813F0040FCE
:107B20000BD1134BC0EBC00203EBC20292F834300E
:107B300043F0020382F83430704700B583B00D4B38
:107B40009B68019300F50053ADF80630C0EBC00010
:107B5000074901EBC0010198FCF774F810B903B0B4
:107B60005DF804FB7846F4F7F9FFF8E7103E0020D3
:107B70009C3D00203477030038B500240DE02046FA
:107B8000FFF73CFF2C4905EB450293001A46CB5CFE
:107B900003F0F9038B540134A4B2012C0FD825460D
:107BA00004EB44029300244AD35C13F0040FE6D1A3
:107BB00013F0020FE6D02046FFF744FFE2E700246F
:107BC0000CB1002429E0254604EB44035A001B4B6A
:107BD00013445B7913F0020F0BD1184A05EB4501F2
:107BE0004B0013445A7922F002025A710134A4B2B4
:107BF000E6E72046FFF762FFEFE72046FFF78CFF3E
:107C00000F4AC5EBC501CB00134493F8342022F092
:107C1000020283F834200134A4B2012C0BD825468B
:107C2000C4EBC403DA00064B134493F8343013F06A
:107C3000020FE5D0E1E738BD143E0020843D00206E
:107C40009C3D002000B585B0084B5969186901902A
:107C5000ADF8081001A9D868FBF7F4FF10B905B01A
:107C60005DF804FB7846F4F779FFF8E73477030012
:107C700030B583B004460D460378012B07D0428807
:107C80004FF6FB739A420CD8002003B030BD01A818
:107C900003F002F86388BDF804209B1A2B800120B2
:107CA000F3E700230B800120EFE7000010B57022FE
:107CB000002114480EF006FB134A00231360938042
:107CC000124A136053609360D3601361536113E0F1
:107CD0000C49C3EBC300C2000A444FF6FF70D080CA
:107CE00090800224D4819081C3EBC300C200114470
:107CF00001228A8413449BB2012BE9D9044B04224C
:107D00001A7010BD9C3D0020843D0020143E0020D0
:107D1000981F00202DE9F04FD3B005468846144641
:107D20001F46BDF8709151A802F0B6FFC5EBC50221
:107D3000644B03EBC2039E89BDF846319E4280F03E
:107D4000BA80BDF844311E44B6B23CB3B4F81EA0AC
:107D5000B4F824B04FAB2169E06883E803000CB1AC
:107D6000247F3CB1C5EBC505564800EBC5056C7CCE
:107D7000FF2C28D057B3B9F1000F2BD024220021BB
:107D800046A80EF09FFA4CAA5146584603F094FFBD
:107D9000054618B3284653B0BDE8F08FC5EBC503C0
:107DA000484A02EBC303B3F804A04FA9D88803F0F4
:107DB00067F8002840F08180BDF83E31002B7ED06E
:107DC0004FF6FF7BCBE7404B1C78D3E77846F4F7C0
:107DD000C5FED0E77846F4F7C1FECFE746AB509931
:107DE0004F9883E80300ADF820618DF8224198F8A0
:107DF0000A208DF8232198F80B208DF824214A972A
:107E0000ADF82C91D8F80C204E9200211846F7F7C7
:107E10000FFE05460028BDD12C4B1B6813F4005FF4
:107E200003D02B4B1B68042B20DC284B1B6813F45E
:107E3000005FAFD0264B1B68042BABDDB9F1800F80
:107E400028BF4FF080092B464B451ED2FA5C2149D2
:107E50000C6810095900265C05A800F8136002F0B0
:107E60000F020131A25C42540133EDE71A4BD3F803
:107E70000435B8F800200192184A009240F2A91285
:107E800017490520FAF704F8CFE705AA002302F8FE
:107E9000193003F1804303F58833D3F80435029297
:107EA000104A0192104A00924FF4D5720C490520F5
:107EB000F9F7EEFF6EE710256CE705256AE7102558
:107EC00068E700BF9C3D0020981F0020741F002021
:107ED000701F0020781F002000100140A4760300CE
:107EE0009B760300B8760300A869030008B5054A2D
:107EF000137803F0FE036FF3410313700220FBF7C6
:107F0000FDFE08BD103E00202DE9F04784B0064676
:107F100090461F460C4691B303AB4246214630467D
:107F2000FFF7D8FB78B3236802934FF6FF72B2EBEA
:107F3000134F2CD04FF0030A25895544ADB2284683
:107F4000FCF7D3FA814688B301462068FFF73BFA75
:107F50002289616809EB0A000EF08BF900954B4607
:107F6000424621463046FFF7D5FE0390C8B9C7B157
:107F70000C9BB3B1C7F800900C9B1D8004E07846C1
:107F8000F4F7ECFDC8E7039804B0BDE8F087BDF84E
:107F90000830FF2B02D94FF0020ACDE74FF0010A5B
:107FA000CAE74846FCF7A5FA0398EDE70420EBE79B
:107FB00038B51C4A137843F00403137013F0020F12
:107FC0002CD113F0010F1CD0002401E00134A4B225
:107FD000012C16D8C4EBC403134A02EBC3039A89DD
:107FE0004FF6FF739A42F1D0C4EBC4050E4B03EB7E
:107FF000C5052846FFF792FC90B92846FFF7F0FC2C
:10800000E4E7FFF7B9FD074B1B7813F0010F01D030
:10801000002038BDFFF716FE0020FAE70B20F8E736
:108020000B20F6E7103E00209C3D00202DE9F04F8C
:108030008DB0054600F11404204603F0B9FF10B9D5
:108040000DB0BDE8F08F4FF6FF73ADF82A300AA9E6
:108050002046FFF70DFE099008B100243DE00DF128
:108060002A01204603F000F80028F6D07846F4F7FD
:1080700075FDF2E7BDF82A103846FFF719FA814678
:108080003EE03F4BD3F804353E4AC4EBC40102EB5B
:10809000C10032F8312041880697CDF814B0CDF8F0
:1080A0001090CDF80CA002910192374A00924FF443
:1080B000866236490720F9F7EBFE47E0C4EBC403BC
:1080C000304A02EBC3039A6A0B9902EBC10256686D
:1080D0001A6B2946A0B2B0470134012CB0DCC4EBC6
:1080E000C407284B03EBC707099B002BC2D0B889F4
:1080F000BDF82890814514BF4FF000094FF00109E9
:10810000204AC4EBC40302EBC30393F8348008F0A5
:10811000010AC4EBC403DB0008331344EA8B5109A2
:1081200053F8216002F01F02D64006F0010B0BAAA3
:1081300029683846FFF79EF90746154B1B6813F46C
:10814000005F03D0134B1B68062B9ADCBAF1000FBB
:10815000C2D0B9F1000FBFD0BBF1000FBCD0002FCF
:10816000BAD02B7D012BA9D1C4EBC403054A02EB85
:10817000C3031A6B2946A0B201F07CF99EE700BF49
:10818000001001409C3D0020C07603009B76030058
:10819000741F0020701F00202DE9F041D0B004466C
:1081A000002868D02068FFF7DDF84F9085B27F2D5A
:1081B00000F095804B4B1B6813F4005F03D04A4BD3
:1081C0001B68042B5BDCE06902F0D1FF8046A069EC
:1081D00002F0B6FF4F9B459326684FF6FF72B2EB55
:1081E000134F58D003231E444696A3884F9A0492F7
:1081F0004FF6FF71B1EB124F53D003229B1A9FB27F
:10820000ADF81C71237A8DF820316389ADF82231E5
:10821000E3684993237C8DF82831638AADF82A31CD
:1082200063694B9394F820308DF83031ADF832818A
:10823000636A4D93ADF838012A4B1B6813F4005F55
:108240004AD0294B1B68042B46DD802F28BF80278E
:108250000023BB422BD2F25C24490C681009590060
:10826000255C04A800F8135002F00F020131A25C53
:1082700042540133EDE77846F4F770FC92E71C4B6B
:10828000D3F8043501951B4A0092FD221A490520B6
:10829000F9F7FEFD97E7FF2D01D90223A3E701239C
:1082A000A1E7FF2D01D90222A8E70122A6E704AA2F
:1082B000002302F8173003F1804303F58833D3F825
:1082C000043502920D4A01920D4A00924FF48A72CF
:1082D00009490520F9F7DCFD45A8FFF7A7FE50B0D6
:1082E000BDE8F081741F0020701F0020781F00205F
:1082F00000100140187703009B7603002C770300E1
:10830000A869030008B5037813B1142B04D008BD85
:108310000430FFF741FFFAE7C388022BF7D1034A85
:10832000137843F002031370F1E700BF103E002002
:10833000B1B1F0B585B0064614461D460F468AB168
:1083400093B103AB0022FFF7C5F908B903980CE01D
:1083500000952346002239463046FFF7DBFC04E057
:108360000E2070470E2000E00E2005B0F0BD08B5CD
:1083700001F0CEF8FEF796FDFFF798FCFFF7B6FD8B
:1083800008BD000008B5FFF791FC0948094B0360E0
:10839000F7F752FB01F0A8F8FEF76AFDFEF728FF99
:1083A000054A137803F0FC036FF38203137008BDD2
:1083B000903D002005830200103E0020002800F0C0
:1083C000AF8070B50C460546002900F0AB80C3684D
:1083D0001BB18368002B00F0A7804FF6FF7323804A
:1083E000EB681BB9AB68002B40F0A080AB88002B7A
:1083F00040F09E8003F002FE002841D12246296809
:10840000A888FEF771FF50B12388C3EBC3034B4A22
:1084100002EBC30393F8343013F0010F30D1E96855
:10842000A868FFF716F8002800F0848023884FF62C
:10843000FF72934265D022882969404BC2EBC20289
:1084400003EBC20211632288A968C2EBC20203EBEC
:10845000C2029162E9682288C2EBC20203EBC20247
:10846000918522886969C2EBC20203EBC202916165
:108470002288C2EBC20103EBC1039A82002058E0BC
:108480000F2056E093B223804FF6FF72934253D0F1
:108490002A4EC3EBC30306EBC303DA802388C3EB86
:1084A000C30306EBC3039A802388A988C3EBC303E5
:1084B00006EBC303998123886988C3EBC30306EBEA
:1084C000C303598023882988C3EBC30326F83310DC
:1084D0002388C3EBC30306EBC3035A742988A88817
:1084E000FEF7E2FE2388C3EBC30206EBC20292F85A
:1084F000343043F0010382F834302088FFF70CFB5E
:1085000099E70022012ABED8C2EBC2010B4800EB5A
:10851000C10191F8341011F0010FB3D00132F1E72D
:108520000E2070470E2004E00E2002E0092000E03B
:10853000052070BD0720FCE70420FAE79C3D0020E1
:1085400070B584B051B304460D460022ADF80E203C
:108550000DF10E03009302ABFFF7D6FC0646B0B94F
:10856000C4EBC4030E4A02EBC303DB7C13F0070F1A
:1085700010D0C4EBC401C90010311144BDF80E3055
:108580000093029B2A4603312046FEF743FE304605
:1085900004B070BD0298FBF7ACFFF8E70E26F6E7D3
:1085A0009C3D002059B110B582B014460A4644B132
:1085B000002300932146FFF7A7FC02B010BD0E2058
:1085C00070470E20F9E7000008B501280DD90023F7
:1085D0001BB3272923D8C0EBC003124A02EBC30305
:1085E000DB888B420FD1002008BDC0EBC0030D4AD1
:1085F00002EBC30393F8343013F0010F01D10023D1
:10860000E6E70123E4E7C0EBC002064B03EBC2033D
:10861000D980FFF781FA0020E6E70520E4E707208C
:10862000E2E700BF9C3D00200A46D1B101280AD9EB
:108630000023C3B1C0EBC0000C4B03EBC000C388E8
:10864000138000207047C0EBC003084901EBC3034F
:1086500093F8343013F0010F01D10023E9E701232F
:10866000E7E70E2070470520704700BF9C3D0020C3
:1086700001282AD808B5C0EBC003174A02EBC30390
:1086800093F8343013F0010F21D0C0EBC00302EB9C
:10869000C303DB7C03F0070301F0070293420AD116
:1086A000C0EBC0030C4A02EBC303DA7CC1F3C40382
:1086B000B3EBD20F0DD0C0EBC002074B03EBC203EC
:1086C000D974FFF729FA002008BD0520704705205E
:1086D000FAE70020F8E700BF9C3D0020B1B110B4DC
:1086E000012815D8C0EBC0030B4A02EBC30393F873
:1086F000343013F0010F0DD0C0EBC00002EBC0000E
:10870000C37C0B7000205DF8044B70470E2070474F
:108710000520F8E70520F6E79C3D002081B310B462
:108720000C467AB301281DD900236BB3C0EBC003FC
:10873000174901EBC3039B6943B30B46C0EBC00170
:1087400003EBC101897CC1F301012170C0EBC000C2
:1087500003EBC000837CC3F38503137000205DF836
:10876000044B7047C0EBC003094901EBC30393F806
:10877000343013F0010F01D10023D6E70123D4E7F1
:108780000E2070470E20EAE70520E8E70620E6E71E
:108790009C3D002070B584B0054600238DF80F3055
:1087A0008DF80D300DF10D020DF10F01FFF7B6FF41
:1087B000E8B9114EEC00C5EBC50306EBC3039B8C77
:1087C000009303AB0DF10E029DF80D109DF80F0004
:1087D000FEF7D4FF601BC000103030449DF80C2021
:1087E0009DF80E100430FEF76DFB04B070BD7846A6
:1087F000F4F7B4F9DDE700BF9C3D002001281BD849
:1088000008B5C0EBC003104A02EBC30393F8343041
:1088100013F0010F12D0C0EBC00302EBC3039B693E
:1088200073B179B1C0EBC002074B03EBC20399846B
:10883000FFF7B0FF002008BD052070470520FAE7CC
:108840000620F8E70720F6E79C3D002001283DD8E8
:1088500010B50446C0EBC003224800EBC30393F8F5
:10886000343013F0010F33D0C4EBC40300EBC30367
:108870009B697BB33F2A2FD803292FD8C4EBC403AD
:1088800000EBC3039B7CB2EB930F08D1C4EBC40392
:1088900000EBC3039B7C03F003038B4220D0114801
:1088A000C4EBC40300EBC3039B7C62F38703C4EBFC
:1088B000C40200EBC20061F3010383742046FFF79A
:1088C00069FF2046FFF728F9002010BD05207047FA
:1088D0000520FAE70620F8E70720F6E70720F4E787
:1088E0000020F2E79C3D002010B5044603F086FB13
:1088F00000283FD1012C17D90023002B3CD0C4EB1A
:10890000C4031F4A02EBC303DB89022B36D10020CC
:1089100001282DD800EB40031A4A12F8233013F037
:10892000010F0FD00130F3E7C4EBC403144A02EB8C
:10893000C30393F8343013F0010F01D10023DCE7B7
:108940000123DAE703F0FB0300EB400143F00103EE
:1089500002F8213080B2C4EBC402094B03EBC2031E
:10896000D881FFF76FF82046FFF7D6F8002006E021
:10897000042004E00F2002E0052000E0002010BDEC
:108980009C3D0020143E002070B501281ED9002314
:10899000CBB3C0EBC0031F4A02EBC303DB89022B3E
:1089A00033D0272933D803EB43031B4A02EB83035D
:1089B00004334D0953F8252001F01F0122FA01F478
:1089C00014F0010410D00024204670BDC0EBC00399
:1089D000104A02EBC30393F8343013F0010F01D1B6
:1089E0000023D5E70123D3E7012606FA01F10A4364
:1089F00043F82520C0EBC000064B03EBC000C08944
:108A0000FFF720F8E0E70524DEE70624DCE707248B
:108A1000DAE700BF9C3D0020143E002038B5034635
:108A200001281CD90022CAB3C3EBC3021E4800EBC5
:108A3000C202D289022A33D0272933D802EB42025C
:108A40001A4800EB820204324D0952F8254001F029
:108A50001F0124FA01F010F001000ED138BDC0EB67
:108A6000C002114800EBC20292F8342012F0010F4C
:108A700001D10022D7E70122D5E7012000FA01F158
:108A800024EA010442F82540C3EBC303064A02EB83
:108A9000C303D889FEF7D6FF0020DFE70520DDE716
:108AA0000620DBE70720D9E79C3D0020143E00208C
:108AB00000293FD02DE9F84317468846002A3BD0CD
:108AC000012810D90023002B38D00646C0EBC00087
:108AD0001E4B03EBC000C389022B31D0B7F80090C6
:108AE00000243C800EE0C0EBC003184A02EBC30335
:108AF00093F8343013F0010F01D10023E3E7012391
:108B0000E1E70134272C13D8C6EBC600A5B22946ED
:108B10000E4B03EBC000FEF7CBFC0028F1D03B88E6
:108B200099450FD928F813503B8801333B80E8E77B
:108B3000002008E00E2070470E2004E0052002E02F
:108B4000062000E00920BDE8F88300BF9C3D00201E
:108B500070B5012816D900235BB311292BD8C0EBBF
:108B6000C003DB000833154A13444D0953F8252090
:108B700001F01F0122FA01F414F0010410D00024C6
:108B8000204670BDC0EBC0030C4A02EBC30393F850
:108B9000343013F0010F01D10023DDE70123DBE7BF
:108BA000012606FA01F10A4343F82520FEF7B4FF37
:108BB000E6E70524E4E70724E2E700BF9C3D002048
:108BC00070B50446012814D9002363B311292CD8A9
:108BD000C4EBC403DB000833154A1A444E0952F8AB
:108BE000265001F01F0125FA01F313F001000ED108
:108BF00070BDC0EBC0030E4A02EBC30393F83430E0
:108C000013F0010F01D10023DFE70123DDE701238A
:108C100003FA01F125EA010542F826502046FEF745
:108C20007BFF0020E4E70520E2E70720E0E700BF44
:108C30009C3D0020B1B370B40D46AAB3012805D9FC
:108C400000239BB31688002313800EE0C0EBC00303
:108C5000184901EBC30393F8343013F0010F01D12D
:108C60000023EEE70123ECE70133072B17D8C0EB15
:108C7000C001C90008310F4C21445C0951F824108F
:108C800003F01F04E14011F0010FEDD011888E4276
:108C90000ED925F81130118801311180E4E7002048
:108CA00070BC70470E2070470E20F9E70520F7E7EB
:108CB0000920F5E79C3D002008B501280DD90023C7
:108CC0001BB3112923D8C0EBC003124A02EBC30324
:108CD0009B888B420FD1002008BDC0EBC0030D4A1A
:108CE00002EBC30393F8343013F0010F01D10023DA
:108CF000E6E70123E4E7C0EBC002064B03EBC20347
:108D00009980FEF709FF0020E6E70520E4E7072049
:108D1000E2E700BF9C3D00200A46D1B101280AD9F4
:108D20000023C3B1C0EBC0000C4B03EBC000838831
:108D3000138000207047C0EBC003084901EBC30358
:108D400093F8343013F0010F01D10023E9E7012338
:108D5000E7E70E2070470520704700BF9C3D0020CC
:108D600000B585B08DF8070010F0800F0AD10128FA
:108D70000AD00DF10701054B9869FAF763FF05B0BA
:108D80005DF804FB0720FAE70720F8E734770300D3
:108D9000014B1878704700BF981F00200A46D1B1D8
:108DA00001280AD90023C3B1C0EBC0000C4B03EB70
:108DB000C000037C137000207047C0EBC00308495B
:108DC00001EBC30393F8343013F0010F01D10023FA
:108DD000E9E70123E7E70E2070470520704700BF51
:108DE0009C3D002008B501280FD900232BB381F04A
:108DF00080037E2B23D9C0EBC003124A02EBC303CE
:108E00005B7C8B420FD1002008BDC0EBC0030D4A34
:108E100002EBC30393F8343013F0010F01D10023A8
:108E2000E4E70123E2E7C0EBC002064B03EBC20319
:108E30005974FEF771FE0020E6E70520E4E70720FD
:108E4000E2E700BF9C3D00200A46D1B101280AD9C3
:108E50000023C3B1C0EBC0000C4B03EBC000437C4C
:108E6000137000207047C0EBC003084901EBC30337
:108E700093F8343013F0010F01D10023E9E7012307
:108E8000E7E70E2070470520704700BF9C3D00209B
:108E9000D0B9034600EB40020C4830F812208A4259
:108EA00001D10020704710B5024603EB430002EBEE
:108EB000400422F81010627942F0010262711846F3
:108EC000FEF7FCFD002010BD05207047843D00200A
:108ED00041B148B900EB4000044A32F810200A8042
:108EE000002070470E20704705207047843D002009
:108EF00049B150B900EB4000054B03EB40008378CB
:108F00000B70002070470E2070470520704700BF8F
:108F1000843D002049B150B900EB4000054B03EB04
:108F20004000C3780B70002070470E20704705206A
:108F3000704700BF843D00200A46F9B101280FD9CF
:108F40000023EBB10F49C0EBC00301EBC3035B8807
:108F50005380C0EBC00031F83030138000207047E0
:108F6000C0EBC003074901EBC30393F8343013F09F
:108F7000010F01D10023E4E70123E2E70E2070474F
:108F8000052070479C3D002030B482B001915AB357
:108F9000154658BB4FF6FF731380034601E00133BB
:108FA0009BB2012B1CD8C3EBC302114901EBC202D7
:108FB00092898242F3D1C3EBC30201EBC202518812
:108FC000BDF806209142EAD1C3EBC304084A32F847
:108FD0003410BDF804209142E1D12B80002000E044
:108FE000052002B030BC70470E20FAE70520F8E7F4
:108FF0009C3D002039B3F0B40E4632B338BB17881D
:109000000023138000E00133012B19D81588BD42DD
:109010001FD2C3EBC301104C04EBC10191F8341013
:1090200011F0010FEFD0C3EBC30104EBC10189893B
:109030008142E8D126F81530118801311180E2E72C
:109040000020F0BC70470E2070470E20F9E7052085
:10905000F7E70920F5E700BF9C3D00200A46D1B1A3
:1090600001280AD90023C3B1C0EBC0000C4B03EBAD
:10907000C000036B136000207047C0EBC0030849B9
:1090800001EBC30393F8343013F0010F01D1002337
:10909000E9E70123E7E70E2070470520704700BF8E
:1090A0009C3D0020F8B50446012833D90023002B4D
:1090B0003ED0204EE700C4EBC400C0001030304466
:1090C000002211460430FDF7FDFE204600F05CFA58
:1090D0003D1B06EBC505E88801F03EFE4FF6FF712B
:1090E000E980A980EA7C02F0F8026FF3C702EA7413
:1090F0006974AA7C02F003026FF30102AA74AB7DCB
:1091000003F003036FF30103AB752046FEF704FD84
:109110000020F8BDC0EBC003064A02EBC30393F87E
:10912000343013F0010F01D10023C0E70123BEE763
:109130000520EEE79C3D002011281AD830B583B0F9
:109140000546002404E02046FFF7ACFF0134A4B23A
:10915000012C0BD80DF106012046FFF7DDFD00289C
:10916000F4D1BDF80630AB42F0D1ECE7002003B0FB
:1091700030BD07207047000010B44FF6FF730B801E
:10918000002300E00133012B0ED80C4C2C2202FBF3
:10919000034292F84020002AF4D02C2202FB034222
:1091A000128B8242EED10B8008884FF6FF73C01AF3
:1091B00018BF01205DF8044B704700BF303E00200F
:1091C000134B2C2202FB0030836B124919440023FD
:1091D0004FF6FF70012B1AD810B403E001339BB295
:1091E000012B11D80A4C2C2202FB034292F840209A
:1091F000002AF3D02C2202FB0342926B541A002C5B
:10920000ECDA18461146E9E75DF8044B7047704701
:10921000303E00200087930310B50446204A2C23DB
:1092200003FB002393F84030B3B11D4BB3F870300B
:10923000B3B11B4A2C2303FB0423002183F8401005
:10924000B2F87030013B9BB2A2F8703023B3B2F891
:109250007230A34208D010BD7846F3F77FFCE4E7F4
:109260007846F3F77BFCE4E72046FFF7A9FF0C4BB9
:10927000A3F872004FF6FF73984209D00848B0F87F
:1092800072302C2202FB0303996BF6F787FEE2E7AC
:109290007846F3F763FCF1E70148F6F767FEDAE793
:1092A000303E0020F0B585B005466B4BB3F870300A
:1092B0005BB16A4B01221A7005F57A76664B4FF660
:1092C000FF72A3F87220002491E07846F3F746FC81
:1092D000EFE72C2303FB0423002183F84010B2F8AE
:1092E00070100139A2F8701003A9188BFFF7B6FEB1
:1092F00048B9594A2C2303FB04235F6B01220399CD
:10930000188BB84772E07846F3F728FCF1E7524B28
:10931000A3F872402C2202FB04F202F11801194456
:1093200013440431188BFFF70BF9074640B14C4B3F
:109330001B6813F4005F03D04A4B1B68042B0ADC44
:10934000AFB1082F13D0042F2AD00F2F28D0784682
:10935000F3F704FC15E0444BD3F804350190434A7D
:109360000092832242490520F8F792FDE8E73A4A45
:109370002C2303FB0423DA6B996B1144996352008D
:10938000DA63354A2C2303FB04231A6B9B6BD31A35
:10939000002B2BDA30492C2303FB04139A6325E0BE
:1093A0002D4B2C2202FB0434A36B03F51C434033EA
:1093B000A363294BB3F87030002B49D0264BB3F888
:1093C0007230012B3ED8244AB2F872302C2101FBB6
:1093D00003239B6B5A1B39D41F4BDA601F4B0022AF
:1093E0001A7005B0F0BD1C4BA3F872400134012C7B
:1093F000DFD8194A2C2303FB042393F84030002BB9
:10940000F4D02C2303FB04231B6B9B1B002BFFF6C8
:1094100060AF114A2C2303FB04239B6B9A1B002A89
:10942000FFF675AF0C4AB2F872204FF6FF718A4210
:10943000D9D009492C2000FB0212926B9B1A002BF9
:10944000D4DAD0E77846F3F789FBBCE7EA1AC3E73A
:10945000014B0022DA60C1E7303E00202E3E0020A2
:10946000741F0020701F00200010014004780300CA
:10947000EF77030070B582B004460E46154601280A
:1094800015D8F7F765FB0DF106012046FFF774FECE
:1094900048B1BDF80600134A2C2303FB00239A8D24
:1094A00033889A4207D0F7F797FB02B070BD784631
:1094B000F3F754FBE5E70B4A2C2303FB0023DA8D7B
:1094C00073889A42EFD1FFF7A7FEBDF80630054A30
:1094D0002C2101FB03235B6B002229462046984781
:1094E000E1E700BF303E002010B5064C7422002199
:1094F00020460CF0E7FE044BA360044B00221A70D8
:1095000010BD00BF303E0020A59202002E3E00207C
:1095100070B582B0F7F71CFB1A4BB3F870300BB97B
:1095200000240BE017480023A0F87030F6F71EFD6A
:10953000F6E7022201992846B0470134012C1DD8D4
:10954000104A2C2303FB042393F84030002BF4D063
:1095500010462C2202FB04F3C1180D8B4E6B1833FE
:10956000002118440CF0AEFE01A92846FFF776FD55
:109570000028DED07846F3F7F1FADAE7F7F72CFBAC
:1095800002B070BD303E002010B582B0012803D972
:109590000524204602B010BD0446F7F7D9FA0DF1B4
:1095A00002012046FFF7E8FD18B90524F7F714FB80
:1095B000EFE7BDF80200FFF72FFE01A92046FFF7F5
:1095C0004DFD60B9BDF80230074A2C2101FB032391
:1095D0005B6B02220199204698470024E6E7784613
:1095E000F3F7BCFAEEE700BF303E002003460F4A17
:1095F000126812F0010F0AD00D4A128890420AD365
:109600000B4840880244934207DB002200E000221E
:10961000104622B970470022FAE70122F8E74B8092
:1096200001230B7000234B60F4E700BFA83E00202D
:10963000084200200B88072B07D801334FF6FF7232
:109640000A80072B20D810B40BE00023F6E703EBC9
:1096500083020E4C34F8222082420ED00133072BB5
:109660000ED85A090A4C54F8222003F01F04E24095
:1096700012F0010FEBD10B80F0E70B80012000E02E
:1096800000205DF8044B70470020704780470020A1
:10969000AC3E00204FF6FF730B8000231F2B21D818
:1096A00010B407E00C884FF6FF72944214D00133D7
:1096B0001F2B13D85A090C4C54F8222003F01F0416
:1096C000E24012F0010FEDD0084A32F82320824226
:1096D000EDD10B80012002E00B80E8E700205DF86F
:1096E000044B704700207047A43E0020B03E00208D
:1096F0004FF6FF730B800023092B26D810B407E028
:109700000C884FF6FF72944217D00133092B18D8FA
:109710005A090F4C54F8222003F01F04E24012F0C3
:10972000010FEDD0162202FB03F20A4CA25A82422C
:10973000EBD108330B80012004E003F108020A801A
:10974000E3E700205DF8044B70470020704700BF3E
:1097500084400020884000204FF6FF730B800023D8
:10976000072B23D810B407E00C884FF6FF72944201
:1097700016D00133072B15D85A090D4C54F8222066
:1097800003F01F04E24012F0010FEDD02A2202FB89
:1097900003F2084CA25A8242EBD10B80012002E076
:1097A0000B80E6E700205DF8044B7047002070470F
:1097B000303F0020343F0020F0B4166800231360CF
:1097C00000E00133072B1ED85C09114D55F82440E9
:1097D00003F01F05EC4014F0010FF2D00D4D2A24C8
:1097E00004FB035464888442EBD11568B5420DD064
:1097F0002A2404FB03F4074F3C5B21F8154014684E
:1098000001341460DDE70120F0BC70470020FBE765
:10981000303F0020343F002070B40D6800230B60FF
:1098200000E00133072B17D85A090E4C54F82220B8
:1098300003F01F04E24012F0010FF2D00C68AC42BA
:109840000DD0AC2202FB03F2074EB25A20F81420CE
:109850000A6801320A60E4E7012070BC704700200A
:10986000FBE700BF1C4200202042002030B4450925
:109870001A4C54F8254000F01F05EC4014F0010F7D
:109880002AD0174CAC2505FB004090F8640010B1BD
:1098900014788C4209D010B1187888420ED0137811
:1098A0008B4212D0002030BC70471C788C42F2D121
:1098B00002990A60039A13600120F4E7029A136088
:1098C0000023039A13600120EDE7029B1A60002336
:1098D000039A13600120E6E70020E4E71C42002021
:1098E00020420020B0B110B404460023092B0DD84B
:1098F000162202FB03F208498A5AA24201D0013320
:10990000F4E7162202FB0313181D00E000205DF8A7
:10991000044B70470020704788400020112865D80C
:1099200030B4072831D8354C072830D803465D09B4
:1099300054F8254003F01F0324FA03F313F0010F3A
:1099400056D00C884FF6FF739C4223D00B88072B10
:1099500050D859092A4C54F8211003F01F04E14053
:1099600011F0010F48D0072836D82649AC2404FB53
:10997000031393F86430022B1DD023492A2303FBE1
:1099800000100430106000202EE0204CCCE7A0F145
:109990000803CCE7072806D81B4C2A2303FB004307
:1099A0005B880B80D2E7A0F10803194C162505FB54
:1099B00003435B88F5E714492A2303FB00139B7DCF
:1099C000002BDAD02A2303FB00F010300B460344AF
:1099D00007331360002007E008380D4B162101FB08
:1099E000003004301060002030BC70470520704704
:1099F0000520F9E70820F7E70820F5E7303F0020C9
:109A00001C42002020420020343F002084400020DF
:109A1000884000200A4B23F8210003EB8103002239
:109A2000DA709A704809074A01F01F01012303FA0E
:109A300001F152F820300B4342F82030704700BF4C
:109A4000B03E0020A43E002010B582B001900B462D
:109A5000000CA0F5805081B21F2911D84A0909488D
:109A600050F8224001F01F02D44014F0010403D04A
:109A70000024204602B010BD1888FFF7CBFFF8E79E
:109A80000524F6E7A43E002010B582B001900C46F4
:109A9000000C012809D1082323800A22A2806380B8
:109AA00023812023E38002B010BD7846F3F756F8F7
:109AB000F1E7000010B582B001900C46000C0128BF
:109AC00015D12388082B16D1A3880A2B16D16388B9
:109AD000082B15D12389082B14D1E388202B13D10F
:109AE0000A4A137843F001031370002004E078461B
:109AF000F3F734F8E5E70B2002B010BD0B20FBE7CD
:109B00000B20F9E70B20F7E70B20F5E718420020C0
:109B100010B582B001900C46000C022809D1094B07
:109B20001B6813F0010F08D0074B1B68236002B0BD
:109B300010BD7846F3F712F8F1E77846F3F70EF820
:109B4000F2E700BFA83E00200842002030B583B0F5
:109B500001900D46040CA4F58054A4B21F2C0FD81C
:109B600063090B4A52F8233004F01F02D34013F06C
:109B7000010F09D0074B33F824302B8003B030BDE0
:109B80007846F2F7EBFFEBE77846F2F7E7FFF1E70D
:109B9000A43E0020B03E002010B5044648B10D4B55
:109BA0009C4213D303F2B4439C4206D94FF6FF7094
:109BB0000EE07846F2F7D2FFF1E7A3F2B440201AA4
:109BC000054CA4FB0030C0F34F1001E04FF6FF70CE
:109BD00010BD00BF9442002083BEA02F38B50446BC
:109BE00008B100200FE07846F2F7B8FFF9E7AC23A0
:109BF00003FB00F303F12002144B13440233A3428E
:109C000022D0013080B207281CD81049AC2303FBB6
:109C1000001393F864100029E9D0AC2303FB00F390
:109C200003F12002094B13440233A3420CD0AC23AE
:109C300003FB00F303F14002044B13440333A3423C
:109C4000DFD101E04FF6FF7038BD00BF2042002099
:109C500010B50446A8B10020072818D8174A2A23AF
:109C600003FB00230433A3420FD02A2303FB00F39A
:109C700003F11002114B13440733A34205D0013006
:109C8000EAE77846F2F76AFFE5E780B210BD0C4BD1
:109C90009C420FD3C6339C4202D94FF6FF70F5E7C2
:109CA000A3F1C600201A074CA4FB003000090830BD
:109CB00080B2EBE74FF6FF70E8E700BF343F0020CB
:109CC0008C400020A38B2EBA2DE9F84306460F46A0
:109CD000904699461068002874D0FFF7B9FF441CDD
:109CE00018E06BB13C4A2A2303FB04239B7D3BB164
:109CF0002A2303FB04231B7E7B4013F03F0F49D034
:109D0000354A2A2303FB04235B797B4013F03F0F82
:109D10004ED00134072C57D86509304B53F82550E5
:109D200004F01F03DD4015F0010FF2D02A4A2A2368
:109D300003FB04235B88B342EBD1294AAC2303FB2A
:109D4000062393F86430002BCBD023492A2202FB50
:109D50000412927D002AC4D02A2202FB04125279F6
:109D60007A4012F03F0FBCD12A2202FB0412127E6D
:109D70007A4012F03F0FB4D10B462A2202FB04F4C2
:109D80000A190432C8F80020103423440733C9F8F4
:109D900000301EE02A2303FB04F303F110020E4BF4
:109DA00013440733C8F800300023C9F8003010E02E
:109DB0002A2303FB04230433C8F800300023C9F826
:109DC000003006E00024A5E70023C8F80030C9F8F9
:109DD0000030BDE8F88300BF343F0020303F002052
:109DE0002042002030B583B001900D46000C0228BF
:109DF00008D10E4B1C6814F0010407D00024204643
:109E000003B030BD7846F2F7A9FEF2E72888F5F7EF
:109E100063FC012808D12A68054B1A60034A1368BD
:109E200043F001031360EAE70B24E8E7A83E0020B3
:109E30000842002070B505460C4616464FF6FF73E3
:109E40000B80F5F749FC3070022823D0032841D05D
:109E5000012841D0002070BD03EB8302204931F876
:109E60002220AA4213D00133072B15D821884FF6A0
:109E7000FF729142F0D15A091A4951F8222003F099
:109E80001F01CA4012F0010FE6D12380EBE72380C7
:109E90000120E0E70023E7E70020DCE7124A32F880
:109EA0002320AA4213D001331F2B17D821884FF645
:109EB000FF729142F2D15A090C4951F8222003F065
:109EC0001F01CA4012F0010FE8D12380EBE7238085
:109ED0000120C0E70023E7E70023E5E70020BAE719
:109EE00080470020AC3E0020B03E0020A43E002071
:109EF00030B583B001900D46040CA4F50054A4B213
:109F0000072C19D86309104A52F8233004F01F02B5
:109F1000D34013F0010F13D004EB84040B4B03EB7D
:109F2000840454F8040F6168A268E36828606960DB
:109F3000AA60EB6003B030BD7846F2F70FFEE1E7B0
:109F40007846F2F70BFEE7E7AC3E002080470020A2
:109F5000F0B583B001900D46040CA4F5A044A4B262
:109F6000092C1ED86309134A52F8233004F01F024B
:109F7000D34013F0010F18D00F49162303FB04F44C
:109F80000A19134653F8067F5E689868DB686F60AD
:109F9000AE60E8602B610B5B2B8053886B8003B055
:109FA000F0BD7846F2F7DAFDDCE77846F2F7D6FD49
:109FB000E2E700BF8440002088400020F0B5083B65
:109FC000124E162505FB03F57419D2F800E0D2F8FD
:109FD00004C09768D268C4F806E0C4F80AC0C4F8A0
:109FE0000E70C4F812200022627101222271618079
:109FF00070535809064903F01F0302FA03F351F89E
:10A000002020134341F82030F0BD00BF88400020DD
:10A010008440002030B583B00190000CA0F5A04230
:10A0200092B2092A19D80D4651090D4B53F8214017
:10A0300002F01F0224FA02F212F0010403D00024FD
:10A04000204603B030BDA0F59F40783883B22A1D6A
:10A0500069882888FFF7B2FFF2E70524F0E700BF20
:10A060008440002070B5A1F1200404EB84020F4964
:10A0700001EB8201066845688268C3684E608D60A6
:10A08000CA600B61F7F71AFE60B96109084A04F06B
:10A090001F04012303FA04F452F82130234342F849
:10A0A000213070BD7846F2F759FDEEE78047002079
:10A0B000AC3E002010B582B00190020CA2F5005316
:10A0C0009BB2072B15D808465C090B4951F8244070
:10A0D00003F01F0324FA03F313F0010403D0002458
:10A0E000204602B010BDA2F5FF5291B2FFF7BAFFB1
:10A0F000F6E70524F4E700BFAC3E002070B582B05F
:10A1000001900D46040CA4F54054A4B2072C2BD8A2
:10A110002422002128460CF0D5F86309214A52F880
:10A12000233004F01F02D34013F0010F20D01E494A
:10A13000AC2303FB04F3CA18CB5A2B8092F864308B
:10A14000AB70134653F8026F58689968DB68C5F81E
:10A150000360C5F80700C5F80B10C5F80F3092F87A
:10A1600064304BB902B070BD7846F2F7F7FCCFE728
:10A170007846F2F7F3FCDAE7AC2303FB04F404F1CE
:10A180001003094C1C4454F8020F6168A268E3688C
:10A19000C5F81300C5F81710C5F81B20C5F81F3007
:10A1A000E0E700BF1C42002020420020F0B583B051
:10A1B00001900C46050CA5F58045ADB2072D2AD8B7
:10A1C0002622002120460CF07DF86B091F4A52F828
:10A1D000233005F01F02D34013F0010F1FD01C489D
:10A1E0002A2202FB05F281180B4653F806CF5F685E
:10A1F0009E68DB68C4F805C0C4F80970C4F80D6037
:10A20000C4F81130835A23804B8863808B7D23717F
:10A210004BB903B0F0BD7846F2F7A0FCD0E7784622
:10A22000F2F79CFCDBE702F1100305461D4455F8EC
:10A23000090F6968AA68EB68C4F81500C4F819101A
:10A24000C4F81D20C4F82130E3E700BF303F0020F0
:10A25000343F0020F8B50D4614462D4BAC2202FBCE
:10A2600004F202F16801194413449967064610B9D3
:10A27000284B01221A70AC2101FB04F12031244B40
:10A28000194402312846F7F7DAFCC8BBAC2101FBC0
:10A2900004F178311E4B194404312846F7F7E4FCE9
:10A2A00090BB1B4FAC2000FB04F03A18D5F800E03F
:10A2B000D5F804C0A968EB68C2F802E0C2F806C08D
:10A2C000C2F80A10C2F80E3000F110033B4400211E
:10A2D000C3F80210C3F80610C3F80A10C3F80E1032
:10A2E0003E5282F8641061090B4A04F01F040123F6
:10A2F00003FA04F452F82130234342F82130F8BD28
:10A300007846F2F72BFCC1E77846F2F727FCC8E75E
:10A3100020420020044200201C420020F0B583B0FF
:10A320000190040CA4F54054A4B2072C3CD80E466E
:10A3300063091E4A52F8235004F01F03DD4015F054
:10A34000010503D00025284603B0F0BD31F8030B0A
:10A350002246FFF77FFFB2781549AC2303FB0413B5
:10A3600083F86420002AEED0AC2303FB04F404F14C
:10A3700010030B44304650F813CF47688668C26814
:10A38000C3F802C0C3F80670C3F80A60C3F80E2011
:10A39000403421440331F7F752FC08B90546D2E7AF
:10A3A0007846F2F7DBFBCEE70525CCE71C42002020
:10A3B0002042002030B583B001900D46040C04F516
:10A3C0004054A4B231F8030B2246FFF743FFAB78A9
:10A3D000064AAC2101FB042484F86430044A137853
:10A3E00043F004031370002003B030BD204200206E
:10A3F000184200202DE9F04106460D4610461C4645
:10A400001F4B2A2202FB04F29918D0F80080D0F8E2
:10A4100004E0D0F808C0C768C1F80680C1F80AE0B7
:10A42000C1F80EC0C1F81270103213440022C3F8F4
:10A430000920C3F80D20C3F81120C3F815200531F9
:10A44000F7F7F2FBB8B90E492A2303FB04F3CA1845
:10A45000002010719075CE5255806109094B04F0AF
:10A460001F04012202FA04F453F82120224343F886
:10A470002120BDE8F0817846F2F770FBE3E700BFEA
:10A48000343F0020303F0020F0B583B00190040C31
:10A49000A4F58044A4B2072C40D80E466309204A94
:10A4A00052F8235004F01F03DD4015F0010503D0DE
:10A4B0000025284603B0F0BD23464A1D4988308850
:10A4C000FFF798FF327917492A2303FB04139A7583
:10A4D000002AEED02A2101FB04F101F110031149F9
:10A4E0001944304650F8157F46688268C368C1F841
:10A4F0000970C1F80D60C1F81120C1F8153008319C
:10A50000F7F792FB30B9074B2A2202FB0434237978
:10A51000E375CEE77846F2F721FBF4E70525C8E7B7
:10A52000303F0020343F0020F0B583B001900D464D
:10A53000000C00F50054A4B2072C1AD900F5805085
:10A5400084B2072C3BD801261E4A137843F004033B
:10A55000137023462A1D69882888FFF74BFF27467A
:10A56000194A2A2303FB04239E7526B9002003B051
:10A57000F0BD0026E8E72A2101FB04F4103411465F
:10A580002144284650F8145F44688268C368C1F8C3
:10A590000950C1F80D40C1F81120C1F8153008313B
:10A5A000F7F742FB38B9084B2A2202FB07373B7901
:10A5B000FB750020DBE77846F2F7D0FAF3E70520D9
:10A5C000D5E700BF18420020343F002010B584B00A
:10A5D000084A52F8044B6B4607CA03C31A806946FF
:10A5E0002046F9F72FFB08B904B010BD7846F2F702
:10A5F000B5FAF9E7DC78030030B583B005460C46C0
:10A600000023ADF800304B0952F8233001F01F024F
:10A61000D34013F0010F0CD00123ADF804302C44CB
:10A62000ADF8064069460198F9F70CFB28B903B06C
:10A6300030BD7846F2F792FAEEE77846F2F78EFAF6
:10A64000F5E70000002940D070B582B005461446F9
:10A650000E460DF1070201A9FFF7ECFB2CB99DF89E
:10A660000730032B01D010201DE0012C1DD078B93C
:10A67000BDF804104FF6FF73994228D02846FFF723
:10A68000C9F9144ABDF804104FF48050FFF7B4FF25
:10A69000BDF80430338084B90F4A02EB8303DA78C3
:10A6A0000132DA70002002B070BD9DF80730032B34
:10A6B000DDD0012BDBD01020F5E7074A02EB830346
:10A6C0009A7801329A700020EDE70E20704704203E
:10A6D000E9E700BFA43E0020B03E0020284B1B78D5
:10A6E00013F0040F4AD030B583B0254B1A786FF3BE
:10A6F00082021A70234B1B690193002400E001348D
:10A70000072C18D86309204A52F8233004F01F029E
:10A71000D34013F0010FF2D0A5B205F54053ADF8C8
:10A7200006300198F9F7C0FA174A29464FF440500D
:10A73000FFF762FFE3E7134B5B690193002400E03E
:10A740000134072C18D86309104A52F8233004F05A
:10A750001F02D34013F0010FF2D0A5B205F58043DC
:10A76000ADF806300198F9F79FFA084A29464FF4E8
:10A770008040FFF741FFE3E703B030BD704700BF03
:10A7800018420020DC7803001C420020303F0020EB
:10A790002DE9F04182B007460C4615464E0952F8A5
:10A7A000263001F01F0823FA08F313F0010F15D02B
:10A7B0000123ADF804303C44ADF806400198F9F7A8
:10A7C00073FA78B9012303FA08F255F8263023EA20
:10A7D000020345F8263002B0BDE8F0817846F2F772
:10A7E000BDF9E5E77846F2F7B9F9EBE708B51F28B8
:10A7F00020D84309264A52F8233000F01F02D340E4
:10A8000013F0010F16D0234B03EB80039B7823B981
:10A81000204B03EB8003DB780BB1002008BD1D4B00
:10A82000002223F820201A4A01464FF48050FFF7F7
:10A83000AFFFF2E7A0F1200189B2072923D84B0925
:10A84000154A52F8233001F01F02D34013F0010FD4
:10A850001BD001EB8103114A02EB83039B782BB9D8
:10A8600001EB810302EB8303DB780BB10020D5E71A
:10A8700001EB81039B000020D052074A4FF40050A7
:10A88000FFF786FFF2E70520C8E70520C6E700BF0F
:10A89000A43E0020B03E0020AC3E002080470020B7
:10A8A00008B5054A137803F0FE036FF341031370F4
:10A8B0000120F9F723FA08BD1842002070B50646BA
:10A8C0000D464FF6FF730B8000240BE004EB840071
:10A8D000104B03EB80001022314604300BF096FC45
:10A8E00098B10134072C13D863090B4A52F823306E
:10A8F00004F01F02D34013F0010FE7D12A884FF66E
:10A90000FF739A42EDD12C80EBE72C80012000E010
:10A91000002070BD80470020AC3E0020F0B583B021
:10A920004FF6FF73ADF80630002840D00C461646AF
:10A93000074600293DD00DF10601FFF7BFFFBDF826
:10A94000063003F12005ADB270B94FF6FF729342A5
:10A9500031D029463846FFF785FB184ABDF8061066
:10A960004FF40050FFF748FE258086B9BDF8063049
:10A97000134A03EB830102EB8101C97803EB8303E4
:10A9800002EB83034A1CDA70002003B0F0BDBDF86F
:10A9900006300B4A03EB830102EB8101897803EB5C
:10A9A000830302EB83034A1C9A700020EDE70E201C
:10A9B000EBE70E20E9E70420E7E700BFAC3E00200C
:10A9C0008047002030B583B005460C46486820B16A
:10A9D0000DF10601FFF772FF18B94FF6FF73ADF8DE
:10A9E00006300DF106012846FEF724FEB0B1BDF891
:10A9F000063003EB83030A4A02EB8303DB7863B17F
:10AA0000658002232370BDF8063003EB8302044BFC
:10AA100003EB82030433636000E0002003B030BD29
:10AA20008047002038B505464FF6FF730B800023A2
:10AA30000BE05A09134850F8222003F01F00C240CF
:10AA400012F0010F08D10B8001331F2B12D80C8894
:10AA50004FF6FF729442ECD00B4A32F82320AA4200
:10AA6000F2D1094A02EB8302D278002AECD00B80A3
:10AA7000012006E0F8F7D2FC4088A84214BF00206D
:10AA8000012038BDA43E0020B03E002000B583B0B8
:10AA9000488003230B7000234B604FF6FE739842EF
:10AAA0000ED007D8031D9BB2012B15D8002003B090
:10AAB0005DF804FB4FF6FF7398420DD10120F6E7D5
:10AAC00001A90120F9F7BAFC10B99DF80400EEE7DE
:10AAD0007846F2F743F8F8E701A9FFF7A3FFE6E7A6
:10AAE0000388012B02D0012B24D0704710B4448876
:10AAF000A4F5405292B2072A01D8142904D0012BA0
:10AB000006D05DF8044B7047A4F5C0444480F8E7D4
:10AB10004288A2F580439BB2072BF2D8242905D0A6
:10AB20001429EED1A2F5C0424280EAE7A2F5A04284
:10AB30004280E6E74288A2F580439BB2072BD4D837
:10AB4000242905D01429D0D1A2F5C04242807047F3
:10AB5000A2F5A0424280704708B5094B1B7813F05C
:10AB6000020F0AD113F0010F03D0FFF7B7FD002049
:10AB700008BDFFF72BFD0020FAE70B20F8E700BF28
:10AB80001842002008B500221F2A07D8144B03EBF7
:10AB900082030021D97099700132F5E7002308E0A3
:10ABA00003EB830291000F4A0A440021D170917097
:10ABB0000133072BF4D900230B4A13600B4A1360AF
:10ABC0000B4A13600B4A13600B4A13600B4A136065
:10ABD0000B4A138053800B4A1370FFF761FE08BDC8
:10ABE000B03E002080470020A83E0020A43E002068
:10ABF000AC3E00201C420020303F0020844000205A
:10AC0000084200200442002008B50648064B0360B5
:10AC1000F4F712FF054A137803F0FD036FF3000306
:10AC2000137008BD0C4200206DB7020018420020CE
:10AC300038B5054670B1164B1C6814F0010424D1D8
:10AC40006B8823B12888F4F747FD012806D00B2430
:10AC5000204638BD7846F1F781FFECE728886B88FD
:10AC6000184480B2013880B2F4F736FD0128EED1E5
:10AC7000074A136843F0010313602968054B196004
:10AC800000210220FFF7B8FCE2E70F24E0E700BF55
:10AC9000A83E00200842002010B5044618B1044B1D
:10ACA0001B68236010BD7846F1F758FFF7E700BF37
:10ACB0000842002008B50122FFF7C4FC08BD0000CF
:10ACC0001F2809D843091D4A52F8233000F01F02FB
:10ACD000D34013F0010F11D1A0F120039BB2072B39
:10ACE0001FD85909164A52F8212003F01F0322FAEF
:10ACF00003F313F0010F16D1002300E00123DBB1B1
:10AD00001F2812D920380F4B00EB800203EB820280
:10AD1000927800EB800003EB8000531C83700020CE
:10AD200070470023EBE70123E9E7074B03EB8000C3
:10AD3000837801338370F2E705207047A43E00203A
:10AD4000AC3E002080470020B03E002008B5012224
:10AD5000FFF7E4FD08BD000008B51F2812D843091D
:10AD60001B4A52F8233000F01F02D34013F0010FAA
:10AD700008D0184B03EB80039A78013A9A70FFF7DA
:10AD800035FD08BDA0F120039BB2072B1BD8590944
:10AD9000114A52F8212003F01F0322FA03F313F0A3
:10ADA000010F12D0A0F120030C4A03EB830102EB48
:10ADB0008101897803EB830302EB83034A1E9A70B7
:10ADC000FFF714FDDDE70520DBE70520D9E700BF2D
:10ADD000A43E0020B03E0020AC3E00208047002072
:10ADE00008B50022FFF72EFC08BD08B50022FFF7CA
:10ADF00095FD08BD1F2809D843091D4A52F8233084
:10AE000000F01F02D34013F0010F11D1A0F1200375
:10AE10009BB2072B1FD85909164A52F8212003F07C
:10AE20001F0322FA03F313F0010F16D1002300E0F1
:10AE30000123DBB11F2812D920380F4B00EB800211
:10AE400003EB8202D27800EB800003EB8000531CFE
:10AE5000C370002070470023EBE70123E9E7074BAD
:10AE600003EB8000C3780133C370F2E7052070471D
:10AE7000A43E0020AC3E002080470020B03E0020D1
:10AE8000002938D010B50C461F2813D843091D4A95
:10AE900052F8233000F01F02D34013F0010F09D005
:10AEA000194B33F820004880F4F716FC207000207E
:10AEB000606010BDA0F120039BB2072B1DD859097B
:10AEC000124A52F8212003F01F0322FA03F313F071
:10AED000010F14D020380E4B00EB800233F82220F3
:10AEE000628000EB800003EB80000430606002238E
:10AEF00023700020DDE70E2070470520D9E70520EC
:10AF0000D7E700BFA43E0020B03E0020AC3E0020AA
:10AF10008047002010B582B004461F2809D8430995
:10AF20002B4A52F8233000F01F02D34013F0010FD8
:10AF300011D1A4F120039BB2072B24D85909254A2B
:10AF400052F8212003F01F0322FA03F313F0010F3C
:10AF50001BD1002300E00123BBB369462046FFF765
:10AF60008FFF70BB9DF80030032B10D0022B2AD12D
:10AF7000A4F1200303EB8301174A02EB8102D2788C
:10AF8000AAB9052022E00023E6E70123E4E7134BFA
:10AF900003EB8403DB780BB9052017E00F4A02EBC3
:10AFA0008402013BD3702046FFF720FC0EE00B46E5
:10AFB000094901EB8303013ADA702046FFF716FCDA
:10AFC00004E0002002E00F2000E0052002B010BDE8
:10AFD000A43E0020AC3E002080470020B03E002070
:10AFE000A0B330B4054699B30023184600E00133FE
:10AFF0001F2B10D85A091A4C54F8222003F01F04B2
:10B00000E24012F0010FF2D00A68824222D025F805
:10B0100010300130EBE7002300E00133072B12D89A
:10B020005A09104C54F8222003F01F04E24012F099
:10B03000010FF2D00A6882420FD003F1200225F8F6
:10B0400010200130E9E70860002004E00E2070477E
:10B050000E2000E0092030BC70470920FBE700BF4C
:10B06000A43E0020AC3E002070B330B583B00C4647
:10B07000054659B34088F4F72FFB02280FD0032868
:10B0800004D0012802D0102003B030BD21466888CA
:10B09000FEF700FB08B10020F6E70520F4E74FF6C5
:10B0A000FF73ADF80630686850B10DF10601FFF787
:10B0B00005FC38B1BDF80630203323800020E3E7DB
:10B0C0000E20E1E70520DFE70E2070470E20DBE7CA
:10B0D00002464FF6FF700023072B26D810B406E077
:10B0E0004FF6FF71884216D00133072B15D8590946
:10B0F000114C54F8211003F01F04E14011F0010F2E
:10B10000EED0AC2101FB03F10C4C615A8A42EBD129
:10B1100098B2012302E098B2E6E7002313B15DF88C
:10B12000044B70474FF6FF70F9E7002303B17047F7
:10B130004FF6FF70704700BF1C42002020420020E5
:10B1400018B108B5FEF74AFD08BD4FF6FF7070470D
:10B1500000B583B00DF10601FEF7FEFA20B1BDF88F
:10B16000060003B05DF804FB4FF6FF70F9E718B175
:10B1700008B5FEF76DFD08BD4FF6FF707047000083
:10B180000A4699B1072813D843090B4951F82330CF
:10B1900000F01F01CB4013F0010F0BD02A2303FB5B
:10B1A00000F0064B1B5A1380002070470E2070479A
:10B1B0000520704705207047303F0020343F0020B5
:10B1C00011286AD838B504460D46002967D00728EB
:10B1D00030D84309354A52F8233000F01F02D340DB
:10B1E00013F0010F5DD0324A2A2303FB00235B8852
:10B1F000072B17D82E4A2A2303FB04235B885909FF
:10B200002C4A52F8212003F01F0322FA03F313F013
:10B21000010F0BD0264B2A2000FB043463882B80BF
:10B22000002038BD7846F1F799FCE3E77846F1F75E
:10B2300095FCEFE7A0F1080462091F4B53F8223098
:10B2400004F01F02D34013F0010F2CD01B4A162329
:10B2500003FB04235B88072B17D8184A162303FB2C
:10B2600004235B885909134A52F8212003F01F0375
:10B2700022FA03F313F0010F0BD01048162303FB3F
:10B28000040463882B800020CBE77846F1F766FC46
:10B29000E3E77846F1F762FCEFE7052070470E2000
:10B2A000BFE70520BDE70520BBE700BF303F00201A
:10B2B000343F00201C4200208440002088400020B1
:10B2C000002900F08D8070B5C6B0054614460E46C4
:10B2D000002A00F08780B0F5805F80F085804FF60F
:10B2E000FF731380002305E021884FF6FF7291421F
:10B2F00016D00133072B15D85A093F4951F822209F
:10B3000003F01F01CA4012F0010FEDD0AC2202FB86
:10B3100003F23A498A5A9542EBD12380012302E095
:10B320002380E6E700236BB12088344BAC2202FB7C
:10B3300000301022314602300AF068FF002856D152
:10B34000032052E022884FF6FF739A4251D03146D3
:10B350002846FEF77FFF284A21884FF44050FFF728
:10B360004BF92388AC2101FB03F18831234B1944AD
:10B3700004312846F4F76DFB214B1B6813F4802F32
:10B3800003D0204B1B68062B01DC00202DE000239E
:10B390000F2B0FD8F25C1C490C6810095900255C72
:10B3A00005A800F8135002F00F020131A25C4254CC
:10B3B0000133EDE705AA00238DF8343003F1804313
:10B3C00003F58833D3F804350292104A0192104AEB
:10B3D000009240F627120F490720F6F759FDD4E7EF
:10B3E0000E2070470E2000E0072046B070BD0F20F1
:10B3F000FBE70420F9E700BF1C42002020420020A8
:10B40000741F0020701F0020781F0020AC780300FC
:10B41000A869030093780300072812D843090B4A50
:10B4200052F8233000F01F02D34013F0010F0AD06E
:10B43000074BAC2202FB003090F864300B70002008
:10B440007047052070470520704700BF1C42002050
:10B450002042002000296AD0F8B504460846072C8F
:10B4600067D86309364A52F8233004F01F02D340EC
:10B4700013F0010F5FD0334AAC2303FB042393F88E
:10B48000643073B1012B58D1AC2303FB04F41034A6
:10B4900014441022A01C0AF0B9FE00284AD008204B
:10B4A00048E02849AC2202FB04F202F110030B44ED
:10B4B0009D1CD0F800E0D0F804C08768C668C3F8C7
:10B4C00002E0C3F806C0C3F80A70C3F80E60403249
:10B4D00011440331F6F7B3FB08BBAC2101FB04F1C7
:10B4E0009031184B194404312846F6F7BDFBD0B90A
:10B4F0001448AC2303FB04F3C118012281F8642033
:10B5000003F1A00101440431C05AF3F759FE0C4A7B
:10B5100021464FF44050FFF76FF800200AE07846CC
:10B52000F1F71CFBD9E77846F1F718FBE0E70E20AE
:10B5300070470520F8BD0520FCE70820FAE700BFAA
:10B540001C4200202042002007282CD810B50446B9
:10B550004309174A52F8233000F01F02D34013F07A
:10B56000010F22D0134AAC2303FB002393F864306D
:10B57000012B01D0082010BD1046AC2303FB04F3BF
:10B58000D118022281F8642003F1A00101440431A2
:10B59000C05AF3F715FE064A21464FF44050FFF714
:10B5A0002BF80020E7E7052070470520E3E700BF00
:10B5B0001C42002020420020072800F2A380F8B59A
:10B5C00005464309514A52F8233000F01F02D34088
:10B5D00013F0010F00F098804D4AAC2303FB0023C9
:10B5E00093F864300BB90820F8BDAC2101FB00F1E1
:10B5F000501801F11003134453F8027F5E689C68F1
:10B60000DB68C0F80270C0F80660C0F80A40C0F8F5
:10B610000E3001F12003134440311144CA1C02339F
:10B620002331176856689468D0681F605E609C601C
:10B63000D860103210338A42F3D112781A70344E27
:10B64000AC2000FB05F000F17802324400F19003D9
:10B65000334453F8044F5968D3F808C0DF68546086
:10B660009160C2F80CC017611C69596954619161FD
:10B670003318002483F8644000F1880131442246E5
:10B680000431305AF3F79CFD00E00134072C31D827
:10B690006309204A52F8233004F01F02D34013F00C
:10B6A000010FF2D01C4A2A2303FB04235B88AB4220
:10B6B000EBD12A2303FB04239B7D002BE5D013460B
:10B6C0002A2101FB04F10A4410310B4453F8077F8F
:10B6D0005E689868D96857609660D06011611B8A6F
:10B6E0009382002393750B4AA1B24FF48040FEF77A
:10B6F00083FFCAE7054A29464FF44050FEF77CFF16
:10B70000002071E70520704705206DE71C420020EE
:10B7100020420020303F0020343F002070B5044616
:10B720000D469DF81060FEF737FA4FF6FF7398420A
:10B7300002D02034AC4200D070BD56B10A4AAC23CE
:10B7400003FB002393F86430012BF5D1FFF7FCFED7
:10B75000F2E7054AAC2303FB002393F86430002B87
:10B76000EAD0FFF729FFE7E7204200200378042B07
:10B7700002D0142B10D0704700B583B0037E427EF8
:10B780000092003B18BF0123426981684068FFF7BF
:10B79000C5FF03B05DF804FBC388012B00D07047E0
:10B7A000024A137843F002031370704718420020D6
:10B7B00040B108B541B1FEF72FF808B1002008BD2F
:10B7C0000920FCE70E2070470E20F8E7002A67D01A
:10B7D000F0B5C7B007460C461D461646002B61D093
:10B7E000F3F77AFF01285FD1072C60D86309344A48
:10B7F00052F8233004F01F02D34013F0010F58D049
:10B800000DF58B713846FDF773FF002853D1BDF855
:10B8100016314FF6FF7293424FD0324621463846DA
:10B82000FEF7CCFBBDF816110839264A89B24FF451
:10B83000A040FEF7E1FEBDF816312B80224B1868C0
:10B8400010F4802031D0214B1B68062B01DC002036
:10B850002BE000230F2B0FD8F25C1D490C68100958
:10B860005900255C05A800F8135002F00F020131C1
:10B87000A25C42540133EDE705AA00248DF8344060
:10B88000144BD3F804350292134A0192134A0092E2
:10B8900040F6272212490720F6F7FAFA204604E07C
:10B8A0000E2070470E2000E0102047B0F0BD0520AC
:10B8B000FBE70520F9E70F20F7E70420F5E700BFD5
:10B8C0001C42002084400020741F0020701F0020B4
:10B8D000781F002000100140BC780300A869030015
:10B8E00093780300A0F1080189B2092919D84B09FE
:10B8F0000D4A52F8233001F01F02D34013F0010F1C
:10B9000001D10520704710B5162303FB01F3002475
:10B91000064AD452044A4FF4A040FEF739FF2046AD
:10B9200010BD0520704700BF8440002088400020E3
:10B93000002A6AD0F0B5C7B006460C461D46174629
:10B94000002B64D0072964D84B09374A52F82330BA
:10B9500001F01F02D34013F0010F5CD0B0F5805FFF
:10B960005BD22946FDF7F8FE68B128882F4B2A22C2
:10B9700002FB00301022394606300AF047FC00284E
:10B980004ED103204AE02B884FF6FF72934249D0F4
:10B990003A4621463046FEF72DFD254A29884FF4C8
:10B9A0008040FEF729FE234B186810F4802035D024
:10B9B000214B1B68062B01DC00202FE000230F2BFE
:10B9C0000FD8FA5C1D490C6810095900255C05A8C0
:10B9D00000F8135002F00F020131A25C425401330F
:10B9E000EDE705AA00248DF83440154BD3F8043553
:10B9F0000292144A0192144A009240F676221349A8
:10BA00000720F6F745FA204608E00E2070470E2082
:10BA100004E0052002E0052000E0072047B0F0BD6B
:10BA20000F20FBE70420F9E71C420020343F0020F0
:10BA3000303F0020741F0020701F0020781F00205E
:10BA400000100140CC780300A8690300937803003C
:10BA500000295AD070B504460846072C57D8630908
:10BA60002E4A52F8233004F01F02D34013F0010F86
:10BA70004FD02B4A2A2303FB04235B88294AAC219D
:10BA800001FB032393F86430012B44D1244A2A2379
:10BA900003FB04239B7D6BB12A2303FB04F41034C6
:10BAA00014441022014604F109000AF0AFFB78B3F8
:10BAB00008202DE01A492A2303FB04F3CA180125A4
:10BAC000957510331944066845688268C368C1F8E3
:10BAD0000960C1F80D50C1F81120C1F815300831C6
:10BAE000F6F7A2F868B90E4A2A2303FB04231A7951
:10BAF000DA750A4A21464FF48040FEF77DFD0020AA
:10BB000006E07846F1F72AF8EDE70E2070470520A9
:10BB100070BD0520FCE70820FAE700BF303F002099
:10BB2000343F002020420020072814D808B54309DC
:10BB30000A4A52F8233000F01F02D34013F0010FDD
:10BB400001D1052008BD054A01464FF48040FEF7AB
:10BB50001FFE0020F6E70520704700BF303F0020A1
:10BB6000072873D838B5044643093B4A52F82330B6
:10BB700000F01F02D34013F0010F69D0364B1B6851
:10BB800013B90823002514E05A421340334A02FB3C
:10BB900003F3DB0E324AD35CF4E759420B402F49E2
:10BBA00001FB03F3DB0E2E49CB5C03EB421300E0F9
:10BBB0000823082B18D001350133072BF8D85A0970
:10BBC000254951F8221003F01F03012000FA03F366
:10BBD0005B420B40002BE0D1013203D11E4B53F8E6
:10BBE0002230F7E70823E4E7012D33D0002500E0F9
:10BBF0000135072D19D86B091A4A52F8233005F080
:10BC00001F02D34013F0010FF2D0174A2A2303FB7F
:10BC100005235B88A342EBD1A8B2FFF785FF00287C
:10BC2000E6D07846F0F79AFFE2E7AC2303FB04F393
:10BC30000E4AD35A13B90E4B00221A70064A2146F7
:10BC40004FF44050FEF7A4FD002038BD052070479A
:10BC50000520FAE70F20F8E71C42002031B57C07E9
:10BC60001C790300303F0020343F00202042002098
:10BC700004420020B1B110B50C46AAB1072815D86E
:10BC800043090C4951F8233000F01F01CB4013F059
:10BC9000010F0DD02146FDF78FFD08B1002010BD2A
:10BCA0000920FCE70E2070470E20F8E70520F6E794
:10BCB0000520F4E71C42002010B582B0ADF8060064
:10BCC00032B30B46144604320DF106011846FDF757
:10BCD00025FE90B9BDF806100E4BAC2202FB0132D6
:10BCE00092F86430022B0AD0AC2303FB01F303F17A
:10BCF0002002084B13440233236002B010BDAC2372
:10BD000003FB01F303F14001024B0B440333F3E760
:10BD10000E20F2E72042002010B50C46FFF7D8F9BC
:10BD2000B4B1072816D843090C4A52F8233000F062
:10BD30001F02D34013F0010F0ED0AC2303FB00F021
:10BD400000F120030648184402302060002010BD96
:10BD50000E20FCE70520FAE70520F8E71C4200204A
:10BD600020420020F0B583B0064615460F4669B163
:10BD700085B106F07F06386880B1FDF72FFF4FF6DA
:10BD8000FF73984225D0013084B208E07846F0F77E
:10BD9000E5FEEDE77846F0F7E1FEEAE70024002350
:10BDA0003B602B60072C16D80C4BAC2101FB04F137
:10BDB00001F120021A4440310B44019500970333EE
:10BDC000023231462046FDF751FD20B90134A4B2BC
:10BDD000E8E70024E3E703B0F0BD00BF2042002005
:10BDE000F8B504460E461D46174662B17DB194B1C2
:10BDF0002046FFF7A5F94FF6FF7290420FD10023BE
:10BE00003B602B60F8BD7846F0F7A8FEEEE7784679
:10BE1000F0F7A4FEEBE77846F0F7A0FEE8E72B4644
:10BE20003A463146FDF750FFECE738B504460D467B
:10BE300021B12046FDF756FD286038BD7846F0F761
:10BE40008DFEF6E7F8B5054616460F4639B156B1F0
:10BE50003868002872D0FDF79FFE441C0DE078463C
:10BE6000F0F77CFEF3E77846F0F778FEF0E7012381
:10BE700000E00023002B44D10134072C60D8630973
:10BE8000314A52F8233004F01F02D34013F0010F5F
:10BE9000F2D02E4AAC2303FB042393F864307BB921
:10BEA000002DE4D0AC2101FB04F1883111440822BB
:10BEB000043128460AF0AAF90028DAD10123D9E78B
:10BEC000CDB1AC2101FB04F18831204B194408228B
:10BED000043128460AF09AF978B1AC2101FB04F14B
:10BEE000A0311A4B19440822043128460AF08EF971
:10BEF00028B90123BEE70123BCE70123BAE70023E9
:10BF0000B8E7134B1B783BB1AC2303FB04F30F4A98
:10BF1000D35A8BB9012100E001210C4BAC2202FB6A
:10BF200004F41A1982F874107034234404333B600B
:10BF300092F86430337005E00021EEE700249CE7BE
:10BF400000233B60F8BD00BF1C42002020420020BF
:10BF50000442002038B504460D46F3F7BDFB022825
:10BF60000FD0032808D0012801D0002038BD294671
:10BF70002046FDF73BFBF9E729462046FEF786FD04
:10BF8000F4E729462046FEF71DFDEFE738B50C46DD
:10BF9000054630B129B1054B1A882A805B88238079
:10BFA00038BD7846F0F7DAFDF5E700BF084200201B
:10BFB00000B583B00378022B0CD0032B05D0012BE6
:10BFC00003D0002003B05DF804FB69464088FFF70A
:10BFD000C1FFF7E769464068FEF770FC0028F1D022
:10BFE000BDF8003003EB8303034A02EB8303D878E8
:10BFF000003818BF0120E5E78047002000B583B076
:10C0000001A8FEF749FEBDF80400003818BF012062
:10C0100003B05DF804FB40B1426842B14378083B8D
:10C02000DBB2F62B05D9002070470E2070470E209A
:10C0300070470720704710B5007848B9002404E025
:10C04000E0B200F0A1F80134A4B2FF2CF8D910BD81
:10C0500000F09AF8FBE7000010B5002000F0A4F80B
:10C06000012000F07FF8094C06E07846F0F776FDF5
:10C070002046FFF7E0FF0834054B9C4205D02046E0
:10C08000FFF7C9FF0028F3D0EFE710BDA863030056
:10C09000C06303002DE9F04707468946924698465B
:10C0A0000E4619E06368304610F8021B424601391B
:10C0B000984708340D4DAC420BD06578BD4201D095
:10C0C000FF2DF6D1237872789342EBD0002BE9D084
:10C0D000EFE7337801331E4409EB0A03B34203D977
:10C0E00033780BB1024CE5E7BDE8F087C06303008D
:10C0F000A8630300F0B40546194B1E7CB6FA86F01F
:10C10000400900216B7D063BDBB28B421ADD6A18C9
:10C11000577F4A1C2A44527F4FEA521C104C04EBB2
:10C120008C04646902F01F0224FA02F212F0010F7B
:10C1300002D101373944E5E75B1A9F4209DA301E24
:10C1400018BF012018B1064A936B01339363F0BC0A
:10C150007047034A536B013353630120F7E700BF75
:10C160002048002008B538B10548064B436000233D
:10C17000037000F0FBFE08BD014800F017FFFAE76E
:10C1800020480020F5C002004109064A00F01F00C7
:10C19000012303FA00F052F82130034342F8213022
:10C1A000704700BF3448002010B50446012802D86B
:10C1B000034B1C7410BD7846F0F7D0FCF8E700BFC5
:10C1C0002048002010B5044648B1E36F5BB1E36F2F
:10C1D000D4F89820D4F894102046984710BD78469B
:10C1E000F0F7BCFCF1E77846F0F7B8FCEFE710B5E4
:10C1F0000446037813F0FE0301D0022B05D1237807
:10C2000003F0FE03022B04D010BD7846F0F7A6FC25
:10C21000F5E7A37963F03F03A371F5E710B582B0AA
:10C22000044626E0002002B010BD7846F0F796FCE8
:10C2300024E004F15C00F2F7C7FA08B1012322E020
:10C24000002320E001233BB3616831B1043904F1DC
:10C250005C00F2F7D7FA0023636001A904F15C00E7
:10C26000F2F764FA0028DDD1019B1A1D62600C33DD
:10C2700063626368002BE7D0002BD6D063681B791C
:10C28000FF2BD6D0002362681279002BDAD10AB9CD
:10C290000123D8E70023D6E70120C4E770B505469F
:10C2A000436893B105F1740695F878303BBB6C6830
:10C2B000237933B32379FF2B01D0013B237105F19F
:10C2C000080000F017FE00BB70BD7846F0F746FC92
:10C2D000E8E7335DC0B2325C325533540134E4B226
:10C2E000F3789C42E3D20B48F3F7B2FFF278B0FB4D
:10C2F000F2F302FB1300C3B2A342EAD1EEE700243B
:10C30000EEE77846F0F72AFCD4E77846F0F726FC0B
:10C31000DAE700BF5C48002000230B650B78002B98
:10C3200037D070B50C4691F8403053B9CB6F33B16C
:10C3300001F18000F4F702FDC8B1012300E0002301
:10C34000BBB104F14406256F94F84430DBB2022BF4
:10C350001BD11048F3F77CFF0F4BA3FB00235B0BB3
:10C3600042F2107202FB13032B44F36070BD0023F2
:10C37000E6E72046FFF752FF054610B9002DF5D03D
:10C38000DFE72046FFF78AFFF8E77846F0F7E6FB9D
:10C39000DFE770475C4800205917B7D110B5044655
:10C3A00050F8202C1379013BDBB2FD2B08D9836DAB
:10C3B00033B11368036741675C30F4F79DFC20B923
:10C3C00054F8201C0B7923B110BD7846F0F7C6FB5A
:10C3D000F6E744F8203C043904F13800F2F712FA89
:10C3E000F2E7000008B50248F3F76CFF08BD00BF94
:10C3F0005C48002038B503780BBB0446012303706A
:10C400004368EBB104F14405246F04F51C54103467
:10C4100047F22F539C4219D90E48F3F719FFA4F5A0
:10C420009C44203CB0FBF4F104FB1104F3F7EAFD5B
:10C43000044404F59C4120312846F3F7AFFD38BD94
:10C440005C30F2F7A4F90028F9D0DBE77846F0F782
:10C4500085FBE1E75C48002008B5002300F8443B79
:10C46000F3F784FD08BD30B583B00C46054638B3FC
:10C470001F2C29D804F1110292B201A905F15C0028
:10C48000F2F7E5F820BB019A101DE4B206345473AC
:10C49000137B022161F30303137395F86830C3F330
:10C4A0004003117B63F38611117355F8693FC2F89D
:10C4B0000F30AB88A2F813300023536003B030BDB7
:10C4C0007846F0F74BFBD3E77846F0F747FBD1E728
:10C4D000042801D10020F1E77846F0F73FFBF9E7A7
:10C4E00070B505460C46B9B1B0B12379C3B1237A12
:10C4F00003F0CF036FF3C71323720023A37234F842
:10C50000042C211F05F15C00F2F7DAF82B7813B147
:10C5100095F8443043B170BD7846F0F71FFBE4E76F
:10C520007846F0F71BFBE2E705F144062C6F04F5B3
:10C530001C54103447F22F539C4213D90B48F3F785
:10C5400087FEA4F59C44203CB0FBF4F104FB1104ED
:10C55000F3F758FD044404F59C4120313046F3F7CD
:10C560001DFDD8E77846F0F7F9FAE7E75C480020C8
:10C5700038B504460D4631B128B1291F04F15C00DD
:10C58000F2F740F938BD7846F0F7E8FAF5E770B50C
:10C590000C46064638B131B1E37843B1E378032B5A
:10C5A00009D800250FE07846F0F7D8FAF4E7784686
:10C5B000F0F7D4FAF2E77846F0F7D0FAF1E77846E8
:10C5C000F0F7CCFA0135E378AB4203D9635D272B52
:10C5D000F8D9F4E7EFF3108372B622687267227914
:10C5E00086F8782096F8772086F83C2003B962B662
:10C5F00070BD70B50C460546B8B1B1B1237813F0E3
:10C60000FE0301D0022B14D1EFF3108672B605F1B0
:10C6100068002368AB66A288A379A5F86C208371B3
:10C62000FFF7E5FD06B962B670BD7846F0F796FAF9
:10C63000E4E77846F0F792FAE6E7000038B50C46F2
:10C64000054678B1132C11D9B4F5205F12D84FF4F8
:10C650007A7101FB04F42C6795F844300BB12B7808
:10C6600063B938BD7846F0F779FAEBE77846F0F72A
:10C6700075FAE9E77846F0F771FAE8E7443504F52A
:10C680001C54103447F22F539C4213D90B48F3F734
:10C69000DFFDA4F59C44203CB0FBF4F104FB110445
:10C6A000F3F7B0FC044404F59C4120312846F3F72D
:10C6B00075FCD6E77846F0F751FAE7E75C480020CA
:10C6C00038B50C46054610B185F8284038BD784687
:10C6D000F0F744FAF8E710B504465C30F1F78EFF46
:10C6E000EFF3108272B663680BB10021197102B9C1
:10C6F00062B610BD10B504464FF08053D3F8A03099
:10C7000013F0010304D0BBB97846F0F727FA03E031
:10C7100003786FF34703037022786FF30002234618
:10C7200003F8012B074A1068C4F8010092889A8028
:10C730002046FFF75CFD10BD0378012262F347033A
:10C740000370E9E7A4000010F8B50D4617461E4631
:10C75000044688B182B10A2E12D9B2B2394604F128
:10C760005C00F1F7F4FE04F16800FFF7C3FF44F644
:10C770002063236700230EE07846F0F7EFF9EAE73D
:10C780007846F0F7EBF9E8E7164AD05CE21882F851
:10C7900074000133DBB2022BF6D984F87730002223
:10C7A00084F878201049216325216185032184F8CC
:10C7B0002C10082184F8281004F17401A16384F876
:10C7C0003C300A4B63636262E567094BE36464656E
:10C7D00022702DB12246074904F18000F4F772FA65
:10C7E000F8BD00BF3C790300D6BE898E9DC3020010
:10C7F00019C30200C5C10200084B01225A60DA6069
:10C800004FF0FF32C3F808230022C3F80022044B84
:10C810004FF48062C3F88021704700BF00A0004041
:10C8200000E100E008B5FFF7E7FF194B0022C3F86D
:10C8300040210121C3F840150420C3F81005C3F8B6
:10C840000425C3F80825134A1348C2F86005A0F56B
:10C8500003503838C2F864054FF48060C2F804050C
:10C8600019600B4BD3F84031002BFAD0084B002253
:10C87000C3F84021074A4FF48061C2F80815A2F5B9
:10C88000B832D2F84805D3F84035C01A08BD00BF09
:10C8900000A0004000F0014040A10040044B4FF0D8
:10C8A000FF32C3F80823034B0222C3F880217047EC
:10C8B0000010004000E100E008B5044B1B681BB10C
:10C8C000024A00211160984708BD00BF804800203F
:10C8D00008B5054B1B7803B908BD00F091FE024B6B
:10C8E00000221A70F8E700BF7E48002008B5074B09
:10C8F0001B7803B108BDFFF7D1FF044B01221A706A
:10C90000FFF790FF00F068FEF4E700BF7E480020CC
:10C9100070B5F3F7E9FE00B170BD1D48F3F7E6F816
:10C920000646E0B10468F3F701FF0546F3F7F8FEA9
:10C930001CB1E3686433834213D81CB1E3686433E9
:10C94000AB4212D3B5F5FA7FE6D900F0A7FEE0B905
:10C95000104B1B78002BDFD1F3F730FFDCE70446E8
:10C96000E1E70120F3F73AFFD6E7FFF7B1FF084808
:10C97000F3F7A7F8864202D07846F0F7EFF80023E5
:10C980006361204600F02AF8C6E7FFF7AFFFC3E770
:10C99000704800207D48002008B5F3F787FF0C4B56
:10C9A0001B68C01A00280BDA0020F3F72BFF094B95
:10C9B00000221A60084B1B7833B1F3F7FFFE08BD65
:10C9C0007846F0F7CBF8EFE7FFF7A2FFF7E700BFF5
:10C9D00078480020844800207F48002070B5044635
:10C9E0000120F3F70FFF0D4D2C60FFF757FFFFF706
:10C9F00019FF2B68DA68024409490A60094C0026CD
:10CA00002670094D01222A701A68196990472E7004
:10CA1000237803B970BDFFF7BFFFFBE78448002010
:10CA2000784800206C4800207C48002010B5124B4C
:10CA30001B68B3B19B686BB1104C012323700E4B84
:10CA40001B689A6818699047002323700C4B1B7869
:10CA500023B910BD7846F0F781F8EDE7FFF79CFFAA
:10CA6000F7E7084B1B7813B100F0E8FDF1E77846D3
:10CA7000F0F774F8F8E700BF844800207C480020F5
:10CA80006C4800207E48002008B50948F2F7F2FF04
:10CA90000023084A1360084A1370084A01211170E4
:10CAA000074A1370074A1370074A82F80A3308BD11
:10CAB00070480020844800207E4800207F480020E5
:10CAC0007C4800206C48002000E100E008B50E4BD7
:10CAD0001B780BB1082008BD0C4B18600A4B0122D3
:10CAE0001A70F3F745FE18B1F3F756FE0020F2E78F
:10CAF000F3F74AFE18B1F3F761FE0020EBE7FFF70A
:10CB0000DBFE0020E7E700BF7F48002080480020D0
:10CB100008B5104B1B7803B108BD00F0BFFD30B95C
:10CB20000D48F2F7E3FF48B10123002BF4D0F3F7EF
:10CB3000B3FD0028F0D0F3F72FFEEDE7074B1B689D
:10CB400023B1074B1B781BB10023EEE70023ECE772
:10CB50000123EAE77F480020704800208448002035
:10CB60006C480020064B1B780BB90820704710B5A5
:10CB70000024034B1C70FFF7CBFF204610BD00BF05
:10CB80007F48002010B50446C0B12368D3B1E368E4
:10CB9000E3B1E268154B9A421CD86369A34221D0E5
:10CBA000646104F114011248F2F76FFF114B1B7816
:10CBB000D3B9114B1B688BB1002016E07846EFF714
:10CBC000CDFFE2E77846EFF7C9FFE0E77846EFF7F9
:10CBD000C5FFDEE77846EFF7C1FFDEE7FFF798FF16
:10CBE000002002E0082000E0002010BD6085010068
:10CBF000704800207F4800208448002008B50F4B73
:10CC00001B6863B1F3F7BAFD68B10D4B1B7873B9BC
:10CC10000C4B1B787BB10A4B01221A7008BD784679
:10CC2000EFF79CFFEEE77846EFF798FFEDE77846E1
:10CC3000EFF794FFECE7FFF7AFFEEFE78448002043
:10CC40006C4800207C48002010B5F3F797FD90B1A8
:10CC5000164B1B68D3B15B688BB1154C0123237055
:10CC6000124B1B685A681869904700232370114BB8
:10CC70001B7843B910BD7846EFF770FFE8E77846B8
:10CC8000EFF76CFFE9E7FFF787FEF3E70A4B1B7846
:10CC900043B100F0BFFC00F001FD0028EAD1F3F73A
:10CCA0008DFDE7E77846EFF759FFF2E7844800206B
:10CCB0007C4800206C4800207E48002008B5F3F72F
:10CCC0005DFD18B1084B1B6823B108BD7846EFF72E
:10CCD00045FFF7E7054B1B7813B1F3F76FFDF4E75A
:10CCE000FFF716FEF1E700BF844800207F480020D0
:10CCF00008B5F3F743FD70B1094B1B6813B17846D3
:10CD0000EFF72CFF074B4FF480621A6002221A6083
:10CD1000FFF7FEFD08BD7846EFF720FFECE700BF08
:10CD20008448002000E100E008B5F3F727FDC0B11A
:10CD30000E4B1B6813B17846EFF710FFFFF7C8FDE5
:10CD4000FFF75AFDFFF7AAFD094B01221A61094BB3
:10CD50004FF48062C3F88020BFF34F8FBFF36F8F13
:10CD600008BD7846EFF7FAFEE2E700BF84480020EE
:10CD700000A0004000E100E008B5034B1B7803B9B8
:10CD800008BDFFF799FDFBE77F480020064B074AE7
:10CD9000C3F8602502F50F423C32C3F864254FF416
:10CDA0008062C3F80425704700F001400411004080
:10CDB00070B50446254BD3F81031CBB1234B00227C
:10CDC000C3F81021224D2B7801332B7000F00AFE9E
:10CDD00094F834202B789A420ED39A422BD9226BA6
:10CDE000D05C00F045F9194BD3F8103153BB70BD3E
:10CDF0007846EFF7B3FEE1E7164BD3F84065164BE4
:10CE00001B681E44F3F752FD0546E36A314604F100
:10CE10001C009847F3F74AFD401B502807D500F047
:10CE20001BFEFFF7EBFE002384F83830DFE778467F
:10CE3000EFF794FEF3E7054B0322C3F8002200F05E
:10CE4000E1FDD0E77846EFF789FED0E7001000401B
:10CE50008C48002000A000408848002070B506469D
:10CE60000C46FFF793FF00F0E3F804F1200000F018
:10CE700013F90021A06A00F05FF9236B187800F025
:10CE8000F7F80125174B1D703046F3F767FD164B79
:10CE90001860E269154BC3F804250022C3F810217D
:10CEA0001022C3F80423124A55641D60D2F84405C9
:10CEB0002946284400F04AFD94F83430AB420AD9A0
:10CEC0000A4B0722C3F80022226B064B1B78D05C6A
:10CED00000F0CEF870BD054B0322C3F8002200F02D
:10CEE00091FDF7E78C4800208848002000100040A2
:10CEF00000A0004010B50446C36A13B394F838305C
:10CF00005BBB174B2360174B6360E36994F83400F5
:10CF100094F82420597801F10A03042A15D0124903
:10CF20008A5C03FB02F32E3303FB00F39833E360C8
:10CF30002461012384F838302046FFF723FE38B9F6
:10CF400010BD7846EFF70AFED8E701F10B03E6E7DC
:10CF50007846EFF703FE0020F2E71120F0E700BF6C
:10CF60005DCE0200B1CD02004079030010B5044649
:10CF700068B163687BB12378012B10D8214611F882
:10CF80000C0B094B03EBC000F4F7C2FE10BD784652
:10CF9000EFF7E4FDEDE77846EFF7E0FDEBE77846E5
:10CFA000EFF7DCFDEAE700BF9048002010B504462B
:10CFB00058B12378012B0CD8214611F80C0B074BE4
:10CFC00003EBC000F4F7CFFE10BD7846EFF7C6FDC7
:10CFD000EFE77846EFF7C2FDEEE700BF904800208C
:10CFE00070B506460D4679B1012E11D80F4B53F896
:10CFF00036408CB154F8083C54F8041C2846984735
:10D00000034680B92468F4E77846EFF7A7FDEBE71D
:10D010007846EFF7A3FDE9E7044B03EBC606736818
:10D02000013373600023184670BD00BF9048002094
:10D030000D4B0022C3F8FC2F0122C3F8FC2F40F255
:10D040005B62C3F8382540F20312C3F83425074A5F
:10D05000C3F83C259622C3F84425D3F8502642F065
:10D060000102C3F850267047001000405555550086
:10D0700010B50446272807D8054B1A5D054BC3F8A1
:10D080000825C3F8544510BD7846EFF767FDF3E770
:10D09000487903000010004010B5044688B3237996
:10D0A000052B32D86388002B33D063880233B3F565
:10D0B000817F32D823781F4AC2F80C352379C2F811
:10D0C0001035A37843F0007343F44033C2F81835A9
:10D0D0006388252B25D90823C3F10802120402F422
:10D0E0007022134343F48073124AC2F81435D2F805
:10D0F000143543F48013C2F814352379042B12D06D
:10D1000010BD7846EFF72AFDC9E77846EFF726FD10
:10D11000C8E77846EFF722FDC7E77846EFF71EFD30
:10D12000C8E70623D8E7D2F8143543F08073C2F875
:10D130001435E5E70010004038B504460D46124BA3
:10D14000D3F81835C3F30243032B06D14DB1012D9B
:10D150000FD07846EFF702FD0AE07846EFF7FEFCC5
:10D16000F4E7220E084BC3F824252402C3F81C451B
:10D1700038BD230C03F47F43034AC2F8243524024C
:10D18000C2F82045F4E700BF00100040074B002222
:10D190001A71EFF3108272B65B781BB1044B022157
:10D1A000C3F8001102B962B6704700BFA048002062
:10D1B00000E100E00D4A53790133DBB2537192F87C
:10D1C0002F20934202D3094B00225A71074B0222AF
:10D1D0001A71EFF3108272B65B781BB1044B022117
:10D1E000C3F8001102B962B6704700BFA048002022
:10D1F00000E100E070B483B00646114B1B68ADF847
:10D2000004301B0C8DF80630002203E0002098B19A
:10D210000132D2B28A420ED20023022BF6D8B55C7C
:10D2200002A8C41814F8044CA54202D00133DBB2A2
:10D23000F3E70120EBE7012003B070BC704700BFAB
:10D240007079030010B5FFF7F3FE1C48FFF724FFC9
:10D2500000241B4BC3F830450BE02146FFF76CFF61
:10D260001749D1F830350122A2401343C1F83035B7
:10D270000134072C08D804F10A03124A02EB830395
:10D2800098680028F4D0E8E70D4B0822C3F804237F
:10D290001122C3F800220022C3F8042103F5F03361
:10D2A000094AC3F8602502F5DE424432C3F864251A
:10D2B0004FF48062C3F8042510BD00BFBC480020B5
:10D2C00000100040A04800200411004008B5114B98
:10D2D0009B6813B17846EFF741FC0E483C2200F101
:10D2E00008018430F1F7B3F9031E0CBF01200020C0
:10D2F0000BD1084A926818320749C1F80425003B4F
:10D3000018BF0123034A937008BD02498A6901329C
:10D310008A61F4E7A04800200010004010B51B4BC4
:10D32000D3F850357BB91A4C6379234493F82C0019
:10D33000FFF79EFEE37853B9FFF7C8FF60B9144BBF
:10D3400001221A7110BD7846EFF708FCEBE7FFF7F2
:10D3500079FF0022E270EFE70E4C012161640B4B74
:10D360005960D4F84405084400F016FB00F04AFB6D
:10D370000023C4F84431084B4FF48062C3F8802185
:10D380004FF40033C4F80433D9E700BF0010004065
:10D39000A048002000A0004000E100E008B5074BD5
:10D3A0001B792BB1013BDBB2012B02D8FFF7B6FF93
:10D3B00008BD7846EFF7D2FBFAE700BFA04800208F
:10D3C00010B50C4B01221A610022C3F80C210A4B44
:10D3D000996831B11C4603F18400F1F713FA002378
:10D3E000A360044BD3F85035002BFAD100F034FB86
:10D3F00010BD00BF00100040A048002008B50D4B34
:10D400001B79012B0BD0022B04D083B17846EFF7A8
:10D41000A5FB03E0FFF7D4FFFFF780FF08BDFFF790
:10D4200055FF0028FAD0044B01229A60F6E7FFF777
:10D43000C7FFF3E7A04800200010004008B5094BE3
:10D440001B79012B0AD0022B04D043B17846EFF7A9
:10D4500085FB03E0FFF7B4FFFFF760FF08BDFFF7B0
:10D46000AFFFFBE7A048002008B5114B1B78012B4C
:10D4700005D0022B06D07846EFF770FB01E0FFF7EE
:10D480009FFF08BD0B4BD3F85035032B0CD8DFE8BA
:10D4900003F002080508FFF781FFF2E7FFF7AEFF90
:10D4A000EFE7FFF7CBFFECE77846EFF757FBE8E74E
:10D4B000A048002000100040F8B5344B9C68344B65
:10D4C000D3F800345BB9314A136901331361214643
:10D4D0003048F1F797F92D4B00229A60F8BD251DD1
:10D4E000627E2A4BDB8B9A4204D9284A5369013366
:10D4F0005361ECE7264AD2F848355B426373D2F8B1
:10D500000834224E0A3306EB83039B68A360D2F8EB
:10D51000543503F03F0323731F4BD3F84875384647
:10D52000F3F71CFA6060234653F81B2FC4F80F2052
:10D530009B88A4F81330237EC3F38011A27B61F390
:10D540004702A273C3F303036375F3680133F36007
:10D55000D6F8903213B1394628469847294600201C
:10D56000FFF73EFD60B9627E084C1732A16804F1F6
:10D570008400F1F7A5F8D4F88000F3F781FBAAE75F
:10D58000024881688430F1F73DF9A4E7A048002003
:10D5900000100040244900200080004010B5F2F740
:10D5A00031FD0446094B9A6A596A8A4208D00144FF
:10D5B0000748F2F7F3FC21460648F2F7EFFC10BDEE
:10D5C00003F16800F2F7D2FCF5E700BFA0480020A5
:10D5D00008490020F048002010B5084C0123637072
:10D5E0000023E370FFF72EFE2378022B00D010BD3E
:10D5F0002379002BFBD0FFF791FEF8E7A04800202D
:10D6000008B5034B00225A70FFF7DAFE08BD00BFD1
:10D61000A048002008B5084BD3F80C3113B9FFF728
:10D6200023FF08BD044B0022C3F80C21D3F80C31B2
:10D63000FFF742FFF3E700BF0010004008B50A4BB8
:10D64000D3F8443163B1084B4FF40032C3F80823D8
:10D650000022C3F84421D3F8443100F0C3F908BDD7
:10D660007846EFF77BFAEEE700A0004008B50A4BDA
:10D670001B7823B1084B1B78012B04D008BD7846DA
:10D68000EFF76CFAF6E7FFF789FF034B02221A70F7
:10D69000FFF73EFAF2E700BFA0480020034B1878DE
:10D6A000022814BF00200120704700BFA0480020BE
:10D6B00038B5054698B10C4C291F04F18400F1F7E8
:10D6C000A1F8A37853B1EFF3108372B662781AB160
:10D6D000064A0221C2F8001103B962B638BD784685
:10D6E000EFF73CFAE7E700BFA048002000E100E0C8
:10D6F00000B583B001A90B48F1F718F868B9019992
:10D7000004310120FFF76CFC20B101980430FFF7D1
:10D71000CFFFEFE70198043000E0002003B05DF890
:10D7200004FB00BF2449002008B50248F1F72FF898
:10D7300008BD00BF24490020024B83F820000122CD
:10D74000DA707047A048002038B504460D4688427C
:10D750000FD30F4B9C4210D840F6B7339D4210D9DF
:10D760000C4B9C625D625C67DC651B78022B0CD005
:10D7700038BD7846EFF7F2F9EBE77846EFF7EEF9C8
:10D78000EAE77846EFF7EAF9EAE7FFF707FFEFE79E
:10D7900000007102A048002070B506460C464B1EE2
:10D7A000DBB2022B10D821463046FFF723FD78B1BB
:10D7B000094D2246314605F12C0008F05AFD0023A0
:10D7C0006B7185F82F4070BD7846EFF7C7F9EAE72F
:10D7D0007846EFF7C3F9EBE7A0480020F8B5054617
:10D7E0000C464B1EDBB2072B0FD80A4E06F1300752
:10D7F00020220021384608F065FDA200294638465F
:10D8000008F037FD0123F370F8BD7846EFF7A6F96D
:10D81000EBE700BFA048002000B583B00D4B1B68AC
:10D82000ADF804301B0C8DF80630032101A8FFF77A
:10D83000B3FF094B009301216846FFF7CFFF032098
:10D84000FFF77AFF05480146FFF77EFF03B05DF85A
:10D8500004FB00BF70790300D6BE898E80841E0051
:10D8600038B50546104C4FF425720021204608F0CB
:10D8700029FD4FF4007204F1900104F18400F0F7E7
:10D8800066FEFFF7C9FF082323772523E383074BB1
:10D890002367074BA3650123237023712846F3F701
:10D8A000CFF9C4F8800038BDA04800208DD1020017
:10D8B000B5D10200037813F0020F0AD1064B0278AB
:10D8C000920843EA022301F5A271044A42F821308A
:10D8D00070474FF00313F2E70300130000600040AD
:10D8E00010B400230B600B4B9C780B4804F1A20290
:10D8F00040F832101B799B0003F1804303F5C043CD
:10D9000000EBC20253600123A340C0F804355DF868
:10D91000044B7047344B002000F00140037813F0B3
:10D92000010F12D013F0020F07D09A080123934081
:10D930004FF0A042C2F80C35704703789A080123D3
:10D9400093404FF0A042C2F8083570470F4B5B7907
:10D95000D3B170B505460C460C4B1B7813F0010F84
:10D9600000D170BD094EB1783046FFF7A3FF0849DA
:10D9700001EB84013046FFF7B3FF163504F5A871BB
:10D98000044B43F82150ECE7704700BF344B0020B4
:10D9900040A1004000A000400F4B5B79DBB170B5A7
:10D9A00005460C460C4B5B7813F0010F00D170BD9F
:10D9B000094B5E1C99783046FFF77CFF074901EB65
:10D9C00084013046FFF78CFF163504F5A871044B2F
:10D9D00043F82150EBE77047344B002040A1004052
:10D9E00000A00040054B5B7933B1044B9A780123CA
:10D9F0009340034AC2F80835704700BF344B0020FB
:10DA000000F00140104B5B79E3B110B40F4B0022E2
:10DA1000C3F810210C4BD8780D4900F1A2020D4C2F
:10DA200041F832401B799B0003F1804303F5C0436A
:10DA300001EBC202536001238340C1F804355DF855
:10DA4000044B7047704700BF344B0020001000406B
:10DA500000F00140101100400F4B5B7903B9704793
:10DA600010B50D4CA378012202FA03F3E1788A4045
:10DA700013430A4AC2F80835237903F5A273A2F5C5
:10DA8000C832002142F823102046FFF747FF601CF0
:10DA9000FFF744FF10BD00BF344B002000F00140F1
:10DAA0000369C268934204D88068801A0344581EF0
:10DAB00070479B1A581E70472DE9F8430446884664
:10DAC0001646C5688768A7EB0509914507D94068E0
:10DAD000284408F0CEFB3544E560BDE8F883406893
:10DAE0004A46284408F0C5FBED1B35442A4608EB9E
:10DAF0000901606808F0BDFBE560EEE72DE9F84339
:10DB0000064688461746C5684FF0000918E0641BB2
:10DB1000621EB3685C1B944228BF1446BC4228BFF7
:10DB20003C46706822464146284408F0A2FBA144C6
:10DB3000A0443F1B2544B368AB4209D0F5604FB108
:10DB40003469A542E3D3B268641B1444621EE0E763
:10DB50000025F3E74846BDE8F8830000114B012299
:10DB60001A615A6110499961104ADA614FF40062F2
:10DB70001A6200229A625A62DA6219630C49596386
:10DB8000802199631A64DA635A640A4A1068C3F8F8
:10DB90000700094A92E803001860998020229A71D0
:10DBA000704700BF3C4B002074790300044C0020F8
:10DBB000844B00208079030084790300F8B50F4678
:10DBC0001646184B451C05EB450503EBC50500EB58
:10DBD000400003EBC000C46A012C11D0022C1CD001
:10DBE00014B100242046F8BD2846FFF759FF8642AD
:10DBF000F8D8324639462846FFF75EFF3446F1E74B
